:020000040800F2
:1000000000500020D54F0008D94E0008E14E0008EE
:10001000E94E0008F14E0008F94E0008000000000B
:10002000000000000000000000000000014F000878
:100030000D4F000800000000194F0008254F000870
:100040001D5000081D5000081D5000081D500008DC
:100050001D5000081D5000081D5000081D500008CC
:100060001D5000081D5000081D500008354F0008A5
:100070001D5000081D5000081D5000081D500008AC
:100080001D5000081D5000081D5000081D5000089C
:10009000494F00081D5000081D5000081D50000861
:1000A0001D5000081D5000081D5000081D5000087C
:1000B0001D5000081D5000081D5000081D5000086C
:1000C0001D5000081D5000081D5000081D5000085C
:1000D0001D5000081D5000081D5000081D5000084C
:1000E0001D5000081D5000081D50000800000000B1
:1000F0000000000000000000000000000000000000
:0C01000000000000000000005FF808F1A3
:10010C0010B5054C237833B9044B13B10448AFF345
:10011C0000800123237010BDE001002000000000CE
:10012C00F4EC000808B5034B1BB103490348AFF3CB
:10013C00008008BD00000000E4010020F4EC000881
:10014C00034613F8012B002AFBD1181A013870470B
:10015C0080B400AF124B1B78DBB2002B1BD0104BC2
:10016C0000221A700F4B1B889AB20F4B1A800D4B42
:10017C005B889AB20D4B1A800A4B9B889AB20C4B37
:10018C001A80084BDB889AB20A4B1A80054B1B89E4
:10019C009AB2094B1A8000BFBD4680BC704700BFA5
:1001AC0029020020080200202A0200202C02002034
:1001BC002E020020300200203202002080B483B0D6
:1001CC0000AF0023FB7110E0FB79214A32F81330A9
:1001DC0099B2FB791F4A52F82320FB790A441D4936
:1001EC0041F82320FB790133FB71FB79042BEBD90C
:1001FC00194B1B780133DAB2174B1A70164B1B785C
:10020C00042B20D90023BB7114E0BB79114A52F89E
:10021C002330124AA2FB03239A08BB7991B2104AED
:10022C0022F81310BB790B4A002142F82310BB793A
:10023C000133BB71BB79042BE7D9074B00221A7031
:10024C00084B01221A7000BF0C37BD4680BC7047AA
:10025C00FC0100201402002028020020CDCCCCCCC4
:10026C00080200202902002080B582B000AF0346AE
:10027C003960FB71FB799BB201339BB2396818462C
:10028C0001F0E4F9034618460837BD4680BD80B539
:10029C0082B000AF03460A46FB711346BB80FB7964
:1002AC009BB201339BB2BA881146184601F0EAF9A9
:1002BC00034618460837BD4680BD90B482B000AFE7
:1002CC000446084611461A462346FB710346BB7189
:1002DC000B467B7113463B71FB792F2B06D9FB79AF
:1002EC00392B03D8FB79303BFB710BE0FB79602B8E
:1002FC0006D9FB79662B03D8FB79573BFB7101E0E0
:10030C00002370E0BB792F2B06D9BB79392B03D88E
:10031C00BB79303BBB710BE0BB79602B06D9BB7949
:10032C00662B03D8BB79573BBB7101E000235AE025
:10033C007B792F2B06D97B79392B03D87B79303BF2
:10034C007B710BE07B79602B06D97B79662B03D80C
:10035C007B79573B7B7101E0002344E03B792F2BE9
:10036C0006D93B79392B03D83B79303B3B710BE0F9
:10037C003B79602B06D93B79662B03D83B79573BED
:10038C003B7101E000232EE0FB799AB23B691A80A5
:10039C003B691B881B019AB23B691A803B691A881E
:1003AC00BB799BB213449AB23B691A803B691B8898
:1003BC001B019AB23B691A803B691A887B799BB204
:1003CC0013449AB23B691A803B691B881B019AB291
:1003DC003B691A803B691A883B799BB213449AB2E9
:1003EC003B691A80012318460837BD4690BC7047FC
:1003FC002DE9F043C1B006AF0DF012FB0346002B04
:10040C0000F0C8860DF020FBC7F8E000D7F8E0300C
:10041C00002BC0F2BE86BD4B1B781A46D7F8E030D5
:10042C00D9B2BB4B995400BFB84B1B781A46B84B8A
:10043C001344012118460DF0C9FB0346012BF3D0E0
:10044C00D7F8E0300D2B04D0D7F8E0300A2B40F071
:10045C009986AE4B1B78002B00F09086AC4B1B782A
:10046C00493B242B00F2788601A252F823F000BFFE
:10047C00C706000865110008651100086511000821
:10048C006511000865110008651100086511000868
:10049C006511000865110008651100086511000858
:1004AC006511000865110008651100086511000848
:1004BC006511000865110008651100086511000838
:1004CC006511000865110008651100086511000828
:1004DC0065110008EB06000865110008651100089D
:1004EC00F509000865110008651100086511000880
:1004FC001105000865110008651100086511000858
:10050C00AD07000807F11003824918460DF03CFFB7
:10051C0000BF07F11003052118460DF057FB0346E9
:10052C00012BF6D000217C4803F028FF03469846A7
:10053C000421794803F022FF0346994608217648A6
:10054C0003F01CFF03461C460C21734803F016FFF6
:10055C0003461D460021714803F010FF03461E465A
:10056C0004216E4803F00AFF03467B6008216B48A8
:10057C0003F004FF03463B600C21684803F0FEFEC9
:10058C00034607F1100005933A6804927B680393C5
:10059C000296019500944B46424661490DF0F4FEDB
:1005AC0000BF07F110031846FFF7CAFD03469AB2C5
:1005BC0007F11003114618460DF008FB0346012BFA
:1005CC00EFD0554B1B685B6B7B60534B1B68996B77
:1005DC003960514B1B68DB6B4F4A1268126C4F49E8
:1005EC000968496B4D480068806B4C4C2468E46B7F
:1005FC004A4D2D682D6C07F1100605950494039057
:10060C000291019200933B687A68464930460DF09E
:10061C00BBFE00BF07F110031846FFF791FD034620
:10062C009AB207F11003114618460DF0CFFA0346A3
:10063C00012BEFD03C4B1B781D463C4B1B881E46B8
:10064C003B4B1B881A463B4B1B8819463A4B1B8865
:10065C001C463A4B1B8807F110000393029401913E
:10066C00009233462A4636490DF08EFE00BF07F144
:10067C0010031846FFF764FD03469AB207F1100306
:10068C00114618460DF0A2FA0346012BEFD02D4B64
:10069C001B781A462C4B1B7807F110002B490DF0D8
:1006AC0073FE00BF07F110031F2118460DF08EFAE0
:1006BC000346012BF6D000F061BD07F1100324496D
:1006CC0018460DF061FE00BF07F110030921184612
:1006DC000DF07CFA0346012BF6D000F04FBD0B4B0E
:1006EC001B78022B4AD10A4B5B78302B04D1194B67
:1006FC0000221A7000F042BD054B5B78312B2BD1D8
:10070C00144B01221A7000F039BD00BF34020020D6
:10071C00380200200CED00081803002060030020B4
:10072C0014ED00082CED0008F00300202A02002034
:10073C002C0200202E020020300200203202002069
:10074C0060ED0008560400205404002098ED0008C9
:10075C00B8ED00085804002007F110039B49184617
:10076C000DF012FE00BF07F11003052118460DF025
:10077C002DFA0346012BF6D000F000BD07F1100353
:10078C00924918460DF000FE00BF07F11003052139
:10079C0018460DF01BFA0346012BF6D000F0EEBC08
:1007AC008B4B1B78082B40F0FE808A4B5B78302BF0
:1007BC0040F2E880874B5B78342B00F2E380854B6A
:1007CC005B78303BDAB2834B5A70824B5B7887F89C
:1007DC00DF30804B9B78662B03D1002387F8E73002
:1007EC0019E07C4B9B78622B03D1012387F8E7300F
:1007FC0011E007F11003784918460DF0C5FD00BF54
:10080C0007F11003102118460DF0E0F90346012BF7
:10081C00F6D000F0B3BC6F4BDB782F2B40F2A180ED
:10082C006C4BDB78392B00F29C806A4B1B792F2B9D
:10083C0040F29780674B1B79392B00F29280654B05
:10084C005B792F2B40F28D80624B5B79392B00F258
:10085C008880604B9B792F2B40F283805D4B9B797A
:10086C00392B7ED85B4BDB792F2B7AD9594BDB7923
:10087C00392B76D8574BDB78303BDAB2554BDA70E4
:10088C00544BDB7887F8DE30524B1B79303BDAB2B5
:10089C00504B1A714F4B1B7987F8DD304D4B5B7900
:1008AC00303BDAB24B4B5A714A4B5B7987F8DC30F0
:1008BC00484B9B79303BDAB2464B9A71454B9B794E
:1008CC0087F8DB30434BDB79303BDAB2414BDA71E2
:1008DC00404BDB7987F8DA3097F8DE309BB2FB813E
:1008EC00FB891A46920013445B009BB2FB8197F87C
:1008FC00DD309AB2FB8913449BB2FB81FB891A460B
:10090C00920013445B009BB2FB8197F8DC309AB2E7
:10091C00FB8913449BB2FB81FB891A46920013445A
:10092C005B009BB2FB8197F8DB309AB2FB891344D6
:10093C009BB2FB81FB891A46920013445B009BB26D
:10094C00FB8197F8DA309AB2FB8913449BB2FB8196
:10095C00FA8997F8E71097F8DF30184603F084FD12
:10096C0032E007F110031D4918460DF00DFD00BFD4
:10097C0007F11003132118460DF028F90346012B3B
:10098C00F6D021E007F11003154918460DF0FCFCD8
:10099C0000BF07F11003132118460DF017F9034699
:1009AC00012BF6D0EAE307F110030E4918460DF0BF
:1009BC00EBFC00BF07F110030A2118460DF006F9F5
:1009CC000346012BF6D0D9E3D8E300BFC4ED0008F1
:1009DC003402002038020020CCED0008E0ED0008C5
:1009EC0000EE000814EE0008BB4B1B78012B40F204
:1009FC009B83BA4B5B78722B40F08680B64B1B788E
:100A0C00042B69D1B54B9A78B44BD97807F10C0308
:100A1C0000930B4630213020FFF74FFC0346002B90
:100A2C0042D0BB89DBB207F10E0211461846FFF724
:100A3C001BFC0346A7F8D830B7F8D830002B19D1D7
:100A4C00BB891A46FB8907F11000A5490DF09CFCE7
:100A5C0000BF07F110031846FFF772FB03469AB26A
:100A6C0007F11003114618460DF0B0F80346012BA0
:100A7C00EFD082E3B7F8D82007F110039949184654
:100A8C000DF082FC00BF07F110031846FFF758FB6E
:100A9C0003469AB207F11003114618460DF096F86A
:100AAC000346012BEFD068E307F110038E4918467B
:100ABC000DF06AFC00BF07F110031846FFF740FB6E
:100ACC0003469AB207F11003114618460DF07EF852
:100ADC000346012BEFD050E307F11003834918466E
:100AEC000DF052FC00BF07F110031846FFF728FB6E
:100AFC0003469AB207F11003114618460DF066F83A
:100B0C000346012BEFD038E3744B5B78772B69D11C
:100B1C00714B1B78082B4DD1704B9A786F4BD97851
:100B2C0007F10C0300930B4630213020FFF7C5FB77
:100B3C000346002B37D0694B1879684B5979674BB2
:100B4C009A79664BDC7907F10E0300932346FFF785
:100B5C00B4FB0346002B1FD0BB89DBB2FA891146CC
:100B6C001846FFF794FB0346A7F8D830B7F8D830EF
:100B7C00002B08D1BB891A46FB8907F110005C4990
:100B8C000DF002FC1CE0B7F8D82007F1100359490E
:100B9C0018460DF0F9FB13E007F1100356491846FF
:100BAC000DF0F2FB0CE007F11003544918460DF060
:100BBC00EBFB05E007F11003514918460DF0E4FB7F
:100BCC0000BF07F110031846FFF7BAFA03469AB2B2
:100BDC0007F11003114618460CF0F8FF0346012BE1
:100BEC00EFD0CAE23D4B5B78642B40F0A9803A4BC6
:100BFC001B78022B40F08C80002387F8E63046E00F
:100C0C0007F10E0297F8E63011461846FFF72CFB59
:100C1C000346A7F8D830B7F8D830002B19D197F87D
:100C2C00E620FB8907F1100036490DF0ADFB00BF43
:100C3C0007F110031846FFF783FA03469AB207F13F
:100C4C001003114618460CF0C1FF0346012BEFD0E0
:100C5C0018E0B7F8D82007F110032B4918460DF00F
:100C6C0093FB00BF07F110031846FFF769FA034620
:100C7C009AB207F11003114618460CF0A7FF034671
:100C8C00012BEFD097F8E630013387F8E63097F870
:100C9C00E6301F2BB4D997F8E63003F00303DBB230
:100CAC00002B40F06A8207F11003184918460DF02A
:100CBC006BFB00BF07F110031846FFF741FA034620
:100CCC009AB207F11003114618460CF07FFF034649
:100CDC00012BEFD051E200BF34020020380200207B
:100CEC0020EE000834EE000848EE00085CEE000828
:100CFC0064EE000878EE00088CEE0008A4EE000804
:100D0C00B8EE0008C4EE0008D4EE0008E0EE0008CF
:100D1C0007F110031D4918460DF036FB00BF07F113
:100D2C0010031846FFF70CFA03469AB207F11003AA
:100D3C00114618460CF04AFF0346012BEFD01CE27B
:100D4C00134B5B78782B29D1124B1B78022B04D1D7
:100D5C0000F0D2FC00F01EFD0FE207F110030E496B
:100D6C0018460DF011FB00BF07F110031846FFF7F2
:100D7C00E7F903469AB207F11003114618460CF036
:100D8C0025FF0346012BEFD0F7E100BFE4EE00088E
:100D9C003802002034020020ECEE0008B44B5B78E3
:100DAC00762B40F04C81B34B1B78022B40F02F81FB
:100DBC00B14B1B889C46B14B1B889E46B04B1B8885
:100DCC001A46B04B1B881946AF4B1B881C46AF4BC1
:100DDC001B881D46AE4B1B881E46AE4B1B8807F16D
:100DEC0010000593049603950294019100927346AA
:100DFC006246A9490DF0C8FA00BF07F11003184666
:100E0C00FFF79EF903469AB207F1100311461846F4
:100E1C000CF0DCFE0346012BEFD0A04B1B881946CF
:100E2C009F4B1B881C469F4B1B881A469E4B1B884E
:100E3C0007F110000193009223460A469B490DF0DE
:100E4C00A3FA00BF07F110031846FFF779F9034620
:100E5C009AB207F11003114618460CF0B7FE034680
:100E6C00012BEFD0924B1B881A46924B1B8807F133
:100E7C00100091490DF088FA00BF07F110031846D5
:100E8C00FFF75EF903469AB207F1100311461846B4
:100E9C000CF09CFE0346012BEFD0884B1B881946A7
:100EAC00874B1B881C46874B1B881A46864B1B8816
:100EBC0007F110000193009223460A4683490DF076
:100ECC0063FA00BF07F110031846FFF739F9034620
:100EDC009AB207F11003114618460CF077FE034640
:100EEC00012BEFD07A4B1B8819467A4B1B881C467A
:100EFC00794B1B881A46794B1B8807F1100001931C
:100F0C00009223460A4676490DF03EFA00BF07F1DF
:100F1C0010031846FFF714F903469AB207F11003B1
:100F2C00114618460CF052FE0346012BEFD06D4BC8
:100F3C001B8819466C4B1B881C466C4B1B881A462D
:100F4C006B4B1B8807F110000193009223460A4655
:100F5C0068490DF019FA00BF07F110031846FFF7A6
:100F6C00EFF803469AB207F11003114618460CF03D
:100F7C002DFE0346012BEFD05F4B1B8819465F4BB0
:100F8C001B881C465E4B1B881A465E4B1B8807F160
:100F9C0010000193009223460A465B490DF0F4F9C8
:100FAC0000BF07F110031846FFF7CAF803469AB2C0
:100FBC0007F11003114618460CF008FE0346012BEE
:100FCC00EFD0524B1B881946514B1B881C46514B7A
:100FDC001B881A46504B1B8807F110000193009296
:100FEC0023460A464D490DF0CFF900BF07F1100317
:100FFC001846FFF7A5F803469AB207F110031146FD
:10100C0018460CF0E3FD0346012BEFD0B5E007F1D9
:10101C001003434918460DF0B7F900BF07F1100350
:10102C001846FFF78DF803469AB207F110031146E4
:10103C0018460CF0CBFD0346012BEFD09DE007F1D9
:10104C001003384918460DF09FF900BF07F1100343
:10105C001846FFF775F803469AB207F110031146CC
:10106C0018460CF0B3FD0346012BEFD085E000BF12
:10107C00380200203402002000040020020400206A
:10108C000404002006040020080400200A040020A8
:10109C000C0400200E040020F4EE000810040020C4
:1010AC0012040020140400201604002050EF000845
:1010BC00180400201E04002094EF000820040020D7
:1010CC00220400202404002026040020ACEF000899
:1010DC00280400202A040020380400203A040020B0
:1010EC00E0EF00082C0400202E0400203C0400201B
:1010FC003E04002014F000083004002032040020CC
:10110C00400400204204002048F000083404002071
:10111C003604002044040020460400207CF0000823
:10112C00B0F00008B8F0000807F110031B4918468E
:10113C000DF02AF900BF07F110031846FFF700F86D
:10114C0003469AB207F11003114618460CF03EFD07
:10115C000346012BEFD010E007F11003104918469D
:10116C000DF012F900BF07F11003022118460CF024
:10117C002DFD0346012BF6D000E000BF094B0022E9
:10118C001A7007E0074B1B780133DAB2054B1A7063
:10119C0000E000BFEC37BD46BDE8F083C8F00008A6
:1011AC00DCF000083402002080B59AB000AF2F4B61
:1011BC001A782F4B1B789A4217D02D4B1A782B4B41
:1011CC001A702B4B1B781A463B1D2A4918460DF0FA
:1011DC00DBF83B1D1846FEF7B3FF03469AB2391DE8
:1011EC004FF0FF33244808F0DFFA244B1A88244BC5
:1011FC001B889A4217D0224B1A88204B1A80204BFE
:10120C001B881A463B1D1F4918460DF0BDF83B1DA7
:10121C001846FEF795FF03469AB2391D4FF0FF337F
:10122C00154808F0C1FA184B1A78184B1B789A42DB
:10123C0017D0164B1A78144B1A70144B1B781A468D
:10124C003B1D134918460DF09FF83B1D1846FEF741
:10125C0077FF03469AB2391D4FF0FF33064808F06A
:10126C00A3FA00BF6837BD4680BD00BF9C020020BA
:10127C00F0030020E0F00008A80300209E020020EC
:10128C0054040020F0F00008A002002056040020B6
:10129C0000F1000880B582B000AF03463960FB71E5
:1012AC00FB799BB201339BB23968184600F0CEF93A
:1012BC00034618460837BD4680BD80B582B000AFE6
:1012CC0003460A46FB711346BB80FB799BB2013384
:1012DC009BB2BA881146184600F0D4F9034618465A
:1012EC000837BD4680BD80B483B000AF78607B68A2
:1012FC001B889BB218460C37BD4680BC7047B0B5F6
:10130C0084B000AF78600B467B8004F023FE7B88B2
:10131C0000221C46154622462B467968012004F013
:10132C00A9FD0346FB7304F03BFEFB7B184610370C
:10133C00BD46B0BD80B588B000AF78600023BB60FF
:10134C0004F008FE0023FB607B687B610123BB611A
:10135C0007F1080207F10C031146184604F0E2FEEF
:10136C000346FB7704F01CFEFB7F18462037BD4676
:10137C0080BD80B487B000AF78607B6802337B613E
:10138C007B6803F580633B610CE07B691B88FB8108
:10139C00FB894FF6FF72934201D17B6908E07B69B0
:1013AC0004337B613B69033B7A699A42EDD300239A
:1013BC0018461C37BD4680BC704780B489B000AF5E
:1013CC00F8600B467A607B81FB680233FB61FB683B
:1013DC0003F580637B610223FB7600233B837B68F0
:1013EC00002B18D1012324E0FB691B887B827B8AAC
:1013FC004FF6FF72934214D0FB6902331B883B8279
:10140C007A8A7B899A4203D13B8A3B830023FB7601
:10141C00FB690433FB617B69043BFA699A42E3D9AB
:10142C0000E000BFFB7E002B02D17B683A8B1A8058
:10143C00FB7E18462437BD4680BC704780B500AF94
:10144C000F48FFF777FF0346002B01D0012315E06F
:10145C000C48FFF76FFF0346002B01D001230DE072
:10146C004AF6AA210648FFF74AFF0346002B01D093
:10147C00012303E0044B024A1A600023184680BD86
:10148C0000F8000800FC00080000002080B483B0C5
:10149C0000AF78607B68054A934201D1044B00E0B1
:1014AC00024B18460C37BD4680BC704700F800084C
:1014BC0000FC000880B588B000AF03460A46FB80EC
:1014CC001346BB803C4B1B687B617869FFF7DEFFE2
:1014DC0038613869FFF72EFF0346002B01D001233A
:1014EC0065E045F255513869FFF709FF0346002BBB
:1014FC0001D001235BE03B690233FB6100237B835A
:10150C003CE07B8B2D4A32F81330FB81FA89FB8847
:10151C009A4202D1BB887B810BE007F10A02FB895E
:10152C0019467869FFF749FF03467B737B7B002BD9
:10153C0020D1FB891946F869FFF7E1FE0346002B21
:10154C0001D0012333E0FB6902337A891146184636
:10155C00FFF7D5FE0346002B01D0012327E0FB69E2
:10156C000433FB613B6903F58063FA699A4202D349
:10157C0003231CE000BF7B8B01337B837B8B3F2BD6
:10158C00BFD97869FFF7D6FE0346002B01D00123A3
:10159C000DE04AF6AA213869FFF7B1FE0346002B8D
:1015AC0001D0012303E0044A3B6913600023184671
:1015BC002037BD4680BD00BF0000002018F4000895
:1015CC0080B582B000AF1E48FFF78DFE0346FB804E
:1015DC001C48FFF788FE0346BB80FB884FF6FF7262
:1015EC00934208D1BB884FF6FF72934203D1FFF7A9
:1015FC0025FF034620E0FB884AF6AA22934209D134
:10160C00BB884FF6FF72934204D10F4B0C4A1A6001
:10161C00002311E0BB884AF6AA22934209D1FB8829
:10162C004FF6FF72934204D1074B064A1A6000230F
:10163C0002E0FFF703FF034618460837BD4680BD9E
:10164C0000F8000800FC00080000002080B584B001
:10165C0000AF03463960FB803B68002B01D10123AE
:10166C000AE0074B1B68F9883A681846FFF7A5FE95
:10167C000346FB73FB7B9BB218461037BD4680BDFF
:10168C000000002080B584B000AF03460A46FB8002
:10169C001346BB80174B1B681846FFF76AFEF860B1
:1016AC00FB68002B17D0FB881946F868FFF727FE5C
:1016BC000346002B01D0012317E0FB680233BA88E4
:1016CC0011461846FFF71BFE0346002B01D00123E1
:1016DC000BE0002309E0BA88FB8811461846FFF797
:1016EC00E9FE0346FB72FB7A9BB218461037BD46E7
:1016FC0080BD00BF0000002080B59AB000AF002371
:10170C0087F8673035E097F867301E4A32F81320B7
:10171C0097F8673011461846FFF7CFFD0346A7F838
:10172C006430B7F86430002B0BD197F8672097F82A
:10173C006730144931F81330384613490CF024FE45
:10174C0006E0B7F864203B46104918460CF01CFE26
:10175C003B461846FEF7F4FC03469AB239464FF066
:10176C00FF330B4808F020F897F86730013387F8FF
:10177C00673097F867303F2BC5D900BF00BF68377B
:10178C00BD4680BD98F300080CF1000818F1000864
:10179C00A8030020F0B5B9B006AFBC490020FFF794
:1017AC0079FDBB490120FFF775FDBA490220FFF70F
:1017BC0071FDB9490320FFF76DFDB8490420FFF70F
:1017CC0069FDB7490520FFF765FDB6490620FFF70F
:1017DC0061FDB5490720FFF75DFDB4490820FFF70F
:1017EC0059FDB3490920FFF755FDB2490A20FFF70F
:1017FC0051FDB1490B20FFF74DFDB0490C20FFF70F
:10180C0049FDAF490D20FFF745FDAE490E20FFF70E
:10181C0041FDAD490F20FFF73DFDAC491820FFF706
:10182C0039FDAB491920FFF735FDAA491A20FFF7FE
:10183C0031FDA9491B20FFF72DFDA8491C20FFF7FE
:10184C0029FDA7491D20FFF725FDA6491E20FFF7FE
:10185C0021FDA5491F20FFF71DFDA4492020FFF7FE
:10186C0019FDA3492120FFF715FDA2492220FFF7FE
:10187C0011FDA1492320FFF70DFDA0492420FFF7FE
:10188C0009FD9F492520FFF705FD9E492620FFF7FE
:10189C0001FD9D492720FFF7FDFC9C492820FFF7FF
:1018AC00F9FC9B492920FFF7F5FC9A492A20FFF700
:1018BC00F1FC99492B20FFF7EDFC98492C20FFF700
:1018CC00E9FC97492D20FFF7E5FC96492E20FFF700
:1018DC00E1FC95492F20FFF7DDFC94493F20FFF7F1
:1018EC00D9FC3B46924918460CF04EFD3B46184637
:1018FC00FEF726FC03469AB239464FF0FF338D486B
:10190C0007F052FF614B1B889C46614B1B889E461F
:10191C00604B1B881A46604B1B8819465F4B1B8813
:10192C001C465F4B1B881D465E4B1B881E465E4B40
:10193C001B883846059304960395029401910092F6
:10194C00734662467C490CF01FFD3B461846FEF779
:10195C00F7FB03469AB239464FF0FF33754807F050
:10196C0023FF564B1B881946554B1B881C46554B61
:10197C001B881A46544B1B88384601930092234609
:10198C000A466E490CF000FD3B461846FEF7D8FBA4
:10199C0003469AB239464FF0FF33664807F004FF0E
:1019AC00514B1B881A464F4B1B88384664490CF028
:1019BC00EBFC3B461846FEF7C3FB03469AB239468E
:1019CC004FF0FF335B4807F0EFFE424B1B88194684
:1019DC00414B1B881C46414B1B881A46404B1B88AD
:1019EC0038460193009223460A4656490CF0CCFC2B
:1019FC003B461846FEF7A4FB03469AB239464FF015
:101A0C00FF334C4807F0D0FE384B1B881946384B37
:101A1C001B881C463D4B1B881A463D4B1B88384681
:101A2C000193009223460A4647490CF0ADFC3B4615
:101A3C001846FEF785FB03469AB239464FF0FF3342
:101A4C003C4807F0B1FE2B4B1B8819462A4B1B88D0
:101A5C001C46304B1B881A462F4B1B88384601936B
:101A6C00009223460A4639490CF08EFC3B46184638
:101A7C00FEF766FB03469AB239464FF0FF332D480A
:101A8C0007F092FE1D4B1B88194661E000040020F4
:101A9C000204002004040020060400200804002096
:101AAC000A0400200C0400200E0400204C0400202A
:101ABC004E0400205004002052040020100400208A
:101ACC001204002014040020160400201C04002022
:101ADC001A040020200400202204002024040020EA
:101AEC00260400201E0400201804002028040020D6
:101AFC002A0400202C0400202E0400203004002096
:101B0C003204002034040020360400203804002065
:101B1C003A0400203C0400203E0400204004002035
:101B2C004204002044040020460400204804002005
:101B3C002CF10008A803002034F1000890F10008F3
:101B4C00D4F10008ECF1000820F2000854F200086F
:101B5C001F4B1B881C461F4B1B881A461E4B1B8891
:101B6C0038460193009223460A461C490CF00CFCA3
:101B7C003B461846FEF7E4FA03469AB239464FF054
:101B8C00FF33174807F010FE164B1B881946164BEF
:101B9C001B881C46154B1B881A46154B1B88384650
:101BAC000193009223460A4612490CF0EDFB3B468A
:101BBC001846FEF7C5FA03469AB239464FF0FF3382
:101BCC00074807F0F1FD00BFCC37BD46F0BD00BFA4
:101BDC0032040020400400204204002088F2000857
:101BEC00A803002034040020360400204404002004
:101BFC0046040020BCF2000880B582B000AF7C4BDC
:101C0C001B780133DAB27A4B1A70794B1B78092B9B
:101C1C0040F2E781764B00221A70764B1B78DBB2D0
:101C2C00002B06D0734B1B78DBB2013BDAB2714B45
:101C3C001A70714B1B78DBB2002B06D06E4B1B78E5
:101C4C00DBB2013BDAB26C4B1A706C4B1B78DBB21B
:101C5C00002B06D0694B1B78DBB2013BDAB2674B29
:101C6C001A70674B1B780133DAB2654B1A70644BF0
:101C7C001B7803F00303DAB2614B1A704FF4804106
:101C8C00604804F07BFC0346002B0CD15C4B1B78AA
:101C9C001A465D4B9B5C5A4A127843F00103D9B249
:101CAC00594B99540BE0564B1B781A46564B9B5C80
:101CBC00534A127823F00103D9B2534B99544FF481
:101CCC000041504804F05AFC0346002B0CD14C4BFD
:101CDC001B781A464C4B9B5C494A127843F0020322
:101CEC00D9B2494B99540BE0454B1B781A46464BDD
:101CFC009B5C434A127823F00203D9B2424B9954AD
:101D0C004FF48051414804F039FC0346002B0CD1B0
:101D1C003B4B1B781A463C4B9B5C394A127843F080
:101D2C000403D9B2384B99540BE0354B1B781A4647
:101D3C00354B9B5C324A127823F00403D9B2324BF8
:101D4C0099544FF40051314804F018FC0346002B11
:101D5C000CD12B4B1B781A462B4B9B5C284A1278C8
:101D6C0043F00803D9B2284B99540BE0244B1B7851
:101D7C001A46254B9B5C224A127823F00803D9B2F1
:101D8C00214B99544FF48041204804F0F7FB034653
:101D9C00002B0CD11A4B1B781A461B4B9B5C184A18
:101DAC00127843F01003D9B2174B99540BE0144B33
:101DBC001B781A46144B9B5C114A127823F01003C3
:101DCC00D9B2114B99544FF40041104804F0D6FB92
:101DDC000346002B1CD10A4B1B781A460A4B9B5C02
:101DEC00074A127843F02003D9B2074B99541BE0F1
:101DFC005A040020040000200500002006000020EA
:101E0C005B040020001001405C040020000C014029
:101E1C00764B1B781A46764B9B5C744A127823F0EF
:101E2C002003D9B2724B9954714B1A78704B5B7872
:101E3C001340DAB26E4B9B781340DAB26C4BDB7802
:101E4C001340DAB26B4B1B781343DAB2694B1A703E
:101E5C00674B1A78664B5B781343DAB2644B9B780A
:101E6C001343DAB2624BDB781343DAB2614B1B7863
:101E7C001340DAB25F4B1A70FEF7A0F95E4B1B7879
:101E8C000133DAB25C4B1A705B4B1B78092B40F2B6
:101E9C00A880594B00221A700023FB7113E0FB79C8
:101EAC00564A32F813309BB2002B09D0FB79534AB7
:101EBC0032F8132092B2013A91B2504A22F8131020
:101ECC00FB790133FB71FB79032BE8D94C4B1B8855
:101EDC009BB24FF6FF72934206D0494B1B889BB2C4
:101EEC0001339AB2464B1A80464B1B889BB2002B8F
:101EFC0006D0444B1B889BB2013B9AB2414B1A80D3
:101F0C00414B1B78DBB2012B27D1404B1B78002BAC
:101F1C0011D03F4B1B78042B06D900224FF40051F3
:101F2C003C4804F042FB4FE001224FF40051394889
:101F3C0004F03BFB48E0364B1B78042B06D90022FF
:101F4C004FF48071344804F030FB3DE001224FF433
:101F5C008071314804F029FB36E02B4B1B78DBB247
:101F6C00022B2BD1294B1B78002B13D0284B1B7821
:101F7C0003F00203002B06D000224FF40051254839
:101F8C0004F013FB20E001224FF40051214804F02F
:101F9C000CFB19E01E4B1B7803F00203002B06D040
:101FAC0000224FF480711C4804F0FFFA0CE001226F
:101FBC004FF48071184804F0F8FA05E000224FF451
:101FCC008071154804F0F1FA114B1B780133DAB229
:101FDC000F4B1A700E4B1B78092B02D90C4B00229D
:101FEC001A7000BF0837BD4680BD00BF5B040020DF
:101FFC005C040020F003002060040020F4030020A7
:10200C00FC030020FE03002057040020580400208D
:10201C0061040020001001400008014080B500AFB1
:10202C00AA4B1B7803F00103002B13D0A84B1B7891
:10203C00DBB2002B07D1A74B1B8843F001039AB2EC
:10204C00A44B1A802FE001224FF40051A24804F057
:10205C00ACFA28E09F4B1B8803F00103002B0DD03A
:10206C009C4B1B8823F001039AB29A4B1A800022D6
:10207C004FF40051984804F098FA11E0944B1B78F7
:10208C00DBB2BE2B0CD8934B1B8843F002039AB2E5
:10209C00904B1A8000224FF400518F4804F085FABF
:1020AC008B4BC8221A70894B1B7803F00203002B50
:1020BC000CD08A4B1B78DBB2002B24D1854B1B88B0
:1020CC0043F004039AB2834B1A801CE0814B1B88AB
:1020DC0003F00403002B07D07E4B1B8823F0040372
:1020EC009AB27C4B1A800BE07C4B1B78DBB2BE2B7C
:1020FC0006D8784B1B8843F008039AB2754B1A80AC
:10210C00764BC8221A70734B1B8803F00F039AB2DC
:10211C00704B1A806F4B1B88002B40F0D4806B4B9C
:10212C001B7803F03C03302B00F2BB8001A252F869
:10213C0023F000BF05220008AF220008AF220008E0
:10214C00AF22000861220008AF220008AF2200086D
:10215C00AF22000813220008AF220008AF220008AB
:10216C00AF22000895220008AF220008AF22000819
:10217C00AF2200082D220008AF220008AF22000871
:10218C00AF220008AF220008AF220008AF220008DF
:10219C00AF220008AF220008AF220008AF220008CF
:1021AC00AF220008AF220008AF220008AF220008BF
:1021BC00AF22000847220008AF220008AF22000817
:1021CC00AF220008AF220008AF220008AF2200089F
:1021DC00AF220008AF220008AF220008AF2200088F
:1021EC00AF220008AF220008AF220008AF2200087F
:1021FC00AF2200087B220008394B64221A70354B41
:10220C0000221A805FE0364B1B78DBB2002B4FD1DB
:10221C00304B1B8843F010039AB22E4B1A8047E0C8
:10222C002F4B1B78DBB2002B44D12A4B1B8843F07D
:10223C0020039AB2274B1A803CE0294B1B78DBB267
:10224C00002B39D1234B1B8843F480739AB2214B5A
:10225C001A8031E0224B1B78DBB2002B2ED11D4BA8
:10226C001B8843F400739AB21A4B1A8026E01C4B5D
:10227C001B78DBB2002B23D1164B1B8843F48063F5
:10228C009AB2144B1A801BE0154B1B78DBB2002B57
:10229C0018D1104B1B8843F400639AB20D4B1A8073
:1022AC0010E00F4B64221A700A4B00221A800AE0CD
:1022BC0000BF08E000BF06E000BF04E000BF02E082
:1022CC0000BF00E000BF00BF80BD00BFF0030020D6
:1022DC0004000020540400200010014005000020E0
:1022EC000600002080B584B002AFA84B1B78182BD9
:1022FC0000F2238601A252F823F000BF6D230008E0
:10230C00252400086F240008B924000803250008C0
:10231C004D250008DD250008272600087126000839
:10232C00BB260008052700084D2700089527000844
:10233C00DD2700085128000899280008E12800082A
:10234C002929000891290008FB290008712A000896
:10235C00132E0008F92A0008A92D0008752E000874
:10236C008B4B1B8803F00103002B14D0894B0222EA
:10237C001A70894B00221A80844B12221A70874BD8
:10238C0000221A7001F064F901F034FA01F004FB38
:10239C0001F0D6FB0BE07E4B1B8803F00203002BF5
:1023AC0005D07E4B00221A70784B13221A707C4B8E
:1023BC001A887C4B1B889A4220D9784B1B7883F067
:1023CC000103DBB2002B19D001224FF400417648F7
:1023DC0004F0EBF8754B1B889BB2002B1AD16D4B9C
:1023EC0001221A70694B17221A7001F07DFC01F062
:1023FC004DFD01F01DFE01F0EFFE0BE000224FF44D
:10240C000041694804F0D1F8694B1A88674B1A806F
:10241C0000F093BD00F091BD664B1B88DAB2664BA1
:10242C001B88D9B2654B1B88DBB20A200190009344
:10243C000B460021012002F009FB574B1B889AB276
:10244C005F4B1B889A4202D3504B11221A705D4B82
:10245C001B78002B40F042854C4B02221A7000F086
:10246C003DBD544B1B88DAB2534B1B88D9B2534B2E
:10247C001B88DBB20A20019000930B46002101203F
:10248C0002F0E4FA444B1B889AB24D4B1B889A42DB
:10249C0002D33E4B11221A704A4B1B78002B00F0D2
:1024AC001F853A4B11221A7000F01ABD414B1B8844
:1024BC00DAB2414B1B88D9B2404B1B88DBB20A20E5
:1024CC00019000930B460121012002F0BFFA324B20
:1024DC001B889AB23A4B1B889A4202D32B4B11227F
:1024EC001A70384B1B78002B40F0FC84274B0422CD
:1024FC001A7000F0F7BC2F4B1B88DAB22E4B1B88DE
:10250C00D9B22E4B1B88DBB20A20019000930B46EC
:10251C000121012002F09AFA1F4B1B889AB2284B1A
:10252C001B889A4202D3194B11221A70254B1B7827
:10253C00002B00F0D984154B11221A7000F0D4BC7A
:10254C001C4B5B88DAB2204B1B88D9B21B4B1B8807
:10255C00DBB20A20019000930B460021022002F00E
:10256C0075FA0D4B1B889AB2184B1B889A4202D3F2
:10257C00064B11221A70134B1B78002B40F0B684BB
:10258C00024B06221A7000F0B1BC00BF56040020AA
:10259C005404002057040020FC03002059040020A0
:1025AC00320200201C04002000080140FE03002021
:1025BC001A0400204C040020200400201E040020DB
:1025CC0010040020F003002022040020120400203C
:1025DC00914B5B88DAB2914B1B88D9B2904B1B881C
:1025EC00DBB20A20019000930B460021022002F07E
:1025FC002DFA8C4B1B889AB28B4B1B889A4202D3B8
:10260C008A4B11221A708A4B1B78002B00F07084B5
:10261C00864B11221A7000F06BBC7F4B5B88DAB2D0
:10262C007E4B1B88D9B27E4B1B88DBB20A200190F3
:10263C0000930B460121022002F008FA794B1B880B
:10264C009AB2794B1B889A4202D3784B11221A709A
:10265C00774B1B78002B40F04D84744B08221A707A
:10266C0000F048BC6C4B5B88DAB26C4B1B88D9B25F
:10267C006B4B1B88DBB20A20019000930B460121A7
:10268C00022002F0E3F9674B1B889AB2664B1B8859
:10269C009A4202D3654B11221A70654B1B78002BA2
:1026AC0000F02A84614B11221A7000F025BC5A4BA1
:1026BC009B88DAB25F4B1B88D9B2594B1B88DBB2B3
:1026CC000A20019000930B460021032002F0BEF972
:1026DC00544B1B889AB2584B1B889A4202D3534BCB
:1026EC0011221A70524B1B78002B40F007844F4B71
:1026FC000A221A7000F002BC474B9B88DAB24D4B91
:10270C001B88D9B2464B1B88DBB20A200190009380
:10271C000B460021032002F099F9424B1B889AB218
:10272C00454B1B889A4202D3404B11221A70404BE6
:10273C001B78002B00F0E4833C4B11221A70DFE372
:10274C00354B9B88DAB23B4B1B88D9B2344B1B8878
:10275C00DBB20A20019000930B460121032002F00A
:10276C0075F9304B1B889AB2334B1B889A4202D3B3
:10277C002E4B11221A702E4B1B78002B40F0C2836B
:10278C002A4B0C221A70BDE3234B9B88DAB2294BDF
:10279C001B88D9B2224B1B88DBB20A200190009314
:1027AC000B460121032002F051F91E4B1B889AB2F3
:1027BC00214B1B889A4202D31C4B11221A701C4BC2
:1027CC001B78002B00F0A083184B11221A709BE38E
:1027DC00114BDB88DAB2194B1B88D9B2104B1B8812
:1027EC00DBB20A20019000930B460021042002F07A
:1027FC002DF90C4B1B889AB2114B1B889A4202D3B1
:10280C000A4B11221A700A4B1B78002B40F07E8366
:10281C00064B0E221A7079E34C040020220400208F
:10282C001E040020FC03002012040020560400208B
:10283C00F0030020240400201404002026040020AF
:10284C0016040020A04BDB88DAB2A04B1B88D9B24F
:10285C009F4B1B88DBB20A20019000930B46002192
:10286C00042002F0F3F89B4B1B889AB29A4B1B88FE
:10287C009A4202D3994B11221A70994B1B78002B58
:10288C0000F04683954B11221A7041E38E4BDB8886
:10289C00DAB28E4B1B88D9B28D4B1B88DBB20A2067
:1028AC00019000930B460121042002F0CFF8894BD4
:1028BC001B889AB2884B1B889A4202D3874B1122F1
:1028CC001A70874B1B78002B40F02483834B10220B
:1028DC001A701FE37C4BDB88DAB27C4B1B88D9B2B5
:1028EC007B4B1B88DBB20A20019000930B46012125
:1028FC00042002F0ABF8774B1B889AB2764B1B88FE
:10290C009A4202D3754B11221A70754B1B78002B0F
:10291C0000F00283714B11221A70FDE2002200219B
:10292C00012001F013FF00220021022001F00EFF14
:10293C0000220021032001F009FF002200210420C5
:10294C0001F004FF00220121012001F0FFFE002212
:10295C000121022001F0FAFE00220121032001F0E6
:10296C00F5FE00220121042001F0F0FE5C4B1B78E7
:10297C00002B40F0D3825B4B00221A70574B16226F
:10298C001A70CBE2534B1B889BB21D2B24D9554B91
:10299C0001221A7000F05CFE0346FB7100F02AFF66
:1029AC000346BB7100F0F8FF03467B7101F0C8F8D9
:1029BC0003463B71FB79042B0ED1BB79042B0BD155
:1029CC007B79042B08D13B79042B05D1454B002294
:1029DC001A70424B16221A70434B1B8803F00203E9
:1029EC00002B00F09D823D4B13221A7098E20022BE
:1029FC000021012001F0AAFE00220021022001F09A
:102A0C00A5FE00220021032001F0A0FE00220021DF
:102A1C00042001F09BFE00220121012001F096FE12
:102A2C0000220121022001F091FE0022012103204D
:102A3C0001F08CFE00220121042001F087FE284BBE
:102A4C001B78002B40F06E82264B00221A70234B11
:102A5C0000221A70244B1B8823F002039AB2224BDB
:102A6C001A805FE200220021012001F06FFE00229B
:102A7C000021022001F06AFE00220021032001F057
:102A8C0065FE00220021042001F060FE00220121DD
:102A9C00012001F05BFE00220121022001F056FE14
:102AAC0000220121032001F051FE0022012104200B
:102ABC0001F04CFE074B1B889BB2132B40F2348267
:102ACC00064B16221A702FE24C040020260400201C
:102ADC001E040020FC0300201604002056040020D5
:102AEC00F003002057040020540400209D4B0022CA
:102AFC001A809D4B1B8803F00103002B0DD09B4BC0
:102B0C0001221A709A4B17221A7001F0EDF801F09D
:102B1C00BDF901F08DFA01F05FFB964B1A88964BCC
:102B2C001B889A4219D901224FF40041934803F0B3
:102B3C003CFD934B1B889BB2002B18D18B4B012275
:102B4C001A708B4B17221A7001F0CEF801F09EF917
:102B5C0001F06EFA01F040FB09E000224FF4004155
:102B6C00864803F022FD874B1A88854B1A807E4BD2
:102B7C001B8803F00203002B03D07D4B18221A7024
:102B8C00D4E1794B1B8803F01003002B17D0774B43
:102B9C0001221A707C4B1B88DAB27C4B1B88D9B291
:102BAC007B4B1B88DBB20020019000930B4600216D
:102BBC00012001F04BFF6E4B01221A70B6E16A4BFB
:102BCC001B8803F02003002B17D0684B01221A70CE
:102BDC006D4B1B88DAB26D4B1B88D9B26C4B1B88C2
:102BEC00DBB20020019000930B460121012001F083
:102BFC002DFF5F4B03221A7098E15B4B1B8803F08F
:102C0C004003002B17D0594B01221A705E4B5B8886
:102C1C00DAB2604B1B88D9B25D4B1B88DBB200204B
:102C2C00019000930B460021022001F00FFF504B46
:102C3C0005221A707AE14C4B1B8803F08003002BA1
:102C4C0017D04A4B01221A704F4B5B88DAB2514BAA
:102C5C001B88D9B24E4B1B88DBB20020019000932D
:102C6C000B460121022001F0F1FE414B07221A70A4
:102C7C005CE13D4B1B8803F48073002B17D03B4B5E
:102C8C0001221A70404B9B88DAB2434B1B88D9B295
:102C9C003F4B1B88DBB20020019000930B460021B8
:102CAC00032001F0D3FE324B09221A703EE12E4B69
:102CBC001B8803F40073002B17D02C4B01221A70C5
:102CCC00314B9B88DAB2344B1B88D9B2304B1B8802
:102CDC00DBB20020019000930B460121032001F090
:102CEC00B5FE234B0B221A7020E11F4B1B8803F4FB
:102CFC008063002B17D01D4B01221A70224BDB88EE
:102D0C00DAB2254B1B88D9B2214B1B88DBB20020D1
:102D1C00019000930B460021042001F097FE144B08
:102D2C000D221A7002E1104B1B8803F40063002B78
:102D3C0000F0FC800D4B01221A70134BDB88DAB2C9
:102D4C00154B1B88D9B2124B1B88DBB200200190AB
:102D5C0000930B460121042001F078FE044B0F2256
:102D6C001A70E3E0FC0300205404002057040020F8
:102D7C0056040020320200201C04002000080140F0
:102D8C00FE0300201A0400204C0400202004002024
:102D9C001E0400202204002024040020694B1B8800
:102DAC009BB2092B24D900F09FFF0346FB7101F065
:102DBC006DF80346BB7101F03BF903467B7101F0E2
:102DCC000BFA03463B71FB79042B11D1BB79042B15
:102DDC000ED17B79042B0BD13B79042B08D15A4BA8
:102DEC0000221A70594B00221A70594B01221A708A
:102DFC00584B1B8803F00203002B00F09980534BB7
:102E0C0018221A7094E000220021012001F09EFC8F
:102E1C0000220021022001F099FC00220021032055
:102E2C0001F094FC00220021042001F08FFC002210
:102E3C000121012001F08AFC00220121022001F075
:102E4C0085FC00220121032001F080FC00220121DD
:102E5C00042001F07BFC3B4B1B889BB2132B69D9E4
:102E6C003A4B00221A7065E000220021012001F08B
:102E7C006DFC00220021022001F068FC00220021E0
:102E8C00032001F063FC00220021042001F05EFC11
:102E9C0000220121012001F059FC00220121022015
:102EAC0001F054FC00220121032001F04FFC002210
:102EBC000121042001F04AFC274B1B78002B3BD14D
:102ECC00214B00221A70214B16221A70214B1B88A1
:102EDC0023F002039AB21F4B1A802DE000BF2CE0A6
:102EEC0000BF2AE000BF28E000BF26E000BF24E0BE
:102EFC0000BF22E000BF20E000BF1EE000BF1CE0CE
:102F0C0000BF1AE000BF18E000BF16E000BF14E0DD
:102F1C0000BF12E000BF10E000BF0EE000BF0CE0ED
:102F2C0000BF0AE000BF08E000BF06E000BF04E0FD
:102F3C0000BF02E000BF00E000BF00BF0837BD4685
:102F4C0080BD00BFFC030020570400205604002065
:102F5C005904002054040020F003002080B500AF79
:102F6C0002F058F800F060F800F0C2FA00F0A2FA93
:102F7C000AF0F0FC00F02EF900F0D0F900F0B2F8F5
:102F8C0000F06EFA05222249224802F07DF9002158
:102F9C00214801F008FA04211F4801F004FA082125
:102FAC001D4801F000FA0C211B4801F0FCF900212E
:102FBC001A4801F0F8F90421184801F0F4F9082135
:102FCC00164801F0F0F90C21144801F0ECF9FEF769
:102FDC00F7FA0346002B01D000BFFDE7FEF7DAFB42
:102FEC000F4B1B88082B03D0FEF786FBFEF7D2FB9A
:102FFC000C4B00221A70FDF7FBF9FDF7A9F8FFF74F
:10300C000DF8FFF76FF9FEF7CFF800BFF3E700BF3D
:10301C00FC010020A4020020180300206003002003
:10302C00480400205904002080B594B000AF07F18B
:10303C0028032822002118460BF0C8F907F11403C5
:10304C0000221A605A609A60DA601A613B1D0022F5
:10305C001A605A609A60DA600123BB624FF48033C5
:10306C00FB6200233B630123BB6302237B644FF4AD
:10307C008033BB644FF48013FB6407F128031846BC
:10308C0005F00CF80346002B01D000F0DBFA0F23FF
:10309C007B610223BB610023FB614FF480633B62C5
:1030AC0000237B6207F114030221184605F078FA1D
:1030BC000346002B01D000F0C5FA12237B604FF4BD
:1030CC000043FB6000233B613B1D184605F0F8FBF9
:1030DC000346002B01D000F0B5FA00BF5037BD46B7
:1030EC0080BD000080B584B000AF3B1D00221A608B
:1030FC005A609A60354B364A1A60344B4FF48072E2
:10310C009A60324B01221A73304B00221A752F4BE6
:10311C004FF46022DA612D4B00225A602B4B0522B2
:10312C001A612A4801F0D8FF0346002B01D000F0A9
:10313C0089FA04237B600123BB600323FB603B1DE6
:10314C001946224802F09AF90346002B01D000F0F0
:10315C0079FA05237B600223BB603B1D19461B4893
:10316C0002F08CF90346002B01D000F06BFA062319
:10317C007B600323BB603B1D1946144802F07EF9AB
:10318C000346002B01D000F05DFA07237B6004237B
:10319C00BB603B1D19460D4802F070F90346002B2D
:1031AC0001D000F04FFA08237B600523BB603B1D68
:1031BC001946064802F062F90346002B01D000F0D4
:1031CC0041FA00BF1037BD4680BD00BFA4020020ED
:1031DC000024014080B58EB000AF07F12803002217
:1031EC001A605A609A60DA6007F1200300221A60B4
:1031FC005A603B1D00221A605A609A60DA601A61AC
:10320C005A619A61444B4FF080421A60424B002243
:10321C005A60414B00229A603F4B44F24F62DA6095
:10322C003D4B00221A613C4B00229A613A4805F052
:10323C00FDFB0346002B01D000F004FA4FF4805341
:10324C00BB6207F128031946334805F05FFE0346BD
:10325C00002B01D000F0F6F92F4805F036FC0346A0
:10326C00002B01D000F0EEF900233B6200237B62BF
:10327C0007F120031946284806F0E8F90346002B0D
:10328C0001D000F0DFF960237B604FF47A73BB60F0
:10329C000023FB6004237B613B1D002219461E4862
:1032AC0005F072FD0346002B01D000F0CBF94FF472
:1032BC00FA63BB603B1D04221946174805F064FDF8
:1032CC000346002B01D000F0BDF940F6B833BB60CB
:1032DC0000237B613B1D082219460F4805F054FD65
:1032EC000346002B01D000F0ADF94FF47A63BB60BC
:1032FC0004237B613B1D0C221946074805F044FD55
:10330C000346002B01D000F09DF9034801F03EFD6F
:10331C0000BF3837BD4680BD1803002080B58EB085
:10332C0000AF07F1280300221A605A609A60DA6035
:10333C0007F1200300221A605A603B1D00221A601C
:10334C005A609A60DA601A615A619A61424B434A38
:10335C001A60414B00225A603F4B00229A603E4B50
:10336C0044F24F62DA603C4B00221A613A4B002265
:10337C009A61394805F05AFB0346002B01D000F046
:10338C0061F94FF48053BB6207F1280319463248A8
:10339C0005F0BCFD0346002B01D000F053F92E487C
:1033AC0005F093FB0346002B01D000F04BF90023F2
:1033BC003B6200237B6207F120031946264806F086
:1033CC0045F90346002B01D000F03CF960237B60EB
:1033DC0041F28833BB600023FB6004237B613B1DFF
:1033EC00002219461C4805F0CFFC0346002B01D0E7
:1033FC0000F028F941F27073BB603B1D04221946A2
:10340C00154805F0C1FC0346002B01D000F01AF959
:10341C0041F65833BB603B1D082219460E4805F097
:10342C00B3FC0346002B01D000F00CF94FF4FA5317
:10343C00BB603B1D0C221946074805F0A5FC034652
:10344C00002B01D000F0FEF8034801F09FFC00BFF8
:10345C003837BD4680BD00BF600300200008004027
:10346C0080B500AF114B124A1A60104B4FF4E13289
:10347C005A600E4B00229A600C4B0022DA600B4B08
:10348C0000221A61094B0C225A61084B00229A61E6
:10349C00064B0022DA61054806F036F90346002B8C
:1034AC0001D000F0CFF800BF80BD00BFA803002002
:1034BC000038014080B582B000AF0C4B5B690B4A01
:1034CC0043F001035361094B5B6903F001037B601B
:1034DC007B68002200210B2002F0A1FA0B2002F0E5
:1034EC00BAFA00BF0837BD4680BD00BF00100240CD
:1034FC0080B588B000AF07F1100300221A605A6043
:10350C009A60DA604B4B9B694A4A43F01003936113
:10351C00484B9B6903F01003FB60FB68454B9B69B0
:10352C00444A43F020039361424B9B6903F0200310
:10353C00BB60BB683F4B9B693E4A43F004039361FD
:10354C003C4B9B6903F004037B607B68394B9B69A4
:10355C00384A43F008039361364B9B6903F0080328
:10356C003B603B6800224FF40051334803F01DF8D8
:10357C00002240F63E41314803F017F800224FF488
:10358C0001412F4803F011F84FF400533B61012324
:10359C007B610023BB610223FB6107F11003194619
:1035AC00254802F067FE4FF440433B6100237B61EA
:1035BC000023BB6107F1100319461F4802F05AFEA5
:1035CC0010233B6103237B6107F1100319461C4850
:1035DC0002F050FE40F63E433B6101237B61002329
:1035EC00BB610223FB6107F110031946134802F07B
:1035FC0041FE4FF470433B6100237B610023BB61B0
:10360C0007F1100319460D4802F034FE4FF4014344
:10361C003B6101237B610023BB610223FB6107F14A
:10362C0010031946064802F025FE00BF2037BD46A0
:10363C0080BD00BF0010024000100140000C014092
:10364C000008014080B400AF72B600BF00BFFDE7B8
:10365C0080B59CB002AF5D4B1A785D4B1B789A42DB
:10366C0017D05B4B1A78594B1A70594B1B781A466A
:10367C003B1D584918460AF087FE3B1D1846FCF7BF
:10368C005FFD03469AB2391D4FF0FF33524806F0E6
:10369C008BF8524B1B889AB2514B1B889A4202D220
:1036AC004B4B00221A704A4B1B78032B76D801A285
:1036BC0052F823F0D13600081D3700084D370008AA
:1036CC007F37000800220021012001F03FF8002282
:1036DC000121012001F03AF8404B1B889AB2404B73
:1036EC001B889A4265D33F4B1B88DAB23E4B1B8832
:1036FC00D9B23E4B1B88DBB20020019000930B46E5
:10370C000021012001F0A2F9314B01221A7050E086
:10371C00344B1B88DAB2344B1B88D9B2334B1B8821
:10372C00DBB20A20019000930B460021012001F02E
:10373C008DF90346002B3ED1254B02221A703AE03C
:10374C00264B1B889AB22A4B1B889A4235D3264BA0
:10375C001B88DAB2254B1B88DBB200210191009348
:10376C0000230021012001F071F9194B03221A707A
:10377C0023E01D4B1B88DAB21C4B1B88DBB20A21E1
:10378C000191009300230021012001F05FF9034611
:10379C00002B14D10E4B04221A7010E000220021D1
:1037AC00012000F0D3FF00220121012000F0CEFF08
:1037BC0006E000BF04E000BF02E000BF00E000BF75
:1037CC00034B1B7818466837BD4680BD07000020A8
:1037DC0062040020F0F20008A8030020FC03002083
:1037EC00280400204C0400200004002018040020B1
:1037FC002A04002080B59CB002AF5D4B1A785D4B5B
:10380C001B789A4217D05B4B1A78594B1A70594B4C
:10381C001B781A463B1D584918460AF0B5FD3B1D4E
:10382C001846FCF78DFC03469AB2391D4FF0FF3356
:10383C00524805F0B9FF524B1B889AB2514B1B886A
:10384C009A4202D24B4B00221A704A4B1B78032B24
:10385C0076D801A252F823F075380008C138000858
:10386C00F13800082339000800220021022000F062
:10387C006DFF00220121022000F068FF404B1B88E5
:10388C009AB2404B1B889A4265D33F4B5B88DAB2A5
:10389C003E4B1B88D9B23E4B1B88DBB200200190FB
:1038AC0000930B460121022001F0D0F8314B01228C
:1038BC001A7050E0344B5B88DAB2344B1B88D9B2A7
:1038CC00334B1B88DBB20A20019000930B4601217D
:1038DC00022001F0BBF80346002B3ED1254B0222FF
:1038EC001A703AE0264B1B889AB22A4B1B889A42D4
:1038FC0035D3264B1B88DAB2254B1B88DBB2002153
:10390C000191009300230121022001F09FF8194B33
:10391C0003221A7023E01D4B1B88DAB21C4B1B8848
:10392C00DBB20A210191009300230121022001F056
:10393C008DF80346002B14D10E4B04221A7010E0A4
:10394C0000220021022000F001FF002201210220B0
:10395C0000F0FCFE06E000BF04E000BF02E000BF88
:10396C0000E000BF034B1B7818466837BD4680BD8E
:10397C000800002063040020FCF20008A8030020CB
:10398C00FC0300202C0400204C0400200404002024
:10399C00180400202E04002080B59CB002AF5D4BB3
:1039AC001A785D4B1B789A4217D05B4B1A78594B9F
:1039BC001A70594B1B781A463B1D584918460AF089
:1039CC00E3FC3B1D1846FCF7BBFB03469AB2391DC2
:1039DC004FF0FF33524805F0E7FE524B1B889AB26A
:1039EC00514B1B889A4202D24B4B00221A704A4B05
:1039FC001B78032B76D801A252F823F0193A000851
:103A0C00653A0008953A0008C73A000800220021E0
:103A1C00032000F09BFE00220121032000F096FE03
:103A2C00404B1B889AB2404B1B889A4265D33F4B44
:103A3C009B88DAB23E4B1B88D9B23E4B1B88DBB25B
:103A4C000020019000930B460021032000F0FEFFA4
:103A5C00314B01221A7050E0344B9B88DAB2364B52
:103A6C001B88D9B2334B1B88DBB20A200190009320
:103A7C000B460021032000F0E9FF0346002B3ED14A
:103A8C00254B02221A703AE0264B1B889AB22B4B1C
:103A9C001B889A4235D3284B1B88DAB2254B1B88DE
:103AAC00DBB200210191009300230021032000F0E0
:103ABC00CDFF194B03221A7023E01F4B1B88DAB27F
:103ACC001C4B1B88DBB20A210191009300230021BF
:103ADC00032000F0BBFF0346002B14D10E4B042235
:103AEC001A7010E000220021032000F02FFE0022AB
:103AFC000121032000F02AFE06E000BF04E000BF15
:103B0C0002E000BF00E000BF034B1B78184668378B
:103B1C00BD4680BD090000206404002008F30008A5
:103B2C00A8030020FC030020300400204C040020DB
:103B3C000404002018040020080400203204002093
:103B4C0080B59CB002AF5D4B1A785D4B1B789A42E6
:103B5C0017D05B4B1A78594B1A70594B1B781A4675
:103B6C003B1D584918460AF00FFC3B1D1846FCF744
:103B7C00E7FA03469AB2391D4FF0FF33524805F06D
:103B8C0013FE524B1B889AB2514B1B889A4202D29D
:103B9C004B4B00221A704A4B1B78032B76D801A290
:103BAC0052F823F0C13B00080D3C00083D3C0008D6
:103BBC006F3C000800220021042000F0C7FD002209
:103BCC000121042000F0C2FD404B1B889AB2404BEF
:103BDC001B889A4265D33F4BDB88DAB23E4B1B887D
:103BEC00D9B23E4B1B88DBB20020019000930B46F0
:103BFC000021042000F02AFF314B01221A7050E002
:103C0C00344BDB88DAB2364B1B88D9B2334B1B886A
:103C1C00DBB20A20019000930B460021042000F037
:103C2C0015FF0346002B3ED1254B02221A703AE0B9
:103C3C00264B1B889AB22B4B1B889A4235D3284BA8
:103C4C001B88DAB2254B1B88DBB200210191009353
:103C5C0000230021042000F0F9FE194B03221A70F6
:103C6C0023E01F4B1B88DAB21C4B1B88DBB20A21EA
:103C7C000191009300230021042000F0E7FE03468D
:103C8C00002B14D10E4B04221A7010E000220021DC
:103C9C00042000F05BFD00220121042000F056FD01
:103CAC0006E000BF04E000BF02E000BF00E000BF80
:103CBC00034B1B7818466837BD4680BD0A000020B0
:103CCC006504002014F30008A8030020FC03002066
:103CDC00340400204C0400200404002018040020AC
:103CEC000C0400203604002080B59CB002AF5D4B64
:103CFC001A785D4B1B789A4217D05B4B1A78594B4C
:103D0C001A70594B1B781A463B1D584918460AF035
:103D1C003BFB3B1D1846FCF713FA03469AB2391DC0
:103D2C004FF0FF33524805F03FFD524B1B889AB2BF
:103D3C00514B1B889A4202D24B4B00221A704A4BB1
:103D4C001B78032B76D801A252F823F0693D0008AA
:103D5C00B53D0008E53D0008173E00080022002193
:103D6C00012000F0F3FC00220121012000F0EEFC08
:103D7C00404B1B889AB2404B1B889A4265D33F4BF1
:103D8C001B88DAB23E4B1B88D9B23E4B1B88DBB288
:103D9C000020019000930B460121012000F056FEFB
:103DAC00314B01221A7050E0344B1B88DAB2344B81
:103DBC001B88D9B2334B1B88DBB20A2001900093CD
:103DCC000B460121012000F041FE0346002B3ED1A1
:103DDC00254B02221A703AE0264B1B889AB22A4BCA
:103DEC001B889A4235D3264B1B88DAB2254B1B888D
:103DFC00DBB200210191009300230121012000F08E
:103E0C0025FE194B03221A7023E01D4B1B88DAB2D6
:103E1C001C4B1B88DBB20A2101910093002301216A
:103E2C00012000F013FE0346002B14D10E4B04228C
:103E3C001A7010E000220021012000F087FC002203
:103E4C000121012000F082FC06E000BF04E000BF6D
:103E5C0002E000BF00E000BF034B1B781846683738
:103E6C00BD4680BD0B0000206604002020F3000836
:103E7C00A8030020FC030020380400204C04002080
:103E8C0002040020180400203A04002080B59CB0E5
:103E9C0002AF5D4B1A785D4B1B789A4217D05B4B87
:103EAC001A78594B1A70594B1B781A463B1D5849B6
:103EBC0018460AF069FA3B1D1846FCF741F903460F
:103ECC009AB2391D4FF0FF33524805F06DFC524B3E
:103EDC001B889AB2514B1B889A4202D24B4B002240
:103EEC001A704A4B1B78032B76D801A252F823F098
:103EFC000D3F0008593F0008893F0008BB3F0008F0
:103F0C0000220021022000F021FC002201210220CD
:103F1C0000F01CFC404B1B889AB2404B1B889A4209
:103F2C0065D33F4B5B88DAB23E4B1B88D9B23E4B14
:103F3C001B88DBB20020019000930B46002102206D
:103F4C0000F084FD314B01221A7050E0344B5B8839
:103F5C00DAB2344B1B88D9B2334B1B88DBB20A2044
:103F6C00019000930B460021022000F06FFD0346E8
:103F7C00002B3ED1254B02221A703AE0264B1B88AF
:103F8C009AB22A4B1B889A4235D3264B1B88DAB23D
:103F9C00254B1B88DBB200210191009300230021EB
:103FAC00022000F053FD194B03221A7023E01D4B25
:103FBC001B88DAB21C4B1B88DBB20A2101910093DF
:103FCC0000230021022000F041FD0346002B14D1F8
:103FDC000E4B04221A7010E000220021022000F087
:103FEC00B5FB00220121022000F0B0FB06E000BF6F
:103FFC0004E000BF02E000BF00E000BF034B1B78F1
:10400C0018466837BD4680BD0C00002067040020B0
:10401C002CF30008A8030020FC0300203C04002023
:10402C004C04002006040020180400203E0400204C
:10403C0080B59CB002AF5D4B1A785D4B1B789A42F1
:10404C0017D05B4B1A78594B1A70594B1B781A4680
:10405C003B1D584918460AF097F93B1D1846FCF7CA
:10406C006FF803469AB2391D4FF0FF33524805F0F2
:10407C009BFB524B1B889AB2514B1B889A4202D223
:10408C004B4B00221A704A4B1B78032B76D801A29B
:10409C0052F823F0B1400008FD4000082D41000803
:1040AC005F41000800220021032000F04FFB00229A
:1040BC000121032000F04AFB404B1B889AB2404B75
:1040CC001B889A4265D33F4B9B88DAB23E4B1B88C8
:1040DC00D9B23E4B1B88DBB20020019000930B46FB
:1040EC000121032000F0B2FC314B01221A7050E088
:1040FC00344B9B88DAB2364B1B88D9B2334B1B88B6
:10410C00DBB20A20019000930B460121032000F042
:10411C009DFC0346002B3ED1254B02221A703AE03F
:10412C00264B1B889AB22B4B1B889A4235D3284BB3
:10413C001B88DAB2254B1B88DBB20021019100935E
:10414C0000230121032000F081FC194B03221A707B
:10415C0023E01F4B1B88DAB21C4B1B88DBB20A21F5
:10416C000191009300230121032000F06FFC034612
:10417C00002B14D10E4B04221A7010E000220021E7
:10418C00032000F0E3FA00220121032000F0DEFA04
:10419C0006E000BF04E000BF02E000BF00E000BF8B
:1041AC00034B1B7818466837BD4680BD0D000020B8
:1041BC006804002038F30008A8030020FC0300204A
:1041CC00400400204C0400200604002018040020A9
:1041DC000A0400204204002080B59CB002AF5D4B65
:1041EC001A785D4B1B789A4217D05B4B1A78594B57
:1041FC001A70594B1B781A463B1D584918460AF041
:10420C00C3F83B1D1846FBF79BFF03469AB2391DBA
:10421C004FF0FF33524805F0C7FA524B1B889AB245
:10422C00514B1B889A4202D24B4B00221A704A4BBC
:10423C001B78032B76D801A252F823F059420008C0
:10424C00A5420008D54200080743000800220021BF
:10425C00042000F07BFA00220121042000F076FA01
:10426C00404B1B889AB2404B1B889A4265D33F4BFC
:10427C00DB88DAB23E4B1B88D9B23E4B1B88DBB2D3
:10428C000020019000930B460121042000F0DEFB7E
:10429C00314B01221A7050E0344BDB88DAB2344BCC
:1042AC001B88D9B2334B1B88DBB20A2001900093D8
:1042BC000B460121042000F0C9FB0346002B3ED124
:1042CC00254B02221A703AE0264B1B889AB22A4BD5
:1042DC001B889A4235D3264B1B88DAB2254B1B8898
:1042EC00DBB200210191009300230121042000F096
:1042FC00ADFB194B03221A7023E01D4B1B88DAB25D
:10430C001C4B1B88DBB20A21019100930023012175
:10431C00042000F09BFB0346002B14D10E4B04220F
:10432C001A7010E000220021042000F00FFA002285
:10433C000121042000F00AFA06E000BF04E000BFEF
:10434C0002E000BF00E000BF034B1B781846683743
:10435C00BD4680BD0E0000206904002044F3000817
:10436C00A8030020FC030020440400204C0400207F
:10437C000E040020180400204604002080B584B0F0
:10438C0000AF786039603968786804F086FE0346BF
:10439C00FB73FB7B022B0CBF01230023DBB2184603
:1043AC001037BD4680BD80B582B000AF78603960F3
:1043BC003968786804F084FC00BF0837BD4680BDBE
:1043CC0080B584B000AFF860B9601346FB80BB6861
:1043DC00002B04D1FB681B68FA885A6313E0BB6896
:1043EC00042B04D1FB681A68FB8893630BE0BB6851
:1043FC00082B04D1FB681A68FB88D36303E0FB68C5
:10440C001A68FB881364B968F86804F0B7FB00BF3E
:10441C001037BD4680BD80B485B000AFF860B96080
:10442C001346FB80BB68002B04D1FB681B68FA8821
:10443C005A6313E0BB68042B04D1FB681A68FB8831
:10444C0093630BE0BB68082B04D1FB681A68FB88EC
:10445C00D36303E0FB681A68FB88136400BF14374E
:10446C00BD4680BC7047000080B582B000AF0346EB
:10447C00FB710B46BB711346BB80FB79013B032BD5
:10448C0000F2588101A252F823F000BFA9440008A1
:10449C004B450008ED45000897460008BB79002BFA
:1044AC0026D1BB88002B09D10021A548FFF77BFF43
:1044BC0000220221A34802F078F83CE10021A04838
:1044CC00FFF75CFF0346002B06D0BB881A46002181
:1044DC009B48FFF7A0FF2EE101220221994802F030
:1044EC0064F8BB881A4600219548FFF769FF22E162
:1044FC00BB88002B09D104219148FFF754FF0022FF
:10450C000221904802F051F815E104218C48FFF784
:10451C0035FF0346002B06D0BB881A460421884879
:10452C00FFF779FF07E101220221864802F03DF8EE
:10453C00BB881A4604218248FFF742FFFBE0BB7997
:10454C00002B26D1BB88002B09D108217C48FFF712
:10455C002AFF002204217B4802F027F8EBE0082117
:10456C007748FFF70BFF0346002B06D0BB881A4693
:10457C0008217348FFF74FFFDDE001220421714849
:10458C0002F013F8BB881A4608216D48FFF718FF94
:10459C00D1E0BB88002B09D10C216948FFF703FF40
:1045AC0000220421674802F000F8C4E00C216448A2
:1045BC00FFF7E4FE0346002B06D0BB881A460C21FD
:1045CC005F48FFF728FFB6E0012204215D4801F0A7
:1045DC00ECFFBB881A460C215948FFF7F1FEAAE004
:1045EC00BB79002B28D1BB88002B0AD1002156485F
:1045FC00FFF7D9FE00224FF48061524801F0D5FF3D
:10460C0099E000215048FFF7B9FE0346002B06D075
:10461C00BB881A4600214C48FFF7FDFE8BE00122B7
:10462C004FF48061474801F0C0FFBB881A46002157
:10463C004548FFF7C5FE7EE0BB88002B0AD104215C
:10464C004148FFF7B0FE00224FF480613D4801F075
:10465C00ACFF70E004213C48FFF790FE0346002BB2
:10466C0006D0BB881A4604213748FFF7D4FE62E017
:10467C0001224FF48061334801F097FFBB881A4642
:10468C0004213148FFF79CFE55E0BB79002B28D163
:10469C00BB88002B0AD108212B48FFF784FE00228F
:1046AC004FF40061274801F080FF44E008212648C0
:1046BC00FFF764FE0346002B06D0BB881A46082180
:1046CC002148FFF7A8FE36E001224FF400611D4897
:1046DC0001F06BFFBB881A4608211B48FFF770FEE0
:1046EC0029E0BB88002B0AD10C211748FFF75BFE91
:1046FC0000224FF40061134801F057FF1BE00C211E
:10470C001148FFF73BFE0346002B06D0BB881A4628
:10471C000C210D48FFF77FFE0DE001224FF40061E4
:10472C00084801F042FFBB881A460C210648FFF7E7
:10473C0047FE00E000BF00BF0837BD4680BD00BF8C
:10474C0018030020000C01406003002080B584B0E9
:10475C0000AF0346FB710B46BB7113467B717B7933
:10476C00FB60FB689B03FB60FB68B44AA2FB032362
:10477C005B09FB60FB687B81FB79013B032B00F23F
:10478C00578101A252F823F0A547000847480008BA
:10479C00E948000893490008BB79002B26D17B8996
:1047AC00002B09D10021A648FFF7FDFD00220221B4
:1047BC00A44801F0FAFE3CE10021A148FFF7DEFD20
:1047CC000346002B06D07B891A4600219C48FFF734
:1047DC0022FE2EE1012202219A4801F0E6FE7B899D
:1047EC001A4600219648FFF7EBFD22E17B89002B4E
:1047FC0009D104219248FFF7D6FD002202219148ED
:10480C0001F0D3FE15E104218D48FFF7B7FD0346F7
:10481C00002B06D07B891A4604218948FFF7FBFD43
:10482C0007E101220221874801F0BFFE7B891A466D
:10483C0004218348FFF7C4FDFBE0BB79002B26D194
:10484C007B89002B09D108217D48FFF7ACFD0022A4
:10485C0004217C4801F0A9FEEBE008217848FFF721
:10486C008DFD0346002B06D07B891A46082174481F
:10487C00FFF7D1FDDDE001220421724801F095FE25
:10488C007B891A4608216E48FFF79AFDD1E07B8997
:10489C00002B09D10C216A48FFF785FD0022042169
:1048AC00684801F082FEC4E00C216548FFF766FD04
:1048BC000346002B06D07B891A460C216048FFF773
:1048CC00AAFDB6E0012204215E4801F06EFE7B8950
:1048DC001A460C215A48FFF773FDAAE0BB79002B4E
:1048EC0028D17B89002B0AD100215748FFF75BFDAB
:1048FC0000224FF48061534801F057FE99E00021EB
:10490C005148FFF73BFD0346002B06D07B891A4626
:10491C0000214D48FFF77FFD8BE001224FF48061B1
:10492C00484801F042FE7B891A4600214648FFF7B1
:10493C0047FD7EE07B89002B0AD104214248FFF71A
:10494C0032FD00224FF480613E4801F02EFE70E0F3
:10495C0004213D48FFF712FD0346002B06D07B894E
:10496C001A4604213848FFF756FD62E001224FF445
:10497C008061344801F019FE7B891A4604213248C3
:10498C00FFF71EFD55E0BB79002B28D17B89002B4E
:10499C000AD108212C48FFF706FD00224FF40061D4
:1049AC00284801F002FE44E008212748FFF7E6FC06
:1049BC000346002B06D07B891A4608212248FFF7B4
:1049CC002AFD36E001224FF400611E4801F0EDFD96
:1049DC007B891A4608211C48FFF7F2FC29E07B89E9
:1049EC00002B0AD10C211848FFF7DDFC00224FF4F4
:1049FC000061144801F0D9FD1BE00C211248FFF7AF
:104A0C00BDFC0346002B06D07B891A460C210E48B0
:104A1C00FFF701FD0DE001224FF40061094801F0A0
:104A2C00C4FD7B891A460C210748FFF7C9FC00E03E
:104A3C0000BF00BF1037BD4680BD00BF1F85EB51C6
:104A4C0018030020000C01406003002090B585B0D5
:104A5C0000AF0446084611461A462346FB7103462E
:104A6C00BB710B467B7113463B7197F82430002BBE
:104A7C0002D00A2B16D09DE0FB79013B97F8202041
:104A8C0091B24F4A084622F81300FB79013BC9B298
:104A9C004C4AD1547A79B979FB791846FFF756FE0E
:104AAC00002388E0FB79013B464AD35C1946FB792D
:104ABC00013B434A32F813309BB2994278D0FB79D0
:104ACC00013B3F4A32F813309AB2FB79013BD1B229
:104ADC003C4AD154FB79013B394A32F813309BB232
:104AEC00002B5DD07A793B799A4226D97B799AB2A0
:104AFC003B799BB2D31AFB8197F820309AB2FB79A1
:104B0C00013B2F4931F813309BB2D31A9BB2FA896F
:104B1C0002FB03F3FB81FA8997F8203092FBF3F345
:104B2C00FB81FB89DBB27A79D31ADAB2B979FB79DA
:104B3C001846FFF70BFE01233DE07A793B799A4248
:104B4C0026D23B799AB27B799BB2D31AFB8197F828
:104B5C0020309AB2FB79013B194931F813309BB2E2
:104B6C00D31A9BB2FA8902FB03F3FB81FA8997F8FB
:104B7C00203092FBF3F3FB81FB89DAB27B7913448F
:104B8C00DAB2B979FB791846FFF7E0FD012312E0A0
:104B9C003A79B979FB791846FFF7D8FD00230AE07A
:104BAC003A79B979FB791846FFF7D0FD002302E07A
:104BBC00012300E0002318461437BD4690BD00BF0A
:104BCC00F40300206C04002080B485B000AF154BBA
:104BDC009B69144A43F001039361124B9B6903F0E8
:104BEC000103BB60BB680F4BDB690E4A43F080537B
:104BFC00D3610C4BDB6903F080537B607B680A4B01
:104C0C005B68FB60FB6823F0E063FB60FB6843F0D0
:104C1C000073FB60044AFB68536000BF1437BD4649
:104C2C0080BC7047001002400000014080B58AB083
:104C3C0000AF786007F1180300221A605A609A607E
:104C4C00DA607B681B68334A93425FD1324B9B69B5
:104C5C00314A43F4007393612F4B9B6903F4007347
:104C6C007B617B692C4B9B692B4A43F0040393615A
:104C7C00294B9B6903F004033B613B69264B9B6901
:104C8C00254A43F008039361234B9B6903F0080307
:104C9C00FB60FB68F023BB610323FB6107F1180386
:104CAC0019461E4801F0E6FA0123BB610323FB61A0
:104CBC0007F1180319461A4801F0DCFA194B1A4A85
:104CCC001A60184B00225A60164B00229A60154B42
:104CDC008022DA60134B4FF480721A61114B4FF43F
:104CEC0080625A610F4B20229A610E4B0022DA61CE
:104CFC000C4800F0D1FE0346002B01D0FEF7A2FCBD
:104D0C007B68084A1A62074A7B68536200BF2837DF
:104D1C00BD4680BD00240140001002400008014047
:104D2C00000C0140D40200200800024080B485B081
:104D3C0000AF78607B681B68B3F1804F0CD1114BCE
:104D4C00DB69104A43F00103D3610E4BDB6903F0BE
:104D5C000103FB60FB6810E07B681B680A4A934206
:104D6C000BD1084BDB69074A43F00403D361054BB5
:104D7C00DB6903F00403BB60BB6800BF1437BD469E
:104D8C0080BC7047001002400008004080B588B01D
:104D9C0000AF786007F1100300221A605A609A6025
:104DAC00DA607B681B68B3F1804F18D11D4B9B698F
:104DBC001C4A43F0040393611A4B9B6903F00403F0
:104DCC00FB60FB680F233B6102237B610223FB61C9
:104DDC0007F110031946144801F04CFA1DE07B68EA
:104DEC001B68124A934218D10E4B9B690D4A43F033
:104DFC00080393610B4B9B6903F00803BB60BB6812
:104E0C004FF470733B6102237B610223FB6107F15A
:104E1C0010031946064801F02DFA00BF2037BD4695
:104E2C0080BD00BF00100240000801400008004097
:104E3C00000C014080B588B000AF786007F110031A
:104E4C0000221A605A609A60DA607B681B681C4A00
:104E5C00934231D11B4B9B691A4A43F480439361B3
:104E6C00184B9B6903F48043FB60FB68154B9B69F3
:104E7C00144A43F004039361124B9B6903F004033F
:104E8C00BB60BB684FF400733B6102237B6103235F
:104E9C00FB6107F1100319460B4801F0EBF94FF4D5
:104EAC0080633B6100237B610023BB6107F110032E
:104EBC001946054801F0DEF900BF2037BD4680BD1C
:104ECC0000380140001002400008014080B400AFDF
:104EDC0000BFFDE780B400AF00BFFDE780B400AFBA
:104EEC0000BFFDE780B400AF00BFFDE780B400AFAA
:104EFC0000BFFDE780B400AF00BFBD4680BC70476B
:104F0C0080B400AF00BFBD4680BC704780B400AF1A
:104F1C0000BFBD4680BC704780B500AF00F0C0F844
:104F2C0000F0B3FD00BF80BD80B500AF024800F0BB
:104F3C006DFE00BF80BD00BFD402002080B500AF65
:104F4C00024801F066FC00BF80BD00BF6412002067
:104F5C0080B586B000AF7860144A154BD31A7B61CC
:104F6C007B693B61134B1B68002B02D1114B124A1E
:104F7C001A60104B1A687B6813443A699A4207D23C
:104F8C0009F02CFA03460C221A604FF0FF3309E0AB
:104F9C00084B1B68FB60074B1A687B681344054A77
:104FAC001360FB6818461837BD4680BD00500020C2
:104FBC000004000070040020A818002080B400AF8A
:104FCC0000BFBD4680BC7047FFF7F8FF0B480C498B
:104FDC000C4A002302E0D458C4500433C4188C4249
:104FEC00F9D3094A094C002301E013600432A242B0
:104FFC00FBD309F0F9F9FDF7B1FF70470000002071
:10500C00DC01002008F50008E0010020A4180020B5
:10501C00FEE7000080B500AF084B1B68074A43F061
:10502C0010031360032000F0EFFC0F2000F008F8D1
:10503C00FFF7CAFD0023184680BD00BF00200240C8
:10504C0080B582B000AF7860124B1A68124B1B7897
:10505C0019464FF47A73B3FBF1F3B2FBF3F3184632
:10506C0000F007FD0346002B01D001230EE07B6806
:10507C000F2B0AD8002279684FF0FF3000F0CFFCDC
:10508C00064A7B681360002300E0012318460837AA
:10509C00BD4680BD10000020180000201400002028
:1050AC0080B400AF054B1B781A46054B1B681344A4
:1050BC00034A136000BFBD4680BC70471800002037
:1050CC007404002080B400AF024B1B681846BD4628
:1050DC0080BC70477404002080B586B000AF786047
:1050EC000023FB7500233B610023BB600023FB60A6
:1050FC007B68002B01D10123BEE07B689B68002BF1
:10510C007B689B6A002B09D17B680022DA627B6882
:10511C00002283F824207868FFF788FD786800F077
:10512C00FFFA0346FB757B689B6A03F01003002BA8
:10513C0040F09980FB7D002B40F095807B689B6A4A
:10514C0023F4885323F0020343F002027B689A6233
:10515C007B685A687B68DB691A437B681B7B5B0046
:10516C001343BA681343BB607B689B68B3F5807FBD
:10517C0003D07B689B68012B02D14FF4807300E055
:10518C0000233A6913433B617B681B7D012B19D1CA
:10519C007B681B7B002B09D17B689B69013B5A0305
:1051AC003B69134343F400633B610BE07B689B6AF0
:1051BC0043F020027B689A627B68DB6A43F0010251
:1051CC007B68DA627B681B685B6823F469417B68E7
:1051DC001B683A690A435A607B681B689A68284BBB
:1051EC0013407A681268B9680B4393607B689B68BC
:1051FC00B3F5807F03D07B689B68012B04D17B685F
:10520C001B69013B1B05FB607B681B68DB6A23F495
:10521C0070017B681B68FA680A43DA627B681B685A
:10522C009A68184B1340BA689A420BD17B680022DB
:10523C00DA627B689B6A23F0030343F001027B680C
:10524C009A6218E07B689B6A23F0120343F0100209
:10525C007B689A627B68DB6A43F001027B68DA62E6
:10526C000123FB7507E07B689B6A43F010027B68A7
:10527C009A620123FB75FB7D18461837BD4680BD2D
:10528C00FDF7E1FFFE0E1FFF80B586B000AFF860A2
:10529C00B9607A600023FB75FB681B68644A934213
:1052AC0004D0FB681B68634A934206D1604B5B6871
:1052BC0003F47023002B40F0B380FB6893F8243088
:1052CC00012B01D10223AEE0FB68012283F82420DC
:1052DC00F86800F0CBF90346FB75FB7D002B40F022
:1052EC009A80FB689B6A23F4706323F0010343F4F8
:1052FC008072FB689A62FB681B684E4A934205D128
:10530C004B4B5B6803F47023002B15D1FB689B6A35
:10531C0023F48012FB689A62FB681B685B6803F4D9
:10532C008063002B26D0FB689B6A23F4405343F424
:10533C008052FB689A621DE0FB689B6A43F4801202
:10534C00FB689A62FB681B68394A934204D0FB687D
:10535C001B68384A93420DD1354B5B6803F480636C
:10536C00002B07D0FB689B6A23F4405343F4805214
:10537C00FB689A62FB689B6A03F48053002B06D08F
:10538C00FB68DB6A23F00602FB68DA6202E0FB686A
:10539C000022DA62FB68002283F82420FB681B6A77
:1053AC00254A9A62FB681B6A244ADA62FB681B6A0C
:1053BC00234A1A63FB681B686FF002021A60FB68D1
:1053CC001B689A68FB681B6842F480729A60FB68E1
:1053DC00186AFB681B684C331946BA687B6800F086
:1053EC00B5FBFB681B689B6803F46023B3F5602F67
:1053FC0008D1FB681B689A68FB681B6842F4A00222
:10540C009A600FE0FB681B689A68FB681B6842F4A3
:10541C0080129A6006E0FB68002283F8242001E0E9
:10542C000123FB75FB7D18461837BD4680BD00BFB8
:10543C000024014000280140AF5700082B580008F9
:10544C004758000880B483B000AF786000BF0C37B9
:10545C00BD4680BC704780B483B000AF786000BF9D
:10546C000C37BD4680BC704780B483B000AF786009
:10547C0000BF0C37BD4680BC7047000080B485B0BF
:10548C0000AF786039600023FB730023BB607B683E
:10549C0093F82430012B01D10223DCE07B6801223C
:1054AC0083F824203B685B68062B1CD87B681B6840
:1054BC00596B3B685A6813469B001344053B1F22EB
:1054CC0002FA03F3DB4319403B6818683B685A68DF
:1054DC0013469B001344053B00FA03F27B681B68E0
:1054EC000A435A633CE03B685B680C2B1CD87B6816
:1054FC001B68196B3B685A6813469B001344233B8B
:10550C001F2202FA03F3DB4319403B6818683B681F
:10551C005A6813469B001344233B00FA03F27B6842
:10552C001B680A431A631BE07B681B68D96A3B68DB
:10553C005A6813469B001344413B1F2202FA03F3A3
:10554C00DB4319403B6818683B685A6813469B005C
:10555C001344413B00FA03F27B681B680A43DA628E
:10556C003B681B68092B1CD97B681B68D9683B6896
:10557C001A6813465B0013441E3B072202FA03F31E
:10558C00DB4319403B6898683B681A6813465B001C
:10559C0013441E3B00FA03F27B681B680A43DA6073
:1055AC0019E07B681B6819693B681A6813465B0035
:1055BC001344072202FA03F3DB4319403B68986853
:1055CC003B681A6813465B00134400FA03F27B68CD
:1055DC001B680A431A613B681B68102B03D03B689D
:1055EC001B68112B32D17B681B681D4A934225D155
:1055FC007B681B689B6803F40003002B26D17B6837
:10560C001B689A687B681B6842F400029A603B68CE
:10561C001B68102B1AD1134B1B68134AA2FB0323D4
:10562C009A0C13469B0013445B00BB6002E0BB6802
:10563C00013BBB60BB68002BF9D107E07B689B6A20
:10564C0043F020027B689A620123FB737B68002283
:10565C0083F82420FB7B18461437BD4680BC70476A
:10566C00002401401000002083DE1B4380B584B071
:10567C0000AF78600023FB600023BB607B681B6875
:10568C009B6803F00103012B40D07B681B689A6870
:10569C007B681B6842F001029A601F4B1B681F4A13
:1056AC00A2FB03239B0CBB6002E0BB68013BBB600D
:1056BC00BB68002BF9D1FFF705FDF8601FE0FFF781
:1056CC0001FD0246FB68D31A022B18D97B681B68B4
:1056DC009B6803F00103012B11D07B689B6A43F09C
:1056EC0010027B689A627B68DB6A43F001027B687C
:1056FC00DA627B68002283F82420012307E07B68B0
:10570C001B689B6803F00103012BD8D100231846BA
:10571C001037BD4680BD00BF1000002083DE1B4348
:10572C0080B584B000AF78600023FB607B681B6899
:10573C009B6803F00103012B2ED17B681B689A68D0
:10574C007B681B6822F001029A60FFF7BBFCF860D3
:10575C001BE0FFF7B7FC0246FB68D31A022B14D9E7
:10576C007B681B689B6803F00103012B0DD17B68E0
:10577C009B6A43F010027B689A627B68DB6A43F099
:10578C0001027B68DA62012307E07B681B689B6877
:10579C0003F00103012BDCD0002318461037BD4663
:1057AC0080BD80B584B000AF78607B685B6AFB60BD
:1057BC00FB689B6A03F05003002B27D1FB689B6AA4
:1057CC0043F40072FB689A62FB681B689B6803F4E5
:1057DC006023B3F5602F15D1FB681B7B002B11D117
:1057EC00FB689B6A23F48072FB689A62FB689B6A75
:1057FC0003F48053002B05D1FB689B6A43F0010234
:10580C00FB689A62F868FFF71DFE04E0FB681B6AF0
:10581C001B6B7868984700BF1037BD4680BD80B5BC
:10582C0084B000AF78607B685B6AFB60F868FFF758
:10583C0012FE00BF1037BD4680BD80B584B000AFEE
:10584C0078607B685B6AFB60FB689B6A43F0400294
:10585C00FB689A62FB68DB6A43F00402FB68DA625D
:10586C00F868FFF701FE00BF1037BD4680BD000091
:10587C0080B485B000AF78607B6803F00703FB60F1
:10588C000C4BDB68BB60BA684FF6FF031340BB6080
:10589C00FB681A02BB68134343F0BF6343F4003345
:1058AC00BB60044ABB68D36000BF1437BD4680BCE4
:1058BC00704700BF00ED00E080B400AF044BDB6824
:1058CC001B0A03F007031846BD4680BC704700BF97
:1058DC0000ED00E080B483B000AF0346FB7197F994
:1058EC000730002B0BDBFB7903F01F02064997F9FD
:1058FC0007305B09012000FA02F241F8232000BFB7
:10590C000C37BD4680BC704700E100E080B483B02A
:10591C0000AF03463960FB7197F90730002B0ADBA7
:10592C003B68DAB20C4997F907301201D2B20B443A
:10593C0083F800230AE03B68DAB20849FB7903F0EC
:10594C000F03043B1201D2B20B441A7600BF0C3782
:10595C00BD4680BC704700BF00E100E000ED00E0F8
:10596C0080B489B000AFF860B9607A60FB6803F06E
:10597C000703FB61FB69C3F10703042B28BF042356
:10598C00BB61FB690433062B02D9FB69033B00E0C6
:10599C0000237B614FF0FF32BB6902FA03F3DA4359
:1059AC00BB681A407B699A404FF0FF317B6901FA62
:1059BC0003F3D9437B680B40134318462437BD4689
:1059CC0080BC704780B582B000AF78607B68013BCB
:1059DC00B3F1807F01D301230FE00A4A7B68013BBE
:1059EC0053600F214FF0FF30FFF790FF054B002263
:1059FC009A60044B07221A60002318460837BD46EC
:105A0C0080BD00BF10E000E080B582B000AF7860D0
:105A1C007868FFF72DFF00BF0837BD4680BD80B505
:105A2C0086B000AF0346B9607A60FB7300237B61DC
:105A3C00FFF742FF78617A68B9687869FFF790FFE1
:105A4C00024697F90F3011461846FFF75FFF00BF6B
:105A5C001837BD4680BD80B582B000AF0346FB71E0
:105A6C0097F907301846FFF735FF00BF0837BD46DA
:105A7C0080BD80B582B000AF78607868FFF7A2FF78
:105A8C00034618460837BD4680BD80B500AFFCF70D
:105A9C00B3F800BF80BD000080B485B000AF786063
:105AAC000023FB607B68002B01D1012343E07B6862
:105ABC001B681A46224B1344224AA2FB03231B09E0
:105ACC009A007B681A647B681F4ADA637B6802223F
:105ADC0083F821207B681B681B68FB60FB6823F440
:105AEC007F5323F03003FB607B685A687B689B68AC
:105AFC001A437B68DB681A437B681B691A437B6813
:105B0C005B691A437B689B691A437B68DB691343A7
:105B1C00FA681343FB607B681B68FA681A607B6841
:105B2C0000229A637B68012283F821207B68002283
:105B3C0083F82020002318461437BD4680BC7047DC
:105B4C00F8FFFDBFCDCCCCCC0000024080B586B0B8
:105B5C0000AFF860B9607A603B600023FB75FB68AE
:105B6C0093F82030012B01D102234BE0FB6801227A
:105B7C0083F82020FB6893F82130DBB2012B3AD15B
:105B8C00FB68022283F82120FB6800229A63FB68E1
:105B9C001B681A68FB681B6822F001021A603B68DC
:105BAC007A68B968F86800F037F9FB68DB6A002B93
:105BBC0008D0FB681B681A68FB681B6842F00E0271
:105BCC001A600FE0FB681B681A68FB681B6822F000
:105BDC0004021A60FB681B681A68FB681B6842F0B9
:105BEC000A021A60FB681B681A68FB681B6842F0A3
:105BFC0001021A6005E0FB68002283F820200223D2
:105C0C00FB75FB7D18461837BD4680BD80B584B04A
:105C1C0000AF78607B68DB6B1B68FB607B681B6884
:105C2C001B68BB607B681B6C04229A40FB681340AA
:105C3C00002B4FD0BB6803F00403002B4AD07B68C9
:105C4C001B681B6803F02003002B07D17B681B68C3
:105C5C001A687B681B6822F004021A607B681B6858
:105C6C00664A934229D07B681B68654A934222D0CE
:105C7C007B681B68634A93421AD07B681B68624A34
:105C8C00934212D07B681B68604A93420AD07B68AF
:105C9C001B685F4A934202D14FF480030EE04FF031
:105CAC0080630BE04FF4802308E04FF4804305E061
:105CBC004FF4806302E0402300E00423554A536014
:105CCC007B68DB6A002B00F094807B68DB6A786869
:105CDC0098478EE07B681B6C02229A40FB6813404D
:105CEC00002B56D0BB6803F00203002B51D07B680D
:105CFC001B681B6803F02003002B0BD17B681B680F
:105D0C001A687B681B6822F00A021A607B68012201
:105D1C0083F821207B681B68384A934229D07B6822
:105D2C001B68374A934222D07B681B68354A9342E2
:105D3C001AD07B681B68344A934212D07B681B686C
:105D4C00324A93420AD07B681B68314A934202D193
:105D5C004FF400130EE04FF000730BE04FF40033E0
:105D6C0008E04FF4005305E04FF4007302E02023E9
:105D7C0000E00223274A53607B68002283F820202E
:105D8C007B689B6A002B34D07B689B6A7868984749
:105D9C002FE07B681B6C08229A40FB681340002B99
:105DAC0028D0BB6803F00803002B23D07B681B684A
:105DBC001A687B681B6822F00E021A607B681A6CEA
:105DCC007B68DB6B012101FA02F25A607B680122CD
:105DDC009A637B68012283F821207B68002283F878
:105DEC0020207B681B6B002B04D07B681B6B7868B6
:105DFC00984700BF00BF1037BD4680BD0800024069
:105E0C001C00024030000240440002405800024096
:105E1C006C0002400000024080B485B000AFF86016
:105E2C00B9607A603B60FB681A6CFB68DB6B012124
:105E3C0001FA02F25A60FB681B683A685A60FB6808
:105E4C005B68102B08D1FB681B687A689A60FB684A
:105E5C001B68BA68DA6007E0FB681B68BA689A606E
:105E6C00FB681B687A68DA6000BF1437BD4680BCDB
:105E7C0070470000F0B587B000AFF860B960C7E9B3
:105E8C0000230123FB750023BB7500237B752F4B6F
:105E9C001B7E012B01D1022354E02C4B01221A76DC
:105EAC004CF2503000F0A8F80346FB75FB7D002B3C
:105EBC0044D1FB68012B02D101237B7507E0FB6801
:105ECC00022B02D102237B7501E004237B75002396
:105EDC00BB752DE0BB7D5A00BB6802EB030CBB7D90
:105EEC001901D7E90023C1F12006A1F1200022FA03
:105EFC0001F403FA06F6344323FA00F0044323FAC0
:105F0C0001F5A3B21946604600F05AF84CF2503035
:105F1C0000F072F80346FB750D4B1B690C4A23F01D
:105F2C0001031361FB7D002B07D1BB7D0133BB75D6
:105F3C00BA7D7B7D9A42CDD300E000BF034B00229B
:105F4C001A76FB7D18461C37BD46F0BD7804002040
:105F5C000020024080B483B000AF0023FB710D4BD6
:105F6C001B6903F08003002B0DD00A4B0A4A5A60C0
:105F7C00084B0A4A5A60074B1B6903F08003002B3D
:105F8C0001D00123FB71FB7918460C37BD4680BC50
:105F9C00704700BF0020024023016745AB89EFCD5D
:105FAC0080B400AF054B1B69044A43F080031361B6
:105FBC0000231846BD4680BC704700BF002002403D
:105FCC0080B483B000AF78600B467B80084B002216
:105FDC00DA61084B1B69074A43F0010313617B68C4
:105FEC007A881A8000BF0C37BD4680BC704700BF52
:105FFC00780400200020024080B584B000AF7860A7
:10600C00FFF760F8F86010E07B68B3F1FF3F0CD04D
:10601C007B68002B07D0FFF755F80246FB68D31AB4
:10602C007A689A4201D2032325E0154BDB6803F012
:10603C000103002BE8D1124BDB6803F02003002B8B
:10604C0002D00F4B2022DA600D4BDB6803F01003FB
:10605C00002B0BD10A4BDB6903F00103002B05D19C
:10606C00074BDB6803F00403002B03D000F00AF8A5
:10607C00012300E0002318461037BD4680BD00BF49
:10608C000020024080B483B000AF00237B60234B20
:10609C00DB6803F01003002B09D0214BDB6943F0C4
:1060AC0002031F4AD3617B6843F010037B601B4BD8
:1060BC00DB6803F00403002B09D0194BDB6943F0B8
:1060CC000103174AD3617B6843F004037B60134BD5
:1060DC00DB6903F00103002B0BD0114BDB6943F0A0
:1060EC0004030F4AD3610D4BDB690C4A23F0010307
:1060FC00D3617B6840F20112934206D1074BDB69F6
:10610C00064A23F00103D36102E0044A7B68D360A2
:10611C0000BF0C37BD4680BC704700BF002002405A
:10612C007804002080B584B000AF7860396001231A
:10613C00FB730023BB602F4B1B7E012B01D1022371
:10614C0053E02C4B01221A767B681B68022B16D16C
:10615C004CF25030FFF750FF0346002B41D1012089
:10616C0000F04CF84CF25030FFF746FF0346FB733F
:10617C00214B1B69204A23F00403136131E04CF2DC
:10618C005030FFF739FF0346002B2AD13B684FF004
:10619C00FF321A607B689B68BB6019E0B86800F03E
:1061AC0049F84CF25030FFF727FF0346FB73124BB4
:1061BC001B69114A23F002031361FB7B002B03D0F4
:1061CC003B68BA681A600CE0BB6803F58063BB607F
:1061DC007B68DB689A027B689B681344BA689A42B6
:1061EC00DCD3044B00221A76FB7B18461037BD46D5
:1061FC0080BD00BF780400200020024080B483B032
:10620C0000AF7860094B0022DA61094B1B69084A20
:10621C0043F004031361064B1B69054A43F040032A
:10622C00136100BF0C37BD4680BC7047780400205A
:10623C000020024080B483B000AF78600B4B00228A
:10624C00DA610B4B1B690A4A43F002031361084ADB
:10625C007B685361064B1B69054A43F0400313618D
:10626C0000BF0C37BD4680BC704700BF78040020CF
:10627C000020024080B48BB000AF786039600023FE
:10628C007B6200233B6269E101227B6A02FA03F321
:10629C00FB613B681B68FA691340BB61BA69FB6917
:1062AC009A4240F058813B685B689A4A93425ED0B0
:1062BC00984A934275D8984A934258D0964A93423A
:1062CC006FD8964A934252D0944A934269D8944AD2
:1062DC0093424CD0924A934263D8924A934246D00E
:1062EC00904A93425DD8122B2AD8122B59D801A26E
:1062FC0052F823F07B6300085563000867630008BD
:10630C00A9630008AF630008AF630008AF6300081F
:10631C00AF630008AF630008AF630008AF63000809
:10632C00AF630008AF630008AF630008AF630008F9
:10633C00AF630008AF6300085D6300087163000879
:10634C00794A934213D02CE03B68DB683B6229E02E
:10635C003B68DB6804333B6224E03B68DB68083352
:10636C003B621FE03B68DB680C333B621AE03B6826
:10637C009B68002B02D104233B6213E03B689B68B3
:10638C00012B05D108233B627B68FA691A6109E08D
:10639C0008233B627B68FA695A6103E000233B6285
:1063AC0000E000BFBB69FF2B01D87B6801E07B6874
:1063BC0004337B61BB69FF2B02D87B6A9B0002E034
:1063CC007B6A083B9B003B617B691A680F213B6928
:1063DC0001FA03F3DB431A40396A3B6901FA03F310
:1063EC001A437B691A603B685B6803F08053002B8F
:1063FC0000F0B1804D4B9B694C4A43F00103936113
:10640C004A4B9B6903F00103BB60BB68484A7B6A3B
:10641C009B08023352F82330FB607B6A03F00303C2
:10642C009B000F2202FA03F3DB43FA681340FB6074
:10643C007B68404A934213D07B683F4A93420DD00D
:10644C007B683E4A934207D07B683D4A934201D118
:10645C00032306E0042304E0022302E0012300E00E
:10646C0000237A6A02F0030292009340FA68134305
:10647C00FB602F497B6A9B080233FA6841F82320A2
:10648C003B685B6803F48013002B06D02D4B9A6895
:10649C002C49BB6913438B6006E02A4B9A68BB6995
:1064AC00DB43284913408B603B685B6803F40013A3
:1064BC00002B06D0234BDA682249BB691343CB600F
:1064CC0006E0204BDA68BB69DB431E491340CB6006
:1064DC003B685B6803F40033002B06D0194B5A68F9
:1064EC001849BB6913434B6006E0164B5A68BB69ED
:1064FC00DB43144913404B603B685B6803F4803307
:10650C00002B21D00F4B1A680E49BB6913430B604B
:10651C0021E000BF000032100000311000002210FA
:10652C000000211000001210000011100010024099
:10653C000000014000080140000C01400010014027
:10654C0000140140000401400B4B1A68BB69DB438B
:10655C00094913400B607B6A01337B623B681A6804
:10656C007B6A22FA03F3002B7FF48EAE00BF00BFD0
:10657C002C37BD4680BC70470004014080B485B008
:10658C0000AF78600B467B807B689A687B881340F1
:10659C00002B02D00123FB7301E00023FB73FB7B78
:1065AC0018461437BD4680BC704780B483B000AF2A
:1065BC0078600B467B8013467B707B78002B03D076
:1065CC007A887B681A6103E07B881A047B681A61FD
:1065DC0000BF0C37BD4680BC704780B584B000AF9F
:1065EC0078607B68002B01D10123E8E07B6893F88D
:1065FC009132DBB2002B06D17B68002283F890220B
:10660C00786807F017FC7B68032283F891227B687B
:10661C0000225A717B681B68184603F0BCFA7B6831
:10662C0018687B6804330ECB03F092FA0346002BF8
:10663C0005D07B68022283F891220123BFE07B689E
:10664C001B680021184603F0C0FA0346002B05D046
:10665C007B68022283F891220123B0E00023FB73B4
:10666C003EE0FA7B796813469B001344DB000B4435
:10667C00113301221A70FA7B796813469B0013447C
:10668C00DB000B441033FA7B1A70FA7B79681346E3
:10669C009B001344DB000B44133300221A70FA7B6B
:1066AC00796813469B001344DB000B442033002213
:1066BC001A60FA7B796813469B001344DB000B4489
:1066CC00243300221A60FB7B79685A1C13469B000A
:1066DC001344DB000B4400221A60FB7B0133FB7379
:1066EC007B681B79FA7B9A42BBD30023FB7344E093
:1066FC00FA7B796813469B001344DB000B4403F2CE
:10670C00511300221A70FA7B796813469B001344CC
:10671C00DB000B4403F5A873FA7B1A70FA7B7968DB
:10672C0013469B001344DB000B4403F2531300226B
:10673C001A70FA7B796813469B001344DB000B44F8
:10674C0003F5B07300221A60FA7B796813469B003C
:10675C001344DB000B4403F5B27300221A60FA7B7E
:10676C00796813469B001344DB000B4403F5B473A8
:10677C0000221A60FB7B0133FB737B681B79FA7B6D
:10678C009A42B5D37B6818687B6804330ECB03F050
:10679C0028FA0346002B05D07B68022283F891224D
:1067AC0001230CE07B6800225A737B68012283F87A
:1067BC0091227B681B68184605F0A7FC002318463D
:1067CC001037BD4680BD80B582B000AF78607B6865
:1067DC0093F89032012B01D1022316E07B68012241
:1067EC0083F890227B681B68184603F0BEF90121E0
:1067FC00786807F092FD7B681B68184605F07BFCF7
:10680C007B68002283F89022002318460837BD4687
:10681C0080BD80B588B000AF78607B681B68184677
:10682C0005F07DFCB861BB6903F40043002B03D079
:10683C00786800F01AFB19E1BB6903F48063002B44
:10684C0013D07B681B68B3F844309AB27B681B6822
:10685C0022F4806292B2A3F84420786807F065FBBA
:10686C000021786800F005F900E1BB6903F480436E
:10687C00002B0CD07B681B68B3F844309AB27B6851
:10688C001B6822F4804292B2A3F84420EEE0BB696C
:10689C0003F40053002B0CD07B681B68B3F8443016
:1068AC009AB27B681B6822F4005292B2A3F844207F
:1068BC00DCE0BB6903F48053002B27D07B681B689A
:1068CC00B3F840309AB27B681B6822F0040292B293
:1068DC00A3F840207B681B68B3F840309AB27B6801
:1068EC001B6822F0080292B2A3F84020786807F0E7
:1068FC0055FB7B681B68B3F844309AB27B681B6805
:10690C0022F4805292B2A3F84420AFE0BB6903F4A6
:10691C000063002B00F083800023FB7710E07B6882
:10692C001B681A46FB7F9B001A44FB7F128892B2AD
:10693C005B0020333B4423F8182CFB7F0133FB779F
:10694C00FB7F072BEBD97B681B68B3F840309AB2FE
:10695C007B681B6842F0010292B2A3F840207B686E
:10696C001B68B3F840309AB27B681B6822F00102B6
:10697C0092B2A3F8402000BF7B681B68B3F8443088
:10698C009BB203F48063002BF6D07B681B68B3F8D2
:10699C0044309AB27B681B6822F4806292B2A3F8EE
:1069AC0044200023FB770FE0FB7F7A6812681146C6
:1069BC00FA7F92000A445B0020333B4433F8183CC6
:1069CC001380FB7F0133FB77FB7F072BECD97B68B4
:1069DC001B68B3F840309AB27B681B6842F008021F
:1069EC0092B2A3F840207B681B68B3F844309AB28B
:1069FC007B681B6822F4006292B2A3F844207B6887
:106A0C001B68B3F840309AB27B681B6842F00402F2
:106A1C0092B2A3F84020786807F0A6FA26E0BB698A
:106A2C0003F40073002B0FD07B681B68B3F8443061
:106A3C009AB27B681B6822F4007292B2A3F84420CD
:106A4C00786807F064FA11E0BB6903F48073002BDB
:106A5C000CD07B681B68B3F844309AB27B681B6817
:106A6C0022F4807292B2A3F8442000BF2037BD46B6
:106A7C0080BD80B582B000AF78600B46FB707B6840
:106A8C0093F89032012B01D1022312E07B68012292
:106A9C0083F890227B68FA785A737B681B68FA78C3
:106AAC001146184605F014FB7B68002283F89022EF
:106ABC00002318460837BD4680BD80B584B000AFB2
:106ACC007860084611461A460346FB700B463B801D
:106ADC001346BB700023FB7297F90330002B0EDAC0
:106AEC00FB7803F0070213469B001344DB001033C2
:106AFC007A681344FB60FB6801225A700EE0FB7845
:106B0C0003F0070213469B001344DB0003F5A87344
:106B1C007A681344FB60FB6800225A70FB7803F020
:106B2C000703DAB2FB681A703A88FB681A61FB68D3
:106B3C00BA78DA70BB78022B02D1FB6800221A718A
:106B4C007B6893F89032012B01D102230EE07B6815
:106B5C00012283F890227B681B68F968184603F0C1
:106B6C005DF87B68002283F89022FB7A1846103778
:106B7C00BD4680BD80B584B000AF78600B46FB701D
:106B8C0097F90330002B0EDAFB7803F0070213465B
:106B9C009B001344DB0010337A681344FB60FB68E2
:106BAC0001225A700EE0FB7803F0070213469B009B
:106BBC001344DB0003F5A8737A681344FB60FB688D
:106BCC0000225A70FB7803F00703DAB2FB681A70E4
:106BDC007B6893F89032012B01D102230EE07B6885
:106BEC00012283F890227B681B68F968184603F031
:106BFC00D5FB7B68002283F89022002318461037BF
:106C0C00BD4680BD80B586B000AFF8607A603B6051
:106C1C000B46FB72FB7A03F0070213469B001344EE
:106C2C00DB0003F5A873FA6813447B617B697A680F
:106C3C005A617B693A689A617B690022DA617B69E7
:106C4C0000225A70FB7A03F00703DAB27B691A70E0
:106C5C00FB681B687969184603F08CFD0023184605
:106C6C001837BD4680BD80B483B000AF78600B464A
:106C7C00FB70FB7803F00702796813469B00134402
:106C8C00DB000B4403F5B6731B6818460C37BD4686
:106C9C0080BC704780B586B000AFF8607A603B600E
:106CAC000B46FB72FB7A03F0070213469B0013445E
:106CBC00DB001033FA6813447B617B697A685A6194
:106CCC007B693A689A617B69012283F824207B698D
:106CDC003A681A627B690022DA617B6901225A7078
:106CEC00FB7A03F00703DAB27B691A70FB681B6846
:106CFC007969184603F03EFD002318461837BD4647
:106D0C0080BD80B584B000AF78600B46FB70FB781B
:106D1C0003F007037A681279934201D901234CE0FE
:106D2C0097F90330002B0EDAFB7803F007021346B9
:106D3C009B001344DB0010337A681344FB60FB6840
:106D4C0001225A700CE0FA7813469B001344DB00C6
:106D5C0003F5A8737A681344FB60FB6800225A7031
:106D6C00FB6801229A70FB7803F00703DAB2FB6828
:106D7C001A707B6893F89032012B01D102231CE02E
:106D8C007B68012283F890227B681B68F96818469F
:106D9C0005F0A1F8FB7803F00703002B08D17B6802
:106DAC001A687B6803F526731946104605F0C6F978
:106DBC007B68002283F89022002318461037BD46CA
:106DCC0080BD80B584B000AF78600B46FB70FB785B
:106DDC0003F00F037A681279934201D9012340E042
:106DEC0097F90330002B0EDAFB7803F007021346F9
:106DFC009B001344DB0010337A681344FB60FB6880
:106E0C0001225A700EE0FB7803F0070213469B0038
:106E1C001344DB0003F5A8737A681344FB60FB682A
:106E2C0000225A70FB6800229A70FB7803F007036B
:106E3C00DAB2FB681A707B6893F89032012B01D19F
:106E4C0002230EE07B68012283F890227B681B688A
:106E5C00F968184605F08FF87B68002283F89022B9
:106E6C00002318461037BD4680BD80B596B000AFE4
:106E7C007860BBE37B681B68B3F84430A7F84E30EE
:106E8C00B7F84E30DBB203F00F0387F84D3097F8AC
:106E9C004D30002B40F07581B7F84E3003F01003E5
:106EAC00002B4ED17B681B681B889BB223F4E143FB
:106EBC0023F07003FB817B681A68FB896FEA4343FC
:106ECC006FEA53439BB213807B6810337B657B68FE
:106EDC001B68B3F850309BB21A467B6D1B78DB00F5
:106EEC00134402335B007A681268134403F5806321
:106EFC001B88C3F309027B6DDA617B6D5A697B6D6C
:106F0C00DB691A447B6D5A610021786806F0E5FF55
:106F1C007B685B7BDBB2002B00F068837B6D9B692D
:106F2C00002B40F063837B685B7BDBB263F07F03F9
:106F3C00DAB27B681B68A3F84C207B6800225A737A
:106F4C0054E37B6803F5A8737B657B681B681B881F
:106F5C00A7F84A30B7F84A3003F40063002B34D05A
:106F6C007B681B68B3F850309BB21A467B6D1B785C
:106F7C00DB00134406335B007A681268134403F594
:106F8C0080631B88C3F309027B6DDA617B68186828
:106F9C007B6803F526717B6DDA887B6DDB699BB2B0
:106FAC0005F01DF97B681B681B889AB240F68F733D
:106FBC0013403B827B681B683A8A42F0800292B293
:106FCC001A80786806F05CFF10E3B7F94A30002BA2
:106FDC0080F20C837B681B681B889AB240F68F7317
:106FEC001340FB837B681B68FA8B42F0800292B2E1
:106FFC001A807B681B68B3F850309BB21A467B6DC5
:10700C001B78DB00134406335B007A681268134468
:10701C0003F580631B88C3F309027B6DDA617B6D1A
:10702C00DB69002B19D07B6D5B69002B15D07B685D
:10703C0018687B6D59697B6DDA887B6DDB699BB257
:10704C0005F0CDF87B6D5A697B6DDB691A447B6D5D
:10705C005A610021786806F025FF7B681B681B8845
:10706C00A7F84A30B7F84A3003F40063002B40F01D
:10707C00BD82B7F84A3003F44053B3F5405F00F0DB
:10708C00B5827B681B68BB617B681B68B3F85030AA
:10709C009BB21A46BB691344BB61BB6903F20C4338
:1070AC007B617B691B889BB2C3F309039AB27B6932
:1070BC001A807B6D1B693E2B1DD97B6D1B695B098F
:1070CC007B647B6D1B6903F01F03002B02D17B6C6F
:1070DC00013B7B647B691B889AB27B6C9BB29B02E5
:1070EC009BB213439BB26FEA43436FEA53439AB28A
:1070FC007B691A8026E07B6D1B69002B0AD17B69AA
:10710C001B889BB26FEA43436FEA53439AB27B6985
:10711C001A8017E07B6D1B695B087B647B6D1B69B8
:10712C0003F00103002B02D07B6C01337B647B6981
:10713C001B889AB27B6C9BB29B029BB213439AB294
:10714C007B691A807B681B681B889BB223F4804385
:10715C0023F070037B827B8A83F480537B827B8A4F
:10716C0083F400537B827B681A687B8A43F07F43ED
:10717C0043F47F0343F4004343F080039BB213803A
:10718C0034E27B681B681A4697F84D309B00134419
:10719C001B88A7F84A30B7F94A30002B80F2FC80E4
:1071AC007B681B681A4697F84D309B0013441B886C
:1071BC009AB240F68F731340A7F848307B681B686F
:1071CC001A4697F84D309B001344B7F8482042F00C
:1071DC00800292B21A8097F84D2013469B001344FC
:1071EC00DB0003F5A8737A6813447B657B6D1B7B0E
:1071FC00002B25D17B681B68B3F850309BB21A4624
:10720C007B6D1B78DB00134406335B007A681268D5
:10721C00134403F580631B88C3F30903A7F85030AC
:10722C00B7F85030002B00F092807B6818687B6DAB
:10723C0059697B6DDA88B7F8503004F0D0FF86E0DE
:10724C007B6DDB78022B0AD1B7F84A301A46796D80
:10725C00786800F0D9F90346A7F8503077E07B68DE
:10726C001B681A467B6D1B789B0013441B889BB2D2
:10727C0023F4E04323F07003A7F852307B681B68BB
:10728C001A467B6D1B789B001A44B7F8523043F0BA
:10729C007F4343F47F0343F4004343F0C0039BB2AA
:1072AC0013807B681B681A467B6D1B789B0013440C
:1072BC001B889BB203F48043002B24D07B681B6893
:1072CC00B3F850309BB21A467B6D1B78DB0013442D
:1072DC0002335B007A681268134403F580631B88E1
:1072EC00C3F30903A7F85030B7F85030002B2ED059
:1072FC007B6818687B6D59697B6D1A89B7F85030BB
:10730C0004F06DFF23E07B681B68B3F850309BB230
:10731C001A467B6D1B78DB00134406335B007A68DE
:10732C001268134403F580631B88C3F30903A7F8A1
:10733C005030B7F85030002B09D07B6818687B6D43
:10734C0059697B6D5A89B7F8503004F048FF7B6D52
:10735C00DA69B7F850301A447B6DDA617B6D5A6983
:10736C00B7F850301A447B6D5A617B6D9B69002BCA
:10737C0005D0B7F850207B6D1B699A4206D27B6D05
:10738C001B781946786806F08DFD05E07B681B6854
:10739C00796D184603F0EEF9B7F84A3003F0800324
:1073AC00002B00F0238197F84D2013469B001344CB
:1073BC00DB0010337A6813447B657B681B681A46C4
:1073CC0097F84D309B0013441B889BB223F4E14388
:1073DC0023F07003A7F842307B681B681A4697F8B5
:1073EC004D309B001A44B7F842306FEA43436FEAC2
:1073FC0053439BB213807B6DDB78012B40F0A28052
:10740C007B6D00229A617B6D1B7B002B00F09380BF
:10741C00B7F84A3003F04003002B46D07B6D5B7805
:10742C00002B26D17B681B687B627B681B68B3F8DA
:10743C0050309BB21A467B6A13447B627B6D1B787F
:10744C001A017B6A134403F204433B623B6A1B88B8
:10745C009BB2C3F309039AB23B6A1A803B6A1B883E
:10746C009BB26FEA43436FEA53439AB23B6A1A806A
:10747C0061E07B6D5B78012B5DD17B681B68FB62E7
:10748C007B681B68B3F850309BB21A46FB6A1344F6
:10749C00FB627B6D1B781A01FB6A134403F20443F5
:1074AC00BB62BB6A00221A8045E07B681B68FB63E9
:1074BC007B6D5B78002B26D17B681B687B637B68BC
:1074CC001B68B3F850309BB21A467B6B13447B633A
:1074DC007B6D1B781A017B6B134403F20C433B63EB
:1074EC003B6B1B889BB2C3F309039AB23B6B1A80AC
:1074FC003B6B1B889BB26FEA43436FEA53439AB2D0
:10750C003B6B1A8017E07B6D5B78012B13D17B688A
:10751C001B68B3F850309BB21A46FB6B1344FB63E9
:10752C007B6D1B781A01FB6B134403F20C43BB639A
:10753C00BB6B00221A807B6D1B781946786806F0AD
:10754C00CCFC53E0B7F84A3003F48073002B46D1DF
:10755C007B681B68B3F850309BB21A467B6D1B7866
:10756C00DB00134402335B007A681268134403F5A2
:10757C0080631B88C3F30903A7F840307B6D9A69BD
:10758C00B7F840309A4207D97B6D9A69B7F840300A
:10759C00D21A7B6D9A6102E07B6D00229A617B6D41
:1075AC009B69002B06D17B6D1B781946786806F019
:1075BC0094FC1BE07B6D5A69B7F840301A447B6D24
:1075CC005A617B6DDA69B7F840301A447B6DDA6129
:1075DC007B681B68796D184603F0CCF806E0B7F8A9
:1075EC004A301A46796D786800F01BF97B681B6885
:1075FC00B3F844309BB21BB2002BFFF63BAC00231C
:10760C0018465837BD4680BD80B588B000AFF860CD
:10761C00B9601346FB80FB8803F48043002B7ED0BB
:10762C00FB681B68B3F850309BB21A46BB681B78DA
:10763C00DB00134402335B00FA681268134403F551
:10764C0080631B88C3F309037B83BB689A697B8BBC
:10765C009A4206D3BB689A697B8BD21ABB689A6133
:10766C0002E0BB6800229A61BB689B69002B23D1A6
:10767C00FB681B681A46BB681B789B0013441B886D
:10768C009BB223F4804323F070033B833B8B83F446
:10769C0000533B83FB681B681A46BB681B789B0036
:1076AC001A443B8B43F07F4343F47F0343F4004382
:1076BC0043F080039BB21380FB8803F04003002B44
:1076CC001FD0FB681B681A46BB681B789B001344D1
:1076DC001B889BB223F4E04323F07003FB82FB680E
:1076EC001B681A46BB681B789B001A44FB8A43F044
:1076FC007F4343F47F0343F4004343F0C0039BB246
:10770C0013807B8B002B00F08780FB681868BB68AC
:10771C005969BB681A897B8B04F061FD7CE0FB68BE
:10772C001B68B3F850309BB21A46BB681B78DB0061
:10773C00134406335B00FA681268134403F5806344
:10774C001B88C3F309037B83BB689A697B8B9A42C2
:10775C0006D3BB689A697B8BD21ABB689A6102E02C
:10776C00BB6800229A61BB689B69002B23D1FB6824
:10777C001B681A46BB681B789B0013441B889BB282
:10778C0023F4804323F07003FB83FB8B83F40053BF
:10779C00FB83FB681B681A46BB681B789B001A446A
:1077AC00FB8B43F07F4343F47F0343F4004343F0EC
:1077BC0080039BB21380FB8803F04003002B1FD186
:1077CC00FB681B681A46BB681B789B0013441B881C
:1077DC009BB223F4E04323F07003BB83FB681B686C
:1077EC001A46BB681B789B001A44BB8B43F07F4343
:1077FC0043F47F0343F4004343F0C0039BB2138074
:10780C007B8B002B08D0FB681868BB685969BB6878
:10781C005A897B8B04F0E3FC7B8B18462037BD46E2
:10782C0080BD80B5A4B000AFF860B9601346FB8092
:10783C00FB8803F04003002B00F0DD81FB681B6824
:10784C00B3F850309BB21A46BB681B78DB0013446C
:10785C0002335B00FA681268134403F580631B88DB
:10786C00C3F30903A7F88630BB689A69B7F886306A
:10787C009A4207D9BB689A69B7F88630D21ABB68A6
:10788C009A6102E0BB6800229A61BB689B69002B7D
:10789C0040F0B980BB685B78002B26D1FB681B6875
:1078AC00FB62FB681B68B3F850309BB21A46FB6A4C
:1078BC001344FB62BB681B781A01FB6A134403F286
:1078CC000443BB62BB6A1B889BB2C3F309039AB225
:1078DC00BB6A1A80BB6A1B889BB26FEA43436FEA90
:1078EC0053439AB2BB6A1A801AE0BB685B78012BCF
:1078FC0016D1FB681B687B63FB681B68B3F85030C0
:10790C009BB21A467B6B13447B63BB681B781A01D2
:10791C007B6B134403F204433B633B6B00221A80E2
:10792C00FB681B687B62BB685B78002B26D1FB680D
:10793C001B68FB61FB681B68B3F850309BB21A469E
:10794C00FB691344FB61BB681B781A01FB69134488
:10795C0003F20C43BB61BB691B889BB2C3F30903E5
:10796C009AB2BB691A80BB691B889BB26FEA43430E
:10797C006FEA53439AB2BB691A8017E0BB685B7815
:10798C00012B13D1FB681B68B3F850309BB21A461D
:10799C007B6A13447B62BB681B781A017B6A1344B5
:1079AC0003F20C433B623B6A00221A80BB681B78D3
:1079BC001946F86806F091FAFB8803F48043002B13
:1079CC0000F0FC82FB681B681A46BB681B789B00A6
:1079DC0013441B889BB223F4E04323F07003FB8217
:1079EC00FB681B681A46BB681B789B001A44FB8A11
:1079FC0043F07F4343F47F0343F4404343F080035D
:107A0C009BB21380DAE2FB8803F48043002B21D075
:107A1C00FB681B681A46BB681B789B0013441B88C9
:107A2C009BB223F4E04323F07003A7F88A30FB6881
:107A3C001B681A46BB681B789B001A44B7F88A303F
:107A4C0043F07F4343F47F0343F4404343F080030C
:107A5C009BB21380BB6893F82430012B40F0AE82AC
:107A6C00BB685A69B7F886301A44BB685A61BB6860
:107A7C00DA69B7F886301A44BB68DA61BB681A6AEF
:107A8C00BB681B699A420BD3BB681B69C7F88C3067
:107A9C00BB681A6AD7F88C30D21ABB681A6217E026
:107AAC00BB681B6A002B08D1B7F88630C7F88C303E
:107ABC00BB68002283F824200AE0BB68002283F80C
:107ACC002420BB681B6AC7F88C30BB6800221A6282
:107ADC00BB685B78002B65D1FB681B68FB63FB689C
:107AEC001B68B3F850309BB21A46FB6B1344FB6314
:107AFC00BB681B781A01FB6B134403F20443BB6392
:107B0C00BB6B1B889BB2C3F309039AB2BB6B1A8085
:107B1C00D7F88C303E2B1DD9D7F88C305B09BB6461
:107B2C00D7F88C3003F01F03002B02D1BB6C013B48
:107B3C00BB64BB6B1B889AB2BB6C9BB29B029BB2A7
:107B4C0013439BB26FEA43436FEA53439AB2BB6B46
:107B5C001A8044E0D7F88C30002B0AD1BB6B1B8801
:107B6C009BB26FEA43436FEA53439AB2BB6B1A80E2
:107B7C0035E0D7F88C305B08BB64D7F88C3003F059
:107B8C000103002B02D0BB6C0133BB64BB6B1B88A5
:107B9C009AB2BB6C9BB29B029BB213439AB2BB6B67
:107BAC001A801CE0BB685B78012B18D1FB681B6842
:107BBC007B64FB681B68B3F850309BB21A467B6C35
:107BCC0013447B64BB681B781A017B6C134403F26F
:107BDC0004433B64D7F88C309AB23B6C1A80FB6838
:107BEC001868BB685969BB681A89D7F88C309BB286
:107BFC0004F0AFFAE2E1FB681B68B3F850309BB2BB
:107C0C001A46BB681B78DB00134406335B00FA682A
:107C1C001268134403F580631B88C3F30903A7F8A8
:107C2C008630BB689A69B7F886309A4207D3BB682E
:107C3C009A69B7F88630D21ABB689A6102E0BB68C1
:107C4C0000229A61BB689B69002B40F0C080BB6826
:107C5C005B78002B26D1FB681B68FB67FB681B68F5
:107C6C00B3F850309BB21A46FB6F1344FB67BB68EA
:107C7C001B781A01FB6F134403F20443BB67BB6F01
:107C8C001B889BB2C3F309039AB2BB6F1A80BB6FFC
:107C9C001B889BB26FEA43436FEA53439AB2BB6FA4
:107CAC001A801AE0BB685B78012B16D1FB681B6845
:107CBC007B66FB681B68B3F850309BB21A467B6E30
:107CCC0013447B66BB681B781A017B6E134403F26A
:107CDC0004433B663B6E00221A80FB681B687B6783
:107CEC00BB685B78002B2BD1FB681B68FB66FB68C1
:107CFC001B68B3F850309BB21A46FB6E1344FB66FC
:107D0C00BB681B781A01FB6E134403F20C43C7F8D3
:107D1C008030D7F880301B889BB2C3F309039AB22A
:107D2C00D7F880301A80D7F880301B889BB26FEA66
:107D3C0043436FEA53439AB2D7F880301A8017E066
:107D4C00BB685B78012B13D1FB681B68B3F8503010
:107D5C009BB21A467B6F13447B67BB681B781A0176
:107D6C007B6F134403F20C433B673B6F00221A807A
:107D7C00BB681B781946F86806F0AFF8FB8803F46B
:107D8C008043002B40F01A81FB681B681A46BB68C5
:107D9C001B789B0013441B889BB223F4E04323F015
:107DAC007003A7F88830FB681B681A46BB681B7801
:107DBC009B001A44B7F8883043F07F4343F47F03A9
:107DCC0043F4404343F080039BB21380F6E0FB88FE
:107DDC0003F48043002B21D1FB681B681A46BB6857
:107DEC001B789B0013441B889BB223F4E04323F0C5
:107DFC007003A7F84E30FB681B681A46BB681B78EB
:107E0C009B001A44B7F84E3043F07F4343F47F0392
:107E1C0043F4404343F080039BB21380BB6893F858
:107E2C002430012B40F0CA80BB685A69B7F8863001
:107E3C001A44BB685A61BB68DA69B7F886301A44D1
:107E4C00BB68DA61BB681A6ABB681B699A420BD3C0
:107E5C00BB681B69C7F88C30BB681A6AD7F88C30C2
:107E6C00D21ABB681A6217E0BB681B6A002B08D1D8
:107E7C00B7F88630C7F88C30BB68002283F8242012
:107E8C000AE0BB681B6AC7F88C30BB6800221A6218
:107E9C00BB68002283F82420FB681B687B65BB68E9
:107EAC005B78002B65D1FB681B68FB65FB681B6866
:107EBC00B3F850309BB21A46FB6D1344FB65BB689C
:107ECC001B781A01FB6D134403F20C43BB65BB6DAD
:107EDC001B889BB2C3F309039AB2BB6D1A80D7F807
:107EEC008C303E2B1DD9D7F88C305B09BB66D7F88C
:107EFC008C3003F01F03002B02D1BB6E013BBB6621
:107F0C00BB6D1B889AB2BB6E9BB29B029BB2134398
:107F1C009BB26FEA43436FEA53439AB2BB6D1A802C
:107F2C0041E0D7F88C30002B0AD1BB6D1B889BB27B
:107F3C006FEA43436FEA53439AB2BB6D1A8032E047
:107F4C00D7F88C305B08BB66D7F88C3003F0010394
:107F5C00002B02D0BB6E0133BB66BB6D1B889AB283
:107F6C00BB6E9BB29B029BB213439AB2BB6D1A8041
:107F7C0019E0BB685B78012B15D1FB681B68B3F863
:107F8C0050309BB21A467B6D13447B65BB681B78E3
:107F9C001A017B6D134403F20C433B65D7F88C300C
:107FAC009AB23B6D1A80FB681868BB685969BB684C
:107FBC005A89D7F88C309BB204F0CBF8FB681B685D
:107FCC001A46BB681B789B0013441B889BB223F496
:107FDC00E04323F04003BB82BB8A83F01003BB82D7
:107FEC00BB8A83F02003BB82FB681B681A46BB6804
:107FFC001B789B001A44BB8A43F07F4343F47F03F6
:10800C0043F4004343F080039BB2138000231846D3
:10801C009037BD4680BD80B487B000AFF8607B6000
:10802C000B467B8113463B817B8903F080039BB21B
:10803C00002B0BD07B8903F0070213469B001344E3
:10804C00DB001033FA6813447B6109E07A8913462C
:10805C009B001344DB0003F5A873FA6813447B619F
:10806C003B89002B07D17B6900221A737B689AB27B
:10807C007B69DA800BE07B6901221A737B689AB208
:10808C007B691A817B681B0C9AB27B695A8100232D
:10809C0018461C37BD4680BC7047000080B586B0C2
:1080AC0000AF78607B68002B01D1012372E27B6802
:1080BC001B6803F00103002B00F08780924B5B6878
:1080CC0003F00C03042B0CD08F4B5B6803F00C03F8
:1080DC00082B12D18C4B5B6803F48033B3F5803FD3
:1080EC000BD1894B1B6803F40033002B6CD07B68DD
:1080FC005B68002B68D101234CE27B685B68B3F5AD
:10810C00803F06D1804B1B687F4A43F48033136059
:10811C002EE07B685B68002B0CD17B4B1B687A4A8A
:10812C0023F480331360784B1B68774A23F4802345
:10813C0013601DE07B685B68B3F5A02F0CD1724B0C
:10814C001B68714A43F4802313606F4B1B686E4AA3
:10815C0043F4803313600BE06B4B1B686A4A23F4C7
:10816C0080331360684B1B68674A23F480231360C9
:10817C007B685B68002B13D0FCF7A4FF386108E028
:10818C00FCF7A0FF02463B69D31A642B01D90323E9
:10819C0000E25D4B1B6803F40033002BF0D014E0BD
:1081AC00FCF790FF386108E0FCF78CFF02463B6956
:1081BC00D31A642B01D90323ECE1534B1B6803F452
:1081CC000033002BF0D100E000BF7B681B6803F08C
:1081DC000203002B63D04C4B5B6803F00C03002BA9
:1081EC000BD0494B5B6803F00C03082B1CD1464B9E
:1081FC005B6803F48033002B16D1434B1B6803F0F0
:10820C000203002B05D07B681B69012B01D00123D5
:10821C00C0E13D4B1B6823F0F8027B685B69DB0017
:10822C00394913430B603AE07B681B69002B20D063
:10823C00364B01221A60FCF745FF386108E0FCF769
:10824C0041FF02463B69D31A022B01D90323A1E15A
:10825C002D4B1B6803F00203002BF0D02A4B1B683C
:10826C0023F0F8027B685B69DB00274913430B6042
:10827C0015E0264B00221A60FCF724FF386108E059
:10828C00FCF720FF02463B69D31A022B01D90323CA
:10829C0080E11D4B1B6803F00203002BF0D17B68BF
:1082AC001B6803F00803002B3AD07B689B69002BFA
:1082BC0019D0174B01221A60FCF704FF386108E053
:1082CC00FCF700FF02463B69D31A022B01D90323AA
:1082DC0060E10D4B5B6A03F00203002BF0D0012030
:1082EC0000F0D0FA1CE00A4B00221A60FCF7EAFE00
:1082FC0038610FE0FCF7E6FE02463B69D31A022B0D
:10830C0008D9032346E100BF00100240000042429E
:10831C0080044242924B5B6A03F00203002BE9D1CA
:10832C007B681B6803F00403002B00F0A68000237D
:10833C00FB758B4BDB6903F08053002B0DD1884B05
:10834C00DB69874A43F08053D361854BDB6903F0CB
:10835C008053BB60BB680123FB75824B1B6803F425
:10836C008073002B18D17F4B1B687E4A43F48073BB
:10837C001360FCF7A7FE386108E0FCF7A3FE024689
:10838C003B69D31A642B01D9032303E1754B1B689A
:10839C0003F48073002BF0D07B68DB68012B06D1D3
:1083AC006F4B1B6A6E4A43F0010313622DE07B682E
:1083BC00DB68002B0CD16A4B1B6A694A23F0010362
:1083CC001362674B1B6A664A23F0040313621CE0BA
:1083DC007B68DB68052B0CD1614B1B6A604A43F050
:1083EC00040313625E4B1B6A5D4A43F00103136284
:1083FC000BE05B4B1B6A5A4A23F001031362584B88
:10840C001B6A574A23F0040313627B68DB68002B5A
:10841C0015D0FCF757FE38610AE0FCF753FE024614
:10842C003B69D31A41F28832934201D90323B1E05C
:10843C004B4B1B6A03F00203002BEED014E0FCF74D
:10844C0041FE38610AE0FCF73DFE02463B69D31A57
:10845C0041F28832934201D903239BE0404B1B6AC3
:10846C0003F00203002BEED1FB7D012B05D13C4B1D
:10847C00DB693B4A23F08053D3617B68DB69002BBB
:10848C0000F08780364B5B6803F00C03082B61D03F
:10849C007B68DB69022B46D1334B00221A60FCF758
:1084AC0011FE386108E0FCF70DFE02463B69D31A59
:1084BC00022B01D903236DE0294B1B6803F00073D9
:1084CC00002BF0D17B681B6AB3F5803F08D1244B9D
:1084DC005B6823F400327B689B68214913434B6033
:1084EC001F4B5B6823F474127B68196A7B685B6AA8
:1084FC000B431B4913434B601B4B01221A60FCF7C7
:10850C00E1FD386108E0FCF7DDFD02463B69D31A5A
:10851C00022B01D903233DE0114B1B6803F00073C0
:10852C00002BF0D035E0104B00221A60FCF7CAFD8E
:10853C00386108E0FCF7C6FD02463B69D31A022BF2
:10854C0001D9032326E0064B1B6803F00073002BB4
:10855C00F0D11EE07B68DB69012B07D1012319E008
:10856C000010024000700040600042420B4B5B6800
:10857C00FB60FB6803F480327B681B6A9A4206D16D
:10858C00FB6803F470127B685B6A9A4201D001238A
:10859C0000E0002318461837BD4680BD001002408D
:1085AC0080B584B000AF786039607B68002B01D156
:1085BC000123D0E06A4B1B6803F007033A689A4228
:1085CC0010D9674B1B6823F0070265493B681343BE
:1085DC000B60634B1B6803F007033A689A4201D0A7
:1085EC000123B8E07B681B6803F00203002B20D04A
:1085FC007B681B6803F00403002B05D0594B5B68A8
:10860C00584A43F4E06353607B681B6803F008032B
:10861C00002B05D0534B5B68524A43F460535360B4
:10862C00504B5B6823F0F0027B689B684D49134309
:10863C004B607B681B6803F00103002B40D07B6808
:10864C005B68012B07D1474B1B6803F40033002BED
:10865C0015D101237FE07B685B68022B07D1414B6E
:10866C001B6803F00073002B09D1012373E03D4B11
:10867C001B6803F00203002B01D101236BE0394B83
:10868C005B6823F003027B685B68364913434B60DD
:10869C00FCF718FDF8600AE0FCF714FD0246FB68D5
:1086AC00D31A41F28832934201D9032353E02D4B64
:1086BC005B6803F00C027B685B689B009A42EBD111
:1086CC00274B1B6803F007033A689A4210D2244BDD
:1086DC001B6823F0070222493B6813430B60204BB5
:1086EC001B6803F007033A689A4201D0012332E079
:1086FC007B681B6803F00403002B08D0194B5B68E4
:10870C0023F4E0627B68DB68164913434B607B689B
:10871C001B6803F00803002B09D0124B5B6823F491
:10872C0060527B681B69DB000E4913434B6000F001
:10873C0021F802460B4B5B681B0903F00F030A4937
:10874C00CB5C22FA03F3094A1360094B1B681846E9
:10875C00FCF776FC002318461037BD4680BD00BFE1
:10876C00002002400010024098F400081000002085
:10877C001400002080B487B000AF0023FB600023FE
:10878C00BB6000237B6100237B6000233B611E4B9D
:10879C005B68FB60FB6803F00C03042B02D0082B16
:1087AC0003D027E0194B3B6127E0FB689B0C03F0DF
:1087BC000F03174AD35C7B60FB6803F48033002BF8
:1087CC0010D0114B5B685B0C03F00103114AD35CB6
:1087DC00BB607B680D4A03FB02F2BB68B2FBF3F390
:1087EC007B6104E07B680C4A02FB03F37B617B69D1
:1087FC003B6102E0094B3B6100BF3B6918461C37EB
:10880C00BD4680BC704700BF00100240001BB70083
:10881C00B0F40008C0F4000800093D0000127A0012
:10882C0080B400AF024B1B681846BD4680BC704735
:10883C001000002080B500AFFFF7F2FF0246054B99
:10884C005B681B0A03F007030349CB5C22FA03F3B2
:10885C00184680BD00100240A8F4000880B500AF97
:10886C00FFF7DEFF0246054B5B68DB0A03F00703EC
:10887C000349CB5C22FA03F3184680BD001002407A
:10888C00A8F4000880B485B000AF78600A4B1B6870
:10889C000A4AA2FB03235B0A7A6802FB03F3FB6020
:1088AC0000BFFB685A1EFA60002BF9D100BF00BF55
:1088BC001437BD4680BC704710000020D34D6210A9
:1088CC0080B586B000AF786000233B610023FB606D
:1088DC007B681B6803F00103002B7DD00023FB7524
:1088EC004F4BDB6903F08053002B0DD14C4BDB69F4
:1088FC004B4A43F08053D361494BDB6903F08053FF
:10890C00BB60BB680123FB75464B1B6803F480738B
:10891C00002B18D1434B1B68424A43F480731360FD
:10892C00FCF7D0FB386108E0FCF7CCFB02463B6956
:10893C00D31A642B01D903236DE03A4B1B6803F463
:10894C008073002BF0D0364B1B6A03F44073FB6032
:10895C00FB68002B2ED07B685B6803F44073FA68CD
:10896C009A4227D02E4B1B6A23F44073FB602E4B8C
:10897C0001221A602C4B00221A60294AFB681362F0
:10898C00FB6803F00103002B14D0FCF79BFB386150
:10899C000AE0FCF797FB02463B69D31A41F2883296
:1089AC00934201D9032336E01D4B1B6A03F00203EB
:1089BC00002BEED01A4B1B6A23F440727B685B6869
:1089CC00174913430B62FB7D012B05D1144BDB695B
:1089DC00134A23F08053D3617B681B6803F00203B6
:1089EC00002B08D00E4B5B6823F440427B689B68DD
:1089FC000B4913434B607B681B6803F01003002B7F
:108A0C0008D0074B5B6823F480027B68DB68044961
:108A1C0013434B60002318461837BD4680BD00BF7A
:108A2C0000100240007000404004424280B582B009
:108A3C0000AF78607B68002B01D1012341E07B689B
:108A4C0093F83D30DBB2002B06D17B68002283F813
:108A5C003C207868FCF76AF97B68022283F83D2099
:108A6C007B681A687B6804331946104600F03EFB9D
:108A7C007B68012283F846207B68012283F83E2024
:108A8C007B68012283F83F207B68012283F8402019
:108A9C007B68012283F841207B68012283F8422005
:108AAC007B68012283F843207B68012283F84420F1
:108ABC007B68012283F845207B68012283F83D20E6
:108ACC00002318460837BD4680BD80B582B000AF84
:108ADC0078607B68002B01D1012341E07B6893F81F
:108AEC003D30DBB2002B06D17B68002283F83C20A2
:108AFC00786800F039F87B68022283F83D207B68A7
:108B0C001A687B6804331946104600F0EFFA7B684C
:108B1C00012283F846207B68012283F83E207B6883
:108B2C00012283F83F207B68012283F840207B6878
:108B3C00012283F841207B68012283F842207B6864
:108B4C00012283F843207B68012283F844207B6850
:108B5C00012283F845207B68012283F83D20002305
:108B6C0018460837BD4680BD80B483B000AF78602E
:108B7C0000BF0C37BD4680BC7047000080B584B088
:108B8C0000AF786039603B68002B09D17B6893F8A3
:108B9C003E30DBB2012B14BF01230023DBB222E0F9
:108BAC003B68042B09D17B6893F83F30DBB2012B77
:108BBC0014BF01230023DBB215E03B68082B09D15D
:108BCC007B6893F84030DBB2012B14BF01230023E8
:108BDC00DBB208E07B6893F84130DBB2012B14BFA9
:108BEC0001230023DBB2002B01D001235EE03B68A4
:108BFC00002B04D17B68022283F83E2013E03B68F3
:108C0C00042B04D17B68022283F83F200BE03B68E5
:108C1C00082B04D17B68022283F8402003E07B6898
:108C2C00022283F841207B681B68012239681846B0
:108C3C0000F0E8FC7B681B681E4A934207D17B68F6
:108C4C001B685A6C7B681B6842F400425A647B6850
:108C5C001B68184A93420ED07B681B68B3F1804F97
:108C6C0009D07B681B68144A934204D07B681B684C
:108C7C00124A934211D17B681B689B6803F007036F
:108C8C00FB60FB68062B10D07B681B681A687B683E
:108C9C001B6842F001021A6007E07B681B681A68C7
:108CAC007B681B6842F001021A60002318461037DB
:108CBC00BD4680BD002C014000040040000800406F
:108CCC0080B582B000AF786039607B681B68002289
:108CDC003968184600F096FC7B681B68294A934259
:108CEC0017D17B681B681A6A41F211131340002BD1
:108CFC000FD17B681B681A6A40F244431340002B67
:108D0C0007D17B681B685A6C7B681B6822F4004295
:108D1C005A647B681B681A6A41F211131340002BCA
:108D2C000FD17B681B681A6A40F244431340002B36
:108D3C0007D17B681B681A687B681B6822F00102EC
:108D4C001A603B68002B04D17B68012283F83E201B
:108D5C0013E03B68042B04D17B68012283F83F208D
:108D6C000BE03B68082B04D17B68012283F8402080
:108D7C0003E07B68012283F8412000231846083762
:108D8C00BD4680BD002C014080B586B000AFF860B8
:108D9C00B9607A600023FB75FB6893F83C30012BBB
:108DAC0001D10223AEE0FB68012283F83C207B68F2
:108DBC000C2B00F29F8001A252F823F0FD8D0008CD
:108DCC00018F0008018F0008018F00083D8E0008FC
:108DDC00018F0008018F0008018F00087F8E0008AA
:108DEC00018F0008018F0008018F0008BF8E00085A
:108DFC00FB681B68B968184600F0E6F9FB681B684D
:108E0C009A69FB681B6842F008029A61FB681B6850
:108E1C009A69FB681B6822F004029A61FB681B6864
:108E2C009969BB681A69FB681B680A439A6164E01C
:108E3C00FB681B68B968184600F02CFAFB681B68C5
:108E4C009A69FB681B6842F400629A61FB681B68B4
:108E5C009A69FB681B6822F480629A61FB681B6844
:108E6C009969BB681B691A02FB681B680A439A6103
:108E7C0043E0FB681B68B968184600F075FAFB689C
:108E8C001B68DA69FB681B6842F00802DA61FB6850
:108E9C001B68DA69FB681B6822F00402DA61FB6864
:108EAC001B68D969BB681A69FB681B680A43DA61DD
:108EBC0023E0FB681B68B968184600F0BFFAFB6832
:108ECC001B68DA69FB681B6842F40062DA61FB68B4
:108EDC001B68DA69FB681B6822F48062DA61FB6844
:108EEC001B68D969BB681B691A02FB681B680A43BB
:108EFC00DA6102E00123FB7500BFFB68002283F8F6
:108F0C003C20FB7D18461837BD4680BD80B584B02B
:108F1C0000AF786039600023FB737B6893F83C30BA
:108F2C00012B01D10223B4E07B68012283F83C20A1
:108F3C007B68022283F83D207B681B689B68BB60C2
:108F4C00BB6823F07703BB60BB6823F47F43BB6033
:108F5C007B681B68BA689A603B681B68B3F5005F56
:108F6C003ED0B3F5005F00F28780B3F5805F00F070
:108F7C008680B3F5805F7FD8702B1AD0702B7BD88E
:108F8C00602B50D0602B77D8502B3CD0502B73D803
:108F9C00402B58D0402B6FD8302B64D0302B6BD853
:108FAC00202B60D0202B67D8002B5CD0102B5AD0F4
:108FBC0062E07B6818683B6899683B685A683B6854
:108FCC00DB6800F000FB7B681B689B68BB60BB68C0
:108FDC0043F07703BB607B681B68BA689A604FE00C
:108FEC007B6818683B6899683B685A683B68DB6823
:108FFC0000F0E9FA7B681B689A687B681B6842F48E
:10900C0080429A603CE07B6818683B6859683B6812
:10901C00DB681A4600F060FA7B681B685021184622
:10902C0000F0B7FA2CE07B6818683B6859683B681D
:10903C00DB681A4600F07EFA7B681B6860211846D4
:10904C0000F0A7FA1CE07B6818683B6859683B681D
:10905C00DB681A4600F040FA7B681B684021184612
:10906C0000F097FA0CE07B681A683B681B6819469D
:10907C00104600F08EFA03E00123FB7300E000BF02
:10908C007B68012283F83D207B68002283F83C201A
:10909C00FB7B18461037BD4680BD80B485B000AF51
:1090AC00786039603B68002B04D17B6893F83E30C4
:1090BC00DBB213E03B68042B04D17B6893F83F30A0
:1090CC00DBB20BE03B68082B04D17B6893F8403093
:1090DC00DBB203E07B6893F84130DBB2FB73FB7BC4
:1090EC0018461437BD4680BC7047000080B485B06C
:1090FC0000AF786039607B681B68FB607B682F4A27
:10910C0093420BD07B68B3F1804F07D07B682C4A1D
:10911C00934203D07B682B4A934208D1FB6823F01F
:10912C007003FB603B685B68FA681343FB607B6809
:10913C00224A93420BD07B68B3F1804F07D07B68F7
:10914C001F4A934203D07B681E4A934208D1FB68A6
:10915C0023F44073FB603B68DB68FA681343FB60E5
:10916C00FB6823F080023B685B691343FB607B6800
:10917C00FA681A603B689A687B68DA623B681A681E
:10918C007B689A627B680D4A934203D13B681A69EB
:10919C007B681A637B6801225A617B681B6903F048
:1091AC000103002B05D07B681B6923F001027B684F
:1091BC001A6100BF1437BD4680BC7047002C0140BB
:1091CC00000400400008004080B487B000AF786015
:1091DC0039607B681B6A7B617B681B6A23F0010228
:1091EC007B681A627B685B683B617B689B69FB6090
:1091FC00FB6823F07003FB60FB6823F00303FB6048
:10920C003B681B68FA681343FB607B6923F002031D
:10921C007B613B689B687A6913437B617B681C4A62
:10922C0093420CD17B6923F008037B613B68DB68BC
:10923C007A6913437B617B6923F004037B617B6850
:10924C00134A934211D13B6923F480733B613B6910
:10925C0023F400733B613B685B693A6913433B61E0
:10926C003B689B693A6913433B617B683A695A6076
:10927C007B68FA689A613B685A687B685A637B68BA
:10928C007A691A6200BF1C37BD4680BC704700BFAC
:10929C00002C014080B487B000AF786039607B68E7
:1092AC001B6A7B617B681B6A23F010027B681A6265
:1092BC007B685B683B617B689B69FB60FB6823F4A4
:1092CC00E043FB60FB6823F44073FB603B681B6866
:1092DC001B02FA681343FB607B6923F020037B615C
:1092EC003B689B681B017A6913437B617B681D4A51
:1092FC0093420DD17B6923F080037B613B68DB6873
:10930C001B017A6913437B617B6923F040037B610A
:10931C007B68144A934213D13B6923F480633B610D
:10932C003B6923F400633B613B685B699B003A69D2
:10933C0013433B613B689B699B003A6913433B6158
:10934C007B683A695A607B68FA689A613B685A682C
:10935C007B689A637B687A691A6200BF1C37BD46CA
:10936C0080BC7047002C014080B487B000AF78609F
:10937C0039607B681B6A7B617B681B6A23F4807293
:10938C007B681A627B685B683B617B68DB69FB60AE
:10939C00FB6823F07003FB60FB6823F00303FB60A6
:1093AC003B681B68FA681343FB607B6923F400730A
:1093BC007B613B689B681B027A6913437B617B680A
:1093CC001D4A93420DD17B6923F400637B613B689A
:1093DC00DB681B027A6913437B617B6923F480632E
:1093EC007B617B68144A934213D13B6923F480530D
:1093FC003B613B6923F400533B613B685B691B0198
:10940C003A6913433B613B689B691B013A691343FF
:10941C003B617B683A695A607B68FA68DA613B6841
:10942C005A687B68DA637B687A691A6200BF1C37FA
:10943C00BD4680BC704700BF002C014080B487B093
:10944C0000AF786039607B681B6A3B617B681B6A84
:10945C0023F480527B681A627B685B687B617B6853
:10946C00DB69FB60FB6823F4E043FB60FB6823F4DF
:10947C004073FB603B681B681B02FA681343FB607C
:10948C003B6923F400533B613B689B681B033A69BF
:10949C0013433B617B680F4A934209D17B6923F4E8
:1094AC0080437B613B685B699B017A6913437B61F9
:1094BC007B687A695A607B68FA68DA613B685A683B
:1094CC007B681A647B683A691A6200BF1C37BD4618
:1094DC0080BC7047002C014080B487B000AFF860AE
:1094EC00B9607A60FB681B6A7B61FB681B6A23F0BE
:1094FC000102FB681A62FB689B693B613B6923F0C4
:10950C00F0033B617B681B013A6913433B617B6948
:10951C0023F00A037B617A69BB6813437B61FB68A8
:10952C003A699A61FB687A691A6200BF1C37BD46BA
:10953C0080BC704780B487B000AFF860B9607A60C7
:10954C00FB681B6A7B61FB681B6A23F01002FB68DB
:10955C001A62FB689B693B613B6923F470433B6176
:10956C007B681B033A6913433B617B6923F0A003BF
:10957C007B61BB681B017A6913437B61FB683A69A9
:10958C009A61FB687A691A6200BF1C37BD4680BCC1
:10959C00704780B485B000AF786039607B689B6899
:1095AC00FB60FB6823F07003FB603A68FB681343B5
:1095BC0043F00703FB607B68FA689A6000BF1437BE
:1095CC00BD4680BC704780B487B000AFF860B9600E
:1095DC007A603B60FB689B687B617B6923F47F430B
:1095EC007B613B681A027B681A43BB6813437A6938
:1095FC0013437B61FB687A699A6000BF1C37BD46D8
:10960C0080BC704780B487B000AFF860B9607A60F6
:10961C00BB6803F01F03012202FA03F37B61FB68B2
:10962C001A6A7B69DB431A40FB681A62FB681A6A88
:10963C00BB6803F01F03796801FA03F31A43FB6854
:10964C001A6200BF1C37BD4680BC704780B485B021
:10965C0000AF786039607B6893F83C30012B01D106
:10966C00022346E07B68012283F83C207B680222BF
:10967C0083F83D207B681B685B68FB607B681B681C
:10968C009B68BB60FB6823F07003FB603B681B6846
:10969C00FA681343FB607B681B68FA685A607B6846
:1096AC001B68164A93420ED07B681B68B3F1804F3F
:1096BC0009D07B681B68124A934204D07B681B68F4
:1096CC00104A93420CD1BB6823F08003BB603B680B
:1096DC005B68BA681343BB607B681B68BA689A60A6
:1096EC007B68012283F83D207B68002283F83C20B4
:1096FC00002318461437BD4680BC7047002C01402F
:10970C00000400400008004080B582B000AF7860D3
:10971C007B68002B01D1012342E07B6893F8413038
:10972C00DBB2002B06D17B68002283F840207868DE
:10973C00FBF780FB7B68242283F841207B681B6845
:10974C00DA687B681B6822F40052DA60786800F0F3
:10975C0071F97B681B681A697B681B6822F490425C
:10976C001A617B681B685A697B681B6822F02A02A5
:10977C005A617B681B68DA687B681B6842F400528C
:10978C00DA607B6800225A647B68202283F84120CF
:10979C007B68202283F842207B6800225A630023D6
:1097AC0018460837BD4680BD80B58AB002AFF86058
:1097BC00B9603B601346FB8000237B61FB6893F828
:1097CC004130DBB2202B75D1BB68002B02D0FB885B
:1097DC00002B01D101236EE0FB6800225A64FB6868
:1097EC00212283F84120FBF76DFC7861FB68FA8835
:1097FC009A84FB68FA88DA84FB689B68B3F5805F0F
:10980C0008D1FB681B69002B04D10023FB61BB68EA
:10981C00BB6103E0BB68FB610023BB612EE03B68CE
:10982C0000937B6900228021F86800F048F8034619
:10983C00002B05D0FB68202283F8412003233AE05B
:10984C00FB69002B0BD1BB691B881A46FB681B6894
:10985C00C2F308025A60BB690233BB6107E0FB69C3
:10986C001A78FB681B685A60FB690133FB61FB6863
:10987C00DB8C9BB2013B9AB2FB68DA84FB68DB8C15
:10988C009BB2002BCBD13B6800937B69002240211B
:10989C00F86800F014F80346002B05D0FB68202272
:1098AC0083F84120032306E0FB68202283F8412043
:1098BC00002300E0022318462037BD4680BD80B54A
:1098CC0086B000AFF860B9603B601346FB713BE0BB
:1098DC003B6AB3F1FF3F37D0FBF7F4FB02463B6822
:1098EC00D31A3A6A9A4202D33B6A002B01D1032362
:1098FC003AE0FB681B68DB6803F00403002B23D001
:10990C00BB68802B20D0BB68402B1DD0FB681B682C
:10991C001B6803F00803082B16D100237B61FB683E
:10992C001B681B687B61FB681B685B687B617B69E0
:10993C00F86800F01DF8FB6808225A64FB680022E6
:10994C0083F8402001230FE0FB681B681A68BB6892
:10995C001340BA689A420CBF01230023DBB21A46AB
:10996C00FB799A42B4D0002318461837BD4680BD07
:10997C0080B495B000AF78607B681B680C337B6358
:10998C007B6B53E8003F3B633B6B23F49073FB64AE
:10999C007B681B680C33FA6C3A64FB63F96B3A6CAA
:1099AC0041E80023BB63BB6B002BE5D17B681B68D4
:1099BC0014333B623B6A53E8003FFB61FB6923F0C5
:1099CC000103BB647B681B681433BA6CFA62BB621C
:1099DC00B96AFA6A41E800237B627B6A002BE5D105
:1099EC007B681B6B012B19D17B681B680C33FB60EC
:1099FC00FB6853E8003FBB60BB6823F010037B643B
:109A0C007B681B680C337A6CBA617B617969BA69C3
:109A1C0041E800233B613B69002BE5D17B682022A8
:109A2C0083F842207B6800221A6300BF5437BD467E
:109A3C0080BC704780B584B000AF78607B681B68D1
:109A4C001B6923F440517B68DA687B681B680A4306
:109A5C001A617B689A687B681B691A437B685B692F
:109A6C001343BB607B681B68DB6823F4B05323F0A3
:109A7C000C037A681268B9680B43D3607B681B6867
:109A8C005B6923F440717B689A697B681B680A43A5
:109A9C005A617B681B682C4A934203D1FEF7DEFEA9
:109AAC00F86002E0FEF7C6FEF860FA6813469B0009
:109ABC0013449A001A447B685B689B00B2FBF3F377
:109ACC00224AA2FB03235B091901FA6813469B0087
:109ADC0013449A001A447B685B689B00B2FBF3F258
:109AEC001A4BA3FB02035B09642000FB03F3D31A9C
:109AFC001B013233154AA2FB03235B0903F0F0036D
:109B0C001944FA6813469B0013449A001A447B6864
:109B1C005B689B00B2FBF3F20C4BA3FB02035B09EB
:109B2C00642000FB03F3D31A1B013233074AA2FB58
:109B3C0003235B0903F00F027B681B680A449A60DD
:109B4C0000BF1037BD4680BD003801401F85EB516A
:109B5C0080B485B000AFF860384680E80E00002372
:109B6C0018461437BD4680BC704780B485B000AF32
:109B7C0078607B680022A3F844204FF43F43FB60DD
:109B8C00FB689AB27B68A3F8402000231846143770
:109B9C00BD4680BC704780B485B000AF78604FF490
:109BAC003F43FB607B68B3F840309AB2FB689BB2D2
:109BBC00DB439BB213409AB27B68A3F8402000238E
:109BCC0018461437BD4680BC704780B483B000AFD4
:109BDC0078600B46FB70002318460C37BD4680BCE2
:109BEC00704780B485B000AFF860384680E80E004E
:109BFC00FB680122A3F84020FB680022A3F8402058
:109C0C00FB680022A3F84420FB680022A3F8502034
:109C1C00002318461437BD4680BC704780B49DB0F5
:109C2C0000AF78603960002387F86F307A683B6842
:109C3C001B789B0013441B889BB223F4EC4323F04A
:109C4C007003A7F86C303B68DB78032B1FD801A29C
:109C5C0052F823F0719C00088D9C0008A39C00080E
:109C6C007F9C0008B7F86C3043F40073A7F86C3095
:109C7C0012E0B7F86C3043F4C063A7F86C300BE01B
:109C8C00B7F86C3043F48063A7F86C3004E0012320
:109C9C0087F86F3000E000BF7A683B681B789B0048
:109CAC001A44B7F86C3043F07F4343F47F0343F41A
:109CBC00004343F080039BB213807A683B681B78A7
:109CCC009B0013441B889BB223F4E04323F07003E6
:109CDC009BB23A6812781343A7F866307A683B68EF
:109CEC001B789B001A44B7F8663043F07F4343F46B
:109CFC007F0343F4004343F080039BB213803B6823
:109D0C001B7B002B40F078813B685B78002B00F0CC
:109D1C0084807B68BB617B68B3F850309BB21A4679
:109D2C00BB691344BB613B681B781A01BB691344C4
:109D3C0003F580637B613B68DB885B089BB25B004F
:109D4C009AB27B691A807A683B681B789B00134433
:109D5C001B887B827B8A03F04003002B1BD07A6824
:109D6C003B681B789B0013441B889BB223F4E04395
:109D7C0023F070033B827A683B681B789B001A4483
:109D8C003B8A43F07F4343F47F0343F4004343F0A7
:109D9C00C0039BB213803B68DB78012B20D07A6820
:109DAC003B681B789B0013441B889BB223F4E04355
:109DBC0023F04003BB81BB8983F02003BB817A680D
:109DCC003B681B789B001A44BB8943F07F4343F4E8
:109DDC007F0343F4004343F080039BB21380D5E22E
:109DEC007A683B681B789B0013441B889BB223F456
:109DFC00E04323F04003FB817A683B681B789B00AF
:109E0C001A44FB8943F07F4343F47F0343F400433C
:109E1C0043F080039BB21380B8E27B683B637B68A2
:109E2C00B3F850309BB21A463B6B13443B633B6810
:109E3C001B781A013B6B134403F58163FB623B688F
:109E4C00DB885B089BB25B009AB2FB6A1A807B686A
:109E5C00BB627B68B3F850309BB21A46BB6A1344A2
:109E6C00BB623B681B781A01BB6A134403F20C43B8
:109E7C007B627B6A1B889BB2C3F309039AB27B6A31
:109E8C001A803B681B693E2B1DD93B681B695B091B
:109E9C00BB663B681B6903F01F03002B02D1BB6E32
:109EAC00013BBB667B6A1B889AB2BB6E9BB29B0262
:109EBC009BB213439BB26FEA43436FEA53439AB28C
:109ECC007B6A1A8026E03B681B69002B0AD17B6AEF
:109EDC001B889BB26FEA43436FEA53439AB27B6A87
:109EEC001A8017E03B681B695B08BB663B681B6903
:109EFC0003F00103002B02D0BB6E0133BB667B6AFF
:109F0C001B889AB2BB6E9BB29B029BB213439AB254
:109F1C007B6A1A807A683B681B789B0013441B8809
:109F2C007B847B8C03F48043002B1BD07A683B68CA
:109F3C001B789B0013441B889BB223F4E04323F053
:109F4C0070033B847A683B681B789B001A443B8CFB
:109F5C0043F07F4343F47F0343F4404343F08003D7
:109F6C009BB213803B681B78002B24D17A683B682A
:109F7C001B789B0013441B889BB223F4804323F073
:109F8C007003BB83BB8B83F48053BB83BB8B83F489
:109F9C000053BB837A683B681B789B001A44BB8BCD
:109FAC0043F07F4343F47F0343F4004343F08003C7
:109FBC009BB21380EAE17A683B681B789B001344E0
:109FCC001B889BB223F4804323F07003FB83FB8B31
:109FDC0083F40053FB837A683B681B789B001A441C
:109FEC00FB8B43F07F4343F47F0343F4004343F084
:109FFC0080039BB21380C9E13B68DB78022B1ED136
:10A00C007A683B681B789B0013441B889BB223F433
:10A01C00E04323F07003A7F862307A683B681B7842
:10A02C009B001A44B7F8623043F07F4343F47F033C
:10A03C0043F4014343F080039BB213801DE07A6824
:10A04C003B681B789B0013441B889BB223F4E243B0
:10A05C0023F07003A7F864307A683B681B789B0088
:10A06C001A44B7F8643043F07F4343F47F0343F45E
:10A07C00004343F080039BB213807B68FB657B68D5
:10A08C00B3F850309BB21A46FB6D1344FB653B682A
:10A09C001B781A01FB6D134403F58063BB653B68A9
:10A0AC001B895B089BB25B009AB2BB6D1A807B6804
:10A0BC007B657B68B3F850309BB21A467B6D1344BA
:10A0CC007B653B681B781A017B6D134403F5816338
:10A0DC003B653B685B895B089BB25B009AB23B6D4E
:10A0EC001A803B685B78002B40F093807A683B6861
:10A0FC001B789B0013441B88A7F84030B7F84030FE
:10A10C0003F48043002B1BD07A683B681B789B00C0
:10A11C0013441B889BB223F4E04323F07003FB87AA
:10A12C007A683B681B789B001A44FB8F43F07F4393
:10A13C0043F47F0343F4404343F080039BB213800A
:10A14C007A683B681B789B0013441B88BB87BB8FCA
:10A15C0003F04003002B1BD07A683B681B789B00F4
:10A16C0013441B889BB223F4E04323F070037B87DA
:10A17C007A683B681B789B001A447B8F43F07F43C3
:10A18C0043F47F0343F4004343F0C0039BB21380BA
:10A19C007A683B681B789B0013441B889BB223F4A2
:10A1AC00804323F070033B873B8F83F480533B87C2
:10A1BC003B8F83F400533B877A683B681B789B008A
:10A1CC001A443B8F43F07F4343F47F0343F4004333
:10A1DC0043F080039BB213807A683B681B789B002A
:10A1EC0013441B889BB223F4E04323F04003FB860B
:10A1FC007A683B681B789B001A44FB8E43F07F43C4
:10A20C0043F47F0343F4004343F080039BB2138079
:10A21C00BCE07A683B681B789B0013441B88A7F84A
:10A22C004E30B7F84E3003F48043002B1DD07A68C3
:10A23C003B681B789B0013441B889BB223F4E043C0
:10A24C0023F07003A7F84C307A683B681B789B00AE
:10A25C001A44B7F84C3043F07F4343F47F0343F484
:10A26C00404343F080039BB213807A683B681B78B1
:10A27C009B0013441B88A7F84A30B7F84A3003F008
:10A28C004003002B1DD07A683B681B789B0013445D
:10A29C001B889BB223F4E04323F07003A7F84830EB
:10A2AC007A683B681B789B001A44B7F8483043F037
:10A2BC007F4343F47F0343F4004343F0C0039BB25A
:10A2CC0013803B68DB78012B24D07A683B681B78C1
:10A2DC009B0013441B889BB223F4E04323F0400300
:10A2EC00A7F84430B7F8443083F02003A7F8443083
:10A2FC007A683B681B789B001A44B7F8443043F0EB
:10A30C007F4343F47F0343F4004343F080039BB249
:10A31C0013801DE07A683B681B789B0013441B88F4
:10A32C009BB223F4E04323F04003A7F846307A684D
:10A33C003B681B789B001A44B7F8463043F07F43C8
:10A34C0043F47F0343F4004343F080039BB2138038
:10A35C007A683B681B789B0013441B889BB223F4E0
:10A36C00804323F07003A7F842307A683B681B786F
:10A37C009B001A44B7F8423043F07F4343F47F0309
:10A38C0043F4004343F080039BB2138097F86F3083
:10A39C0018467437BD4680BC704700BF80B48DB082
:10A3AC0000AF786039603B681B7B002B40F08E80DF
:10A3BC003B685B78002B44D07A683B681B789B0029
:10A3CC0013441B88BB81BB8903F04003002B1BD0BB
:10A3DC007A683B681B789B0013441B889BB223F460
:10A3EC00E04323F070037B817A683B681B789B0009
:10A3FC001A447B8943F07F4343F47F0343F40043C7
:10A40C0043F0C0039BB213807A683B681B789B00B7
:10A41C0013441B889BB223F4E04323F040033B819D
:10A42C007A683B681B789B001A443B8943F07F4356
:10A43C0043F47F0343F4004343F080039BB2138047
:10A44C0092E17A683B681B789B0013441B887B82E3
:10A45C007B8A03F48043002B1BD07A683B681B7803
:10A46C009B0013441B889BB223F4E04323F070033E
:10A47C003B827A683B681B789B001A443B8A43F00A
:10A48C007F4343F47F0343F4404343F080039BB288
:10A49C0013807A683B681B789B0013441B889BB223
:10A4AC0023F4804323F07003FB817A683B681B78AC
:10A4BC009B001A44FB8943F07F4343F47F0343F42E
:10A4CC00004343F080039BB213804DE13B685B7803
:10A4DC00002B40F0A5807A683B681B789B001344E6
:10A4EC001B883B843B8C03F48043002B1BD07A6885
:10A4FC003B681B789B0013441B889BB223F4E043FE
:10A50C0023F07003FB837A683B681B789B001A442A
:10A51C00FB8B43F07F4343F47F0343F4404343F00E
:10A52C0080039BB213807A683B681B789B001344B2
:10A53C001B88BB83BB8B03F04003002B1BD07A68BA
:10A54C003B681B789B0013441B889BB223F4E043AD
:10A55C0023F070037B837A683B681B789B001A445A
:10A56C007B8B43F07F4343F47F0343F4004343F07E
:10A57C00C0039BB213807A683B681B789B00134422
:10A58C001B889BB223F4E04323F070033B837A686F
:10A59C003B681B789B001A443B8B43F07F4343F48E
:10A5AC007F0343F4004343F0C0039BB213807A68EB
:10A5BC003B681B789B0013441B889BB223F480439D
:10A5CC0023F07003FB827A683B681B789B001A446B
:10A5DC00FB8A43F07F4343F47F0343F4004343F08F
:10A5EC0080039BB213807A683B681B789B001344F2
:10A5FC001B889BB223F4E04323F04003BB827A68B0
:10A60C003B681B789B001A44BB8A43F07F4343F49E
:10A61C007F0343F4004343F080039BB21380A3E019
:10A62C007A683B681B789B0013441B88FB85FB8D69
:10A63C0003F48043002B1BD07A683B681B789B008B
:10A64C0013441B889BB223F4E04323F07003BB85B7
:10A65C007A683B681B789B001A44BB8D43F07F43A0
:10A66C0043F47F0343F4404343F080039BB21380D5
:10A67C007A683B681B789B0013441B887B857B8D19
:10A68C0003F04003002B1BD07A683B681B789B00BF
:10A69C0013441B889BB223F4E04323F070033B85E7
:10A6AC007A683B681B789B001A443B8D43F07F43D0
:10A6BC0043F47F0343F4004343F0C0039BB2138085
:10A6CC007A683B681B789B0013441B889BB223F46D
:10A6DC00E04323F07003FB847A683B681B789B0093
:10A6EC001A44FB8C43F07F4343F47F0343F4404311
:10A6FC0043F080039BB213807A683B681B789B0005
:10A70C0013441B889BB223F4E04323F04003BB8427
:10A71C007A683B681B789B001A44BB8C43F07F43E0
:10A72C0043F47F0343F4004343F080039BB2138054
:10A73C007A683B681B789B0013441B889BB223F4FC
:10A74C00804323F070037B847A683B681B789B0002
:10A75C001A447B8C43F07F4343F47F0343F4004360
:10A76C0043F080039BB21380002318463437BD4658
:10A77C0080BC704780B5C2B000AF07F58473A3F5F9
:10A78C008273186007F58473A3F58473196007F559
:10A79C008473A3F584731B685B78012B40F0B78638
:10A7AC0007F58473A3F584731B689A6907F58473A2
:10A7BC00A3F584731B681B699A4208D907F5847347
:10A7CC00A3F584731B681B69C7F8043107E007F510
:10A7DC008473A3F584731B689B69C7F8043107F570
:10A7EC008473A3F584731B681B7B002B3AD107F58C
:10A7FC008473A3F584731B68596907F58473A3F5F7
:10A80C0084731B68DA88D7F804319BB207F584701F
:10A81C00A0F58270006801F09CFC07F58473A3F529
:10A82C0082731B683B6107F58473A3F582731B6805
:10A83C00B3F850309BB21A463B6913443B6107F5A1
:10A84C008473A3F584731B681B781A013B6913444A
:10A85C0003F20443FB60D7F804319AB2FB681A8008
:10A86C0000F01FBE07F58473A3F584731B68DB78B7
:10A87C00022B40F0628407F58473A3F584731B6884
:10A88C001A6A07F58473A3F584731B681B699A42D3
:10A89C0040F2DF8307F58473A3F582731A6807F51A
:10A8AC008473A3F584731B681B789B0013441B886B
:10A8BC009BB223F4E04323F07003A7F8563007F55E
:10A8CC008473A3F582731A6807F58473A3F58473F4
:10A8DC001B681B789B001A44B7F8563043F07F4333
:10A8EC0043F47F0343F4014343F080039BB2138092
:10A8FC0007F58473A3F584731B681A6AD7F80431BF
:10A90C00D21A07F58473A3F584731B681A6207F5D2
:10A91C008473A3F582731A6807F58473A3F58473A3
:10A92C001B681B789B0013441B889BB203F04003ED
:10A93C00002B00F0C78107F58473A3F582731B68A5
:10A94C003B6307F58473A3F584731B685B78002B5A
:10A95C0077D107F58473A3F582731B68BB6207F587
:10A96C008473A3F582731B68B3F850309BB21A46FC
:10A97C00BB6A1344BB6207F58473A3F584731B682D
:10A98C001B781A01BB6A134403F20C437B627B6A8B
:10A99C001B889BB2C3F309039AB27B6A1A80D7F85F
:10A9AC0004313E2B21D9D7F804315B09C7F80031AB
:10A9BC00D7F8043103F01F03002B04D1D7F8003172
:10A9CC00013BC7F800317B6A1B889AB2D7F800317B
:10A9DC009BB29B029BB213439BB26FEA43436FEA59
:10A9EC0053439AB27B6A1A8050E0D7F80431002B9B
:10A9FC000AD17B6A1B889BB26FEA43436FEA5343CD
:10AA0C009AB27B6A1A8041E0D7F804315B08C7F828
:10AA1C000031D7F8043103F00103002B04D0D7F830
:10AA2C0000310133C7F800317B6A1B889AB2D7F822
:10AA3C0000319BB29B029BB213439AB27B6A1A8081
:10AA4C0024E007F58473A3F584731B685B78012BF2
:10AA5C001CD107F58473A3F582731B68B3F85030CF
:10AA6C009BB21A463B6B13443B6307F58473A3F507
:10AA7C0084731B681B781A013B6B134403F20C4361
:10AA8C00FB62D7F804319AB2FB6A1A8007F584731B
:10AA9C00A3F584731B685B89A7F8763007F584737C
:10AAAC00A3F584731B685969D7F804319BB2B7F8C6
:10AABC00762007F58470A0F58270006801F049FBE0
:10AACC0007F58473A3F584731B685A69D7F80431AE
:10AADC001A4407F58473A3F584731B685A6107F550
:10AAEC008473A3F584731B681A6A07F58473A3F542
:10AAFC0084731B681B699A420FD907F58473A3F5FD
:10AB0C0084731B681A6AD7F80431D21A07F5847358
:10AB1C00A3F584731B681A620EE007F58473A3F522
:10AB2C0084731B681B6AC7F8043107F58473A3F59B
:10AB3C0084731B6800221A6207F58473A3F584736F
:10AB4C001B685B78002B77D107F58473A3F58273B0
:10AB5C001B68BB6107F58473A3F582731B68B3F89C
:10AB6C0050309BB21A46BB691344BB6107F5847322
:10AB7C00A3F584731B681B781A01BB69134403F299
:10AB8C0004437B617B691B889BB2C3F309039AB2B4
:10AB9C007B691A80D7F804313E2B21D9D7F80431C0
:10ABAC005B09C7F8FC30D7F8043103F01F03002B06
:10ABBC0004D1D7F8FC30013BC7F8FC307B691B880B
:10ABCC009AB2D7F8FC309BB29B029BB213439BB258
:10ABDC006FEA43436FEA53439AB27B691A8056E09B
:10ABEC00D7F80431002B0AD17B691B889BB26FEA22
:10ABFC0043436FEA53439AB27B691A8047E0D7F814
:10AC0C0004315B08C7F8FC30D7F8043103F00103BA
:10AC1C00002B04D0D7F8FC300133C7F8FC307B692B
:10AC2C001B889AB2D7F8FC309BB29B029BB21343A1
:10AC3C009AB27B691A802AE007F58473A3F58473B2
:10AC4C001B685B78012B22D107F58473A3F5827303
:10AC5C001B683B6207F58473A3F582731B68B3F81A
:10AC6C0050309BB21A463B6A13443B6207F584731F
:10AC7C00A3F584731B681B781A013B6A134403F217
:10AC8C000443FB61D7F804319AB2FB691A8007F5CB
:10AC9C008473A3F584731B681B89A7F8763007F5BA
:10ACAC008473A3F584731B685969D7F804319BB27C
:10ACBC00B7F8762007F58470A0F58270006801F073
:10ACCC0048FAEEE307F58473A3F584731B685B788D
:10ACDC00002B77D107F58473A3F582731B68BB64D3
:10ACEC0007F58473A3F582731B68B3F850309BB2DD
:10ACFC001A46BB6C1344BB6407F58473A3F58473C9
:10AD0C001B681B781A01BB6C134403F204437B646D
:10AD1C007B6C1B889BB2C3F309039AB27B6C1A80C1
:10AD2C00D7F804313E2B21D9D7F804315B09C7F889
:10AD3C00F830D7F8043103F01F03002B04D1D7F8F7
:10AD4C00F830013BC7F8F8307B6C1B889AB2D7F807
:10AD5C00F8309BB29B029BB213439BB26FEA434306
:10AD6C006FEA53439AB27B6C1A8056E0D7F80431E1
:10AD7C00002B0AD17B6C1B889BB26FEA43436FEAB2
:10AD8C0053439AB27B6C1A8047E0D7F804315B08C6
:10AD9C00C7F8F830D7F8043103F00103002B04D0C6
:10ADAC00D7F8F8300133C7F8F8307B6C1B889AB2AF
:10ADBC00D7F8F8309BB29B029BB213439AB27B6CD0
:10ADCC001A802AE007F58473A3F584731B685B78FB
:10ADDC00012B22D107F58473A3F582731B683B65A5
:10ADEC0007F58473A3F582731B68B3F850309BB2DC
:10ADFC001A463B6D13443B6507F58473A3F58473C6
:10AE0C001B681B781A013B6D134403F20443FB646B
:10AE1C00D7F804319AB2FB6C1A8007F58473A3F54A
:10AE2C0084731B681B89A7F8763007F58473A3F528
:10AE3C0084731B685969D7F804319BB2B7F8762034
:10AE4C0007F58470A0F58270006801F082F907F5AF
:10AE5C008473A3F584731B685A69D7F804311A44B8
:10AE6C0007F58473A3F584731B685A6107F5847323
:10AE7C00A3F584731B681A6A07F58473A3F58473AE
:10AE8C001B681B699A420FD907F58473A3F5847369
:10AE9C001B681A6AD7F80431D21A07F58473A3F524
:10AEAC0084731B681A620EE007F58473A3F5847330
:10AEBC001B681B6AC7F8043107F58473A3F5847308
:10AECC001B6800221A6207F58473A3F582731B6852
:10AEDC003B6407F58473A3F584731B685B78002BC4
:10AEEC0077D107F58473A3F582731B68BB6307F5F1
:10AEFC008473A3F582731B68B3F850309BB21A4667
:10AF0C00BB6B1344BB6307F58473A3F584731B6895
:10AF1C001B781A01BB6B134403F20C437B637B6BF2
:10AF2C001B889BB2C3F309039AB27B6B1A80D7F8C8
:10AF3C0004313E2B21D9D7F804315B09C7F8F43022
:10AF4C00D7F8043103F01F03002B04D1D7F8F430E9
:10AF5C00013BC7F8F4307B6B1B889AB2D7F8F430FE
:10AF6C009BB29B029BB213439BB26FEA43436FEAC3
:10AF7C0053439AB27B6B1A8050E0D7F80431002B04
:10AF8C000AD17B6B1B889BB26FEA43436FEA534336
:10AF9C009AB27B6B1A8041E0D7F804315B08C7F892
:10AFAC00F430D7F8043103F00103002B04D0D7F8A8
:10AFBC00F4300133C7F8F4307B6B1B889AB2D7F8A6
:10AFCC00F4309BB29B029BB213439AB27B6B1A80F8
:10AFDC0024E007F58473A3F584731B685B78012B5D
:10AFEC001CD107F58473A3F582731B68B3F850303A
:10AFFC009BB21A463B6C13443B6407F58473A3F570
:10B00C0084731B681B781A013B6C134403F20C43CA
:10B01C00FB63D7F804319AB2FB6B1A8007F5847383
:10B02C00A3F584731B685B89A7F8763007F58473E6
:10B03C00A3F584731B685969D7F804319BB2B7F830
:10B04C00762007F58470A0F58270006801F081F815
:10B05C0027E207F58473A3F584731B681B6AC7F892
:10B06C00043107F58473A3F582731A6807F58473AA
:10B07C00A3F584731B681B789B0013441B889BB23D
:10B08C0023F4E24323F07003A7F8623007F58473CE
:10B09C00A3F582731A6807F58473A3F584731B6890
:10B0AC001B789B001A44B7F8623043F07F4343F49B
:10B0BC007F0343F4004343F080039BB2138007F5F6
:10B0CC008473A3F582731B68FB6507F58473A3F582
:10B0DC0082731B68B3F850309BB21A46FB6D134455
:10B0EC00FB6507F58473A3F584731B681B781A0141
:10B0FC00FB6D134403F20443BB65D7F804319AB2D9
:10B10C00BB6D1A8007F58473A3F584731B681B89C8
:10B11C00A7F8763007F58473A3F584731B68596917
:10B12C00D7F804319BB2B7F8762007F58470A0F5F8
:10B13C008270006801F00DF8B3E107F58473A3F594
:10B14C0084731B681A6AD7F80431D21A07F5847312
:10B15C00A3F584731B681A6207F58473A3F58273D5
:10B16C001A6807F58473A3F584731B681B789B001E
:10B17C0013441B889BB203F04003002B00F0C680E5
:10B18C0007F58473A3F582731B683B6707F584731B
:10B19C00A3F584731B685B78002B77D107F5847358
:10B1AC00A3F582731B68BB6607F58473A3F58273E2
:10B1BC001B68B3F850309BB21A46BB6E1344BB6687
:10B1CC0007F58473A3F584731B681B781A01BB6E97
:10B1DC00134403F20C437B667B6E1B889BB2C3F358
:10B1EC0009039AB27B6E1A80D7F804313E2B21D911
:10B1FC00D7F804315B09C7F8F030D7F8043103F005
:10B20C001F03002B04D1D7F8F030013BC7F8F03006
:10B21C007B6E1B889AB2D7F8F0309BB29B029BB224
:10B22C0013439BB26FEA43436FEA53439AB27B6E6C
:10B23C001A8050E0D7F80431002B0AD17B6E1B88A2
:10B24C009BB26FEA43436FEA53439AB27B6E1A8008
:10B25C0041E0D7F804315B08C7F8F030D7F8043177
:10B26C0003F00103002B04D0D7F8F0300133C7F8FA
:10B27C00F0307B6E1B889AB2D7F8F0309BB29B02F1
:10B28C009BB213439AB27B6E1A8024E007F5847349
:10B29C00A3F584731B685B78012B1CD107F58473B1
:10B2AC00A3F582731B68B3F850309BB21A463B6F00
:10B2BC0013443B6707F58473A3F584731B681B78F1
:10B2CC001A013B6F134403F20C43FB66D7F80431AD
:10B2DC009AB2FB6E1A8007F58473A3F584731B680E
:10B2EC005B89A7F8763007F58473A3F584731B6824
:10B2FC005969D7F804319BB2B7F8762007F58470FA
:10B30C00A0F58270006800F024FFCAE007F5847392
:10B31C00A3F584731B685B78002B77D107F58473D6
:10B32C00A3F582731B68FB6707F58473A3F582731F
:10B33C001B68B3F850309BB21A46FB6F1344FB6783
:10B34C0007F58473A3F584731B681B781A01FB6FD4
:10B35C00134403F20443BB67BB6F1B889BB2C3F35C
:10B36C0009039AB2BB6F1A80D7F804313E2B21D94E
:10B37C00D7F804315B09C7F8EC30D7F8043103F087
:10B38C001F03002B04D1D7F8EC30013BC7F8EC308D
:10B39C00BB6F1B889AB2D7F8EC309BB29B029BB266
:10B3AC0013439BB26FEA43436FEA53439AB2BB6FAA
:10B3BC001A805CE0D7F80431002B0AD1BB6F1B88D4
:10B3CC009BB26FEA43436FEA53439AB2BB6F1A8046
:10B3DC004DE0D7F804315B08C7F8EC30D7F80431EE
:10B3EC0003F00103002B04D0D7F8EC300133C7F87D
:10B3FC00EC30BB6F1B889AB2D7F8EC309BB29B0237
:10B40C009BB213439AB2BB6F1A8030E007F584737A
:10B41C00A3F584731B685B78012B28D107F5847323
:10B42C00A3F582731B68C7F8843007F58473A3F502
:10B43C0082731B68B3F850309BB21A46D7F884302D
:10B44C001344C7F8843007F58473A3F584731B6821
:10B45C001B781A01D7F88430134403F20443C7F85D
:10B46C008030D7F804319AB2D7F880301A8007F5BB
:10B47C008473A3F584731B681B89A7F8763007F5D2
:10B48C008473A3F584731B685969D7F804319BB294
:10B49C00B7F8762007F58470A0F58270006800F08C
:10B4AC0058FE07F58473A3F582731A6807F5847345
:10B4BC00A3F584731B681B789B0013441B889BB2F9
:10B4CC0023F4E04323F040037B817B8983F010035A
:10B4DC007B817B8983F020037B8107F58473A3F543
:10B4EC0082731A6807F58473A3F584731B681B7841
:10B4FC009B001A447B8943F07F4343F47F0343F45E
:10B50C00004343F080039BB2138000F0DEBC07F5D0
:10B51C008473A3F584731B681B7B002B40F0BB80EA
:10B52C0007F58473A3F584731B689A6907F5847314
:10B53C00A3F584731B681B699A4217D907F58473AA
:10B54C00A3F584731B681B69C7F8043107F5847372
:10B55C00A3F584731B689A69D7F80431D21A07F5DE
:10B56C008473A3F584731B689A610EE007F58473EA
:10B57C00A3F584731B689B69C7F8043107F58473C2
:10B58C00A3F584731B6800229A6107F58473A3F5F5
:10B59C0082731B68C7F8903007F58473A3F5827328
:10B5AC001B68B3F850309BB21A46D7F8903013444E
:10B5BC00C7F8903007F58473A3F584731B681B7868
:10B5CC001A01D7F89030134403F20C43C7F88C30AF
:10B5DC00D7F88C301B889BB2C3F309039AB2D7F807
:10B5EC008C301A80D7F804313E2B24D9D7F804318B
:10B5FC005B09C7F8E830D7F8043103F01F03002BC0
:10B60C0004D1D7F8E830013BC7F8E830D7F88C30D4
:10B61C001B889AB2D7F8E8309BB29B029BB21343BB
:10B62C009BB26FEA43436FEA53439AB2D7F88C301C
:10B63C001A8000F010BCD7F80431002B0CD1D7F8CD
:10B64C008C301B889BB26FEA43436FEA53439AB228
:10B65C00D7F88C301A80FEE3D7F804315B08C7F8B2
:10B66C00E830D7F8043103F00103002B04D0D7F8ED
:10B67C00E8300133C7F8E830D7F88C301B889AB221
:10B68C00D7F8E8309BB29B029BB213439AB2D7F81F
:10B69C008C301A80DFE307F58473A3F584731B6881
:10B6AC00DB78022B40F0188207F58473A3F58473C2
:10B6BC001B685B78002B40F09D8007F58473A3F525
:10B6CC0082731B68C7F8AC3007F58473A3F58273DB
:10B6DC001B68B3F850309BB21A46D7F8AC30134401
:10B6EC00C7F8AC3007F58473A3F584731B681B781B
:10B6FC001A01D7F8AC30134403F20443C7F8A8304E
:10B70C00D7F8A8301B889BB2C3F309039AB2D7F8B9
:10B71C00A8301A8007F58473A3F584731B681B6922
:10B72C003E2B2BD907F58473A3F584731B681B6917
:10B73C005B09C7F8E43007F58473A3F584731B68C1
:10B74C001B6903F01F03002B04D1D7F8E430013B35
:10B75C00C7F8E430D7F8A8301B889AB2D7F8E43091
:10B76C009BB29B029BB213439BB26FEA43436FEABB
:10B77C0053439AB2D7F8A8301A8070E007F5847357
:10B78C00A3F584731B681B69002B0CD1D7F8A83068
:10B79C001B889BB26FEA43436FEA53439AB2D7F8C4
:10B7AC00A8301A805BE007F58473A3F584731B68DB
:10B7BC001B695B08C7F8E43007F58473A3F5847341
:10B7CC001B681B6903F00103002B04D0D7F8E4308D
:10B7DC000133C7F8E430D7F8A8301B889AB2D7F8F1
:10B7EC00E4309BB29B029BB213439AB2D7F8A830B9
:10B7FC001A8034E007F58473A3F584731B685B78B7
:10B80C00012B2CD107F58473A3F582731B68C7F841
:10B81C00B43007F58473A3F582731B68B3F850300A
:10B82C009BB21A46D7F8B4301344C7F8B43007F5B6
:10B83C008473A3F584731B681B781A01D7F8B43092
:10B84C00134403F20443C7F8B03007F58473A3F52F
:10B85C0084731B681B699AB2D7F8B0301A8007F54D
:10B86C008473A3F582731B68C7F8A43007F584733F
:10B87C00A3F584731B685B78002B40F09D8007F563
:10B88C008473A3F582731B68C7F89C3007F5847327
:10B89C00A3F582731B68B3F850309BB21A46D7F8E5
:10B8AC009C301344C7F89C3007F58473A3F584735C
:10B8BC001B681B781A01D7F89C30134403F20C4315
:10B8CC00C7F89830D7F898301B889BB2C3F309039C
:10B8DC009AB2D7F898301A8007F58473A3F584735D
:10B8EC001B681B693E2B2BD907F58473A3F5847356
:10B8FC001B681B695B09C7F8E03007F58473A3F577
:10B90C0084731B681B6903F01F03002B04D1D7F849
:10B91C00E030013BC7F8E030D7F898301B889AB27A
:10B92C00D7F8E0309BB29B029BB213439BB26FEAF9
:10B93C0043436FEA53439AB2D7F898301A8069E0C0
:10B94C0007F58473A3F584731B681B69002B0CD15A
:10B95C00D7F898301B889BB26FEA43436FEA534386
:10B96C009AB2D7F898301A8054E007F58473A3F58F
:10B97C0084731B681B695B08C7F8E03007F5847398
:10B98C00A3F584731B681B6903F00103002B04D01F
:10B99C00D7F8E0300133C7F8E030D7F898301B887F
:10B9AC009AB2D7F8E0309BB29B029BB213439AB287
:10B9BC00D7F898301A802DE007F58473A3F58473BB
:10B9CC001B685B78012B25D107F58473A3F5827373
:10B9DC001B68B3F850309BB21A46D7F8A430134406
:10B9EC00C7F8A43007F58473A3F584731B681B7820
:10B9FC001A01D7F8A430134403F20C43C7F8A03053
:10BA0C0007F58473A3F584731B681B699AB2D7F886
:10BA1C00A0301A8007F58473A3F584731B68DB6967
:10BA2C00002B00F0188207F58473A3F582731A6853
:10BA3C0007F58473A3F584731B681B789B00134470
:10BA4C001B88A7F89630B7F8963003F48043002B88
:10BA5C0005D0B7F8963003F04003002B0DD1B7F8A2
:10BA6C00963003F48043002B40F0F581B7F8963004
:10BA7C0003F04003002B40F0EE8107F58473A3F52F
:10BA8C0082731A6807F58473A3F584731B681B789B
:10BA9C009B0013441B889BB223F4E04323F07003F8
:10BAAC00A7F8943007F58473A3F582731A6807F529
:10BABC008473A3F584731B681B789B001A44B7F836
:10BACC00943043F07F4343F47F0343F4004343F04B
:10BADC00C0039BB21380BEE107F58473A3F5847396
:10BAEC001B68DB78012B40F0B48107F58473A3F558
:10BAFC0084731B689A6907F58473A3F584731B68B8
:10BB0C001B699A4217D907F58473A3F584731B68D4
:10BB1C001B69C7F8043107F58473A3F584731B689C
:10BB2C009A69D7F80431D21A07F58473A3F5847394
:10BB3C001B689A610EE007F58473A3F584731B6888
:10BB4C009B69C7F8043107F58473A3F584731B68EC
:10BB5C0000229A6107F58473A3F584731B685B78E4
:10BB6C00002B40F0858007F58473A3F582731B6866
:10BB7C00C7F8CC3007F58473A3F582731B68B3F850
:10BB8C0050309BB21A46D7F8CC301344C7F8CC309F
:10BB9C0007F58473A3F584731B681B781A01D7F817
:10BBAC00CC30134403F20443C7F8C830D7F8C8307C
:10BBBC001B889BB2C3F309039AB2D7F8C8301A801A
:10BBCC00D7F804313E2B23D9D7F804315B09C7F8D9
:10BBDC00DC30D7F8043103F01F03002B04D1D7F865
:10BBEC00DC30013BC7F8DC30D7F8C8301B889AB280
:10BBFC00D7F8DC309BB29B029BB213439BB26FEA2B
:10BC0C0043436FEA53439AB2D7F8C8301A8060E0C6
:10BC1C00D7F80431002B0CD1D7F8C8301B889BB255
:10BC2C006FEA43436FEA53439AB2D7F8C8301A808D
:10BC3C004FE0D7F804315B08C7F8DC30D7F8043193
:10BC4C0003F00103002B04D0D7F8DC300133C7F824
:10BC5C00DC30D7F8C8301B889AB2D7F8DC309BB2EE
:10BC6C009B029BB213439AB2D7F8C8301A8030E0CB
:10BC7C0007F58473A3F584731B685B78012B28D1BB
:10BC8C0007F58473A3F582731B68C7F8D43007F5E6
:10BC9C008473A3F582731B68B3F850309BB21A46B9
:10BCAC00D7F8D4301344C7F8D43007F58473A3F510
:10BCBC0084731B681B781A01D7F8D430134403F231
:10BCCC000443C7F8D030D7F804319AB2D7F8D03043
:10BCDC001A8007F58473A3F582731B68C7F8C43008
:10BCEC0007F58473A3F584731B685B78002B40F015
:10BCFC00858007F58473A3F582731B68C7F8BC3085
:10BD0C0007F58473A3F582731B68B3F850309BB2AC
:10BD1C001A46D7F8BC301344C7F8BC3007F5847307
:10BD2C00A3F584731B681B781A01D7F8BC30134435
:10BD3C0003F20C43C7F8B830D7F8B8301B889BB265
:10BD4C00C3F309039AB2D7F8B8301A80D7F8043184
:10BD5C003E2B23D9D7F804315B09C7F8D830D7F874
:10BD6C00043103F01F03002B04D1D7F8D830013B6A
:10BD7C00C7F8D830D7F8B8301B889AB2D7F8D83073
:10BD8C009BB29B029BB213439BB26FEA43436FEA95
:10BD9C0053439AB2D7F8B8301A805CE0D7F8043124
:10BDAC00002B0CD1D7F8B8301B889BB26FEA4343F9
:10BDBC006FEA53439AB2D7F8B8301A804BE0D7F8F1
:10BDCC0004315B08C7F8D830D7F8043103F001030D
:10BDDC00002B04D0D7F8D8300133C7F8D830D7F8B7
:10BDEC00B8301B889AB2D7F8D8309BB29B029BB262
:10BDFC0013439AB2D7F8B8301A802CE007F5847345
:10BE0C00A3F584731B685B78012B24D107F584732D
:10BE1C00A3F582731B68B3F850309BB21A46D7F85F
:10BE2C00C4301344C7F8C43007F58473A3F5847386
:10BE3C001B681B781A01D7F8C430134403F20C4367
:10BE4C00C7F8C030D7F804319AB2D7F8C0301A808E
:10BE5C0001E001233AE007F58473A3F582731A68B5
:10BE6C0007F58473A3F584731B681B789B0013443C
:10BE7C001B889BB223F4804323F07003A7F88A300D
:10BE8C00B7F88A3083F48053A7F88A30B7F88A3031
:10BE9C0083F40053A7F88A3007F58473A3F58273F3
:10BEAC001A6807F58473A3F584731B681B789B00D1
:10BEBC001A44B7F88A3043F07F4343F47F0343F4CA
:10BECC00004343F080039BB213800023184607F510
:10BEDC008477BD4680BD80B485B000AF7860396092
:10BEEC003B685B78002B20D07A683B681B789B0002
:10BEFC0013441B889BB223F4E04323F04003BB8123
:10BF0C00BB8983F01003BB817A683B681B789B006C
:10BF1C001A44BB8943F07F4343F47F0343F400434B
:10BF2C0043F080039BB213801FE07A683B681B7858
:10BF3C009B0013441B889BB223F4804323F07003B3
:10BF4C00FB81FB8983F48053FB817A683B681B7807
:10BF5C009B001A44FB8943F07F4343F47F0343F473
:10BF6C00004343F080039BB2138000231846143720
:10BF7C00BD4680BC704780B487B000AF7860396034
:10BF8C003B681B7B002B40F09D803B685B78002B53
:10BF9C004CD07A683B681B789B0013441B883B820F
:10BFAC003B8A03F04003002B1BD07A683B681B785C
:10BFBC009B0013441B889BB223F4E04323F07003D3
:10BFCC00FB817A683B681B789B001A44FB8943F021
:10BFDC007F4343F47F0343F4004343F0C0039BB21D
:10BFEC0013803B68DB78012B6CD07A683B681B783C
:10BFFC009B0013441B889BB223F4E04323F04003C3
:10C00C00BB81BB8983F02003BB817A683B681B78BA
:10C01C009B001A44BB8943F07F4343F47F0343F4F2
:10C02C00004343F080039BB213804BE07A683B687B
:10C03C001B789B0013441B88FB82FB8A03F4804310
:10C04C00002B1BD07A683B681B789B0013441B8821
:10C05C009BB223F4E04323F07003BB827A683B6805
:10C06C001B789B001A44BB8A43F07F4343F47F0345
:10C07C0043F4404343F080039BB213807A683B68DF
:10C08C001B789B0013441B889BB223F4804323F042
:10C09C0070037B827B8A83F480537B827B8A83F45C
:10C0AC0000537B827A683B681B789B001A447B8A1E
:10C0BC0043F07F4343F47F0343F4004343F0800396
:10C0CC009BB21380002318461C37BD4680BC7047BA
:10C0DC0080B483B000AF78600B46FB70FB78002B0C
:10C0EC0003D17B688022A3F84C20002318460C3720
:10C0FC00BD4680BC704780B483B000AF786000232D
:10C10C0018460C37BD4680BC704780B483B000AF76
:10C11C007860002318460C37BD4680BC704780B44D
:10C12C0085B000AF78607B68B3F844309BB2FB609D
:10C13C00FB6818461437BD4680BC704780B483B08A
:10C14C0000AF78603960002318460C37BD4680BCC0
:10C15C00704780B48BB000AFF860B96011461A46D6
:10C16C000B46FB801346BB80BB8801335B08BB616D
:10C17C00FB687B61BB68FB61FB885A007B691344DD
:10C18C0003F580633B62BB697B621FE0FB691B7834
:10C19C007B82FB6901331B781BB21B021AB2B7F905
:10C1AC00123013431BB27B823B6A7A8A1A803B6A39
:10C1BC0002333B623B6A02333B62FB690133FB6136
:10C1CC00FB690133FB617B6A013B7B627B6A002B61
:10C1DC00DCD100BF00BF2C37BD4680BC704780B49B
:10C1EC008BB000AFF860B96011461A460B46FB8065
:10C1FC001346BB80BB885B089BB2BB61FB687B6151
:10C20C00BB68FB61FB885A007B69134403F58063B0
:10C21C003B62BB697B621BE03B6A1B889BB23B6148
:10C22C003B6A02333B623B69DAB2FB691A70FB6909
:10C23C000133FB613B691B0ADAB2FB691A70FB69BB
:10C24C000133FB613B6A02333B627B6A013B7B62DD
:10C25C007B6A002BE0D1BB8803F001039BB2002B5F
:10C26C0007D03B6A1B889BB23B613B69DAB2FB6926
:10C27C001A7000BF2C37BD4680BC704780B584B0A7
:10C28C0000AF78600B46FB700023FB737B681B7C54
:10C29C00002B15D14FF4007302228121786801F034
:10C2AC0000FF7B680122DA624FF400730222012145
:10C2BC00786801F0F6FE7B680122C3F86C2112E06D
:10C2CC00402302228121786801F0EBFE7B68012279
:10C2DC00DA62402302220121786801F0E2FE7B68D9
:10C2EC000122C3F86C21082303228221786801F013
:10C2FC00D8FE7B6801221A644FF4077001F0F8FF36
:10C30C0002467B68C3F8B8227B68D3F8B832002B9E
:10C31C0002D10123FB7326E07B68D3F8B832BB60F3
:10C32C007B68D3F8BC321B689847BB680022C3F803
:10C33C001422BB680022C3F818227B681B7C002BDC
:10C34C0009D1BB68D3F804224FF40073012178683B
:10C35C0001F097FF07E0BB68D3F8042240230121CA
:10C36C00786801F08EFFFB7B18461037BD4680BD08
:10C37C0080B584B000AF78600B46FB700023FB7374
:10C38C008121786801F0B3FE7B680022DA6201211A
:10C39C00786801F0ACFE7B680022C3F86C21822126
:10C3AC00786801F0A4FE7B6800221A647B68D3F8DD
:10C3BC00B832002B0ED07B68D3F8BC325B68984740
:10C3CC007B68D3F8B832184601F09EFF7B680022D8
:10C3DC00C3F8B822FB7B18461037BD4680BD80B52C
:10C3EC0086B000AF786039607B68D3F8B8323B61B7
:10C3FC000023FB730023BB810023FB753B681B7878
:10C40C0003F06003002B39D0202B7FD13B68DB88F5
:10C41C00002B29D03B681B785BB2002B11DA7B68B0
:10C42C00D3F8BC329B683A68507839693A68D2883C
:10C43C00984739693B68DB881A46786801F006FA38
:10C44C006BE03B685A783B6983F800223B68DB88D9
:10C45C00DAB23B6983F8012239693B68DB881A46FA
:10C46C00786801F021FA58E07B68D3F8BC329B68FD
:10C47C003A6850780022396898474EE03B685B7800
:10C48C000B2B2ED00B2B38DC002B02D00A2B14D00C
:10C49C0033E07B6893F89C32032B07D107F10C0334
:10C4AC0002221946786801F0D1F92EE039687868D3
:10C4BC0001F062F90223FB7527E07B6893F89C324C
:10C4CC00032B07D107F10F0301221946786801F0FD
:10C4DC00BDF91AE03968786801F04EF90223FB7552
:10C4EC0013E07B6893F89C32032B0DD03968786885
:10C4FC0001F042F90223FB7506E03968786801F017
:10C50C003BF90223FB7500E000BF06E03968786850
:10C51C0001F032F90223FB7500BFFB7D184618377A
:10C52C00BD4680BD80B584B000AF78600B46FB7013
:10C53C007B68D3F8B832FB607B68D3F8C032BB6041
:10C54C007B68D3F8B832002B3AD0FA787968134666
:10C55C009B0013449B000B441C331B68002B29D0FD
:10C56C00FA78796813469B0013449B000B441C33E8
:10C57C001A68F978B8680B469B000B44DB0003443F
:10C58C0020331B68B2FBF3F101FB03F3D31A002B2E
:10C59C0010D1FA78796813469B0013449B000B4426
:10C5AC001C3300221A60F97800230022786801F00D
:10C5BC0045FE03E0FB680022C3F81422002300E0D0
:10C5CC00022318461037BD4680BD80B584B000AF3D
:10C5DC0078600B46FB707B68D3F8B832FB60FB7855
:10C5EC001946786801F070FE0246FB68C3F80C220D
:10C5FC007B68D3F8B832002B0DD07B68D3F8BC32F3
:10C60C00DB68FA68D2F80402FA6802F50372114684
:10C61C009847002300E0022318461037BD4680BD22
:10C62C0080B584B000AF78607B68D3F8B832FB601B
:10C63C007B68D3F8BC32002B14D0FB6893F8003223
:10C64C00FF2B0FD07B68D3F8BC329B68FA6892F84A
:10C65C000002F968FA6892F801229847FB68FF22F9
:10C66C0083F80022002318461037BD4680BD000019
:10C67C0080B483B000AF78607B6843221A80034B90
:10C68C0018460C37BD4680BC704700BFA400002084
:10C69C0080B483B000AF78607B6843221A80034B70
:10C6AC0018460C37BD4680BC704700BF60000020A8
:10C6BC0080B483B000AF78607B6843221A80034B50
:10C6CC0018460C37BD4680BC704700BFE800002000
:10C6DC0080B483B000AF78607B680A221A80034B69
:10C6EC0018460C37BD4680BC704700BF1C000020AC
:10C6FC0080B485B000AF786039600223FB733B686F
:10C70C00002B05D07B683A68C3F8BC220023FB736E
:10C71C00FB7B18461437BD4680BC704780B487B08D
:10C72C0000AFF860B9601346FB80FB68D3F8B832F1
:10C73C007B617B69BA68C3F80822FA887B69C3F805
:10C74C001022002318461C37BD4680BC704780B4AD
:10C75C0085B000AF786039607B68D3F8B832FB6085
:10C76C00FB683A68C3F80422002318461437BD4608
:10C77C0080BC704780B584B000AF78607B68D3F81C
:10C78C00B832FB607B68D3F8B832002B1CD0FB6846
:10C79C00D3F81432002B15D1FB680122C3F81422F4
:10C7AC00FB68D3F810227B681A63FB68D3F8082265
:10C7BC00FB68D3F810329BB28121786801F03EFD02
:10C7CC00002302E0012300E0022318461037BD4687
:10C7DC0080BD80B584B000AF78607B68D3F8B83288
:10C7EC00FB607B68D3F8B832002B17D07B681B7CBE
:10C7FC00002B09D1FB68D3F804224FF400730121FC
:10C80C00786801F03EFD07E0FB68D3F80422402372
:10C81C000121786801F035FD002300E00223184661
:10C82C001037BD4680BD80B584B000AFF860B960EC
:10C83C001346FB71FB68002B01D102231AE0FB6845
:10C84C00D3F8B432002B03D0FB680022C3F8B42217
:10C85C00BB68002B03D0FB68BA68C3F8B022FB6836
:10C86C00012283F89C22FB68FA791A70F86801F0AF
:10C87C00A3FB002318461037BD4680BD80B485B09D
:10C88C0000AF786039600023FB733B68002B06D047
:10C89C007B683A68C3F8B4220023FB7301E00223DF
:10C8AC00FB73FB7B18461437BD4680BC704780B5C4
:10C8BC0082B000AF7860786801F0D8FB002318468E
:10C8CC000837BD4680BD80B483B000AF78600023CC
:10C8DC0018460C37BD4680BC704780B584B000AF9D
:10C8EC0078600B46FB700223FB737B68D3F8B43281
:10C8FC00002B0CD07B68D3F8B4321B68FA78114645
:10C90C00786898470346002B01D10023FB73FB7B0F
:10C91C0018461037BD4680BD80B582B000AF786038
:10C92C000B46FB707B68D3F8B4325B68FA7811461F
:10C93C0078689847002318460837BD4680BD80B5F7
:10C94C0082B000AF786039607B6803F52A73396870
:10C95C00184600F0D8FE7B680122C3F894227B684D
:10C96C00B3F8AE321A467B68C3F898227B6893F80A
:10C97C00A83203F01F03022B16D0022B1CD8002B5D
:10C98C0002D0012B08D017E07B6803F52A731946F7
:10C99C00786800F0CBF91AE07B6803F52A73194626
:10C9AC00786800F02DFA12E07B6803F52A731946BB
:10C9BC00786800F06DFA0AE07B6893F8A83223F0EF
:10C9CC007F03DBB21946786801F0B0FB00BF00238F
:10C9DC0018460837BD4680BD80B586B000AFF860FC
:10C9EC000B467A60FB72FB7A002B4BD1FB6803F58C
:10C9FC00AA737B61FB68D3F89432032B34D17B6927
:10CA0C00DA687B691B699A4219D97B69DA687B6998
:10CA1C001B69D21A7B69DA607B69DA687B691B69EE
:10CA2C009A4203D27B69DB689BB202E07B691B698B
:10CA3C009BB21A467968F86800F054FF38E0FB683E
:10CA4C00D3F8B4321B69002B0AD0FB6893F89C32E4
:10CA5C00032B05D1FB68D3F8B4321B69F8689847EF
:10CA6C00F86800F051FF23E0FB68D3F89432052BF3
:10CA7C001ED1FB680022C3F894220021F86801F053
:10CA8C0055FB15E0FB68D3F8B4329B69002B0DD035
:10CA9C00FB6893F89C32032B08D1FB68D3F8B432B3
:10CAAC009B69FA7A1146F868984701E0022300E086
:10CABC00002318461837BD4680BD80B586B000AF40
:10CACC00F8600B467A60FB72FB7A002B7FD1FB6817
:10CADC0014337B61FB68D3F89432022B5CD17B69F5
:10CAEC00DA687B691B699A4215D97B69DA687B69BC
:10CAFC001B69D21A7B69DA607B69DB689BB21A46C8
:10CB0C007968F86800F0BEFE002300220021F86866
:10CB1C0001F0B7FB4EE07B699B687A691269B3FB45
:10CB2C00F2F101FB02F29B1A002B1CD17B699A6873
:10CB3C007B691B699A4216D37B699A68FB68D3F8A8
:10CB4C0098329A420FD200220021F86800F09AFE27
:10CB5C00FB680022C3F89822002300220021F86809
:10CB6C0001F08FFB26E0FB68D3F8B432DB68002BB6
:10CB7C000AD0FB6893F89C32032B05D1FB68D3F8E1
:10CB8C00B432DB68F86898478021F86801F0CEFA77
:10CB9C00F86800F0CCFE0DE0FB68D3F89432042B5F
:10CBAC0004D0FB68D3F89432002B03D18021F868B1
:10CBBC0001F0BCFAFB6893F8A032012B1DD1F86888
:10CBCC00FFF781FEFB68002283F8A02215E0FB68CA
:10CBDC00D3F8B4325B69002B0DD0FB6893F89C3210
:10CBEC00032B08D1FB68D3F8B4325B69FA7A11468F
:10CBFC00F868984701E0022300E000231846183734
:10CC0C00BD4680BD80B582B000AF78604023002265
:10CC1C000021786801F045FA7B680122C3F858219D
:10CC2C007B684022C3F8642140230022802178686D
:10CC3C0001F037FA7B6801229A617B6840225A62C4
:10CC4C007B68012283F89C227B680022C3F8942223
:10CC5C007B6800225A607B680022C3F8A4227B68A0
:10CC6C00D3F8B832002B09D07B68D3F8B4325B68A8
:10CC7C007A685268D2B211467868984700231846F1
:10CC8C000837BD4680BD80B483B000AF78600B46DA
:10CC9C00FB707B68FA781A74002318460C37BD4673
:10CCAC0080BC704780B483B000AF78607B6893F829
:10CCBC009C227B6883F89D227B68042283F89C224B
:10CCCC00002318460C37BD4680BC704780B483B037
:10CCDC0000AF78607B6893F89C32042B05D17B689D
:10CCEC0093F89D227B6883F89C22002318460C370E
:10CCFC00BD4680BC704780B582B000AF78607B6861
:10CD0C0093F89C32032B0BD17B68D3F8B432DB69DC
:10CD1C00002B05D07B68D3F8B432DB697868984770
:10CD2C00002318460837BD4680BD000080B584B08E
:10CD3C0000AF786039600023FB733B681B7803F00D
:10CD4C006003402B05D0402B4FD8002B09D0202B53
:10CD5C004BD17B68D3F8B4329B68396878689847B4
:10CD6C0048E03B685B78092B39D801A252F823F0D4
:10CD7C00CDCD0008E1CD0008EBCD0008D7CD0008E3
:10CD8C00EBCD0008AFCD0008A5CD0008EBCD000819
:10CD9C00C3CD0008B9CD00083968786800F0DCF91B
:10CDAC0022E03968786800F03FFB1DE0396878684C
:10CDBC0000F07EFB18E03968786800F007FC13E09F
:10CDCC003968786800F037FC0EE03968786800F054
:10CDDC0065FC09E03968786800F074FC04E0396897
:10CDEC00786800F0C9FC00BF04E03968786800F08E
:10CDFC00C3FC00BFFB7B18461037BD4680BD00BF8F
:10CE0C0080B584B000AF786039600023FB733B6859
:10CE1C001B7803F06003402B05D0402B2ED8002B41
:10CE2C0001D0202B2AD17B6893F89C32013B022B3A
:10CE3C001DD83B689B88DBB2012B13D87B68D3F8D9
:10CE4C00B4329B683968786898470346FB733B6833
:10CE5C00DB88002B10D1FB7B002B0DD1786800F008
:10CE6C0053FD09E03968786800F086FC04E0396805
:10CE7C00786800F081FC00E000BF04E03968786855
:10CE8C0000F07AFC00BF002318461037BD4680BD69
:10CE9C0080B584B000AF786039600023FB733B68C9
:10CEAC009B88BB733B681B7803F06003402B07D057
:10CEBC00402B00F24681002B0AD0202B40F0418100
:10CECC007B68D3F8B4329B683968786898473DE141
:10CEDC003B681B7803F06003202B0AD17B68D3F8E6
:10CEEC00B4329B683968786898470346FB73FB7BC0
:10CEFC002DE13B685B78032B07D0032B00F31B81E0
:10CF0C00002B72D0012B3AD015E17B6893F89C3240
:10CF1C00022B02D0032B15D02BE0BB7B002B0CD0AB
:10CF2C00BB7B802B09D0BB7B1946786801F0FEF8DF
:10CF3C008021786801F0FAF820E03968786800F010
:10CF4C001BFC1BE03B685B88002B0ED1BB7B002BD2
:10CF5C000BD0BB7B802B08D03B68DB88002B04D12B
:10CF6C00BB7B1946786801F0E1F8786800F0CCFCDE
:10CF7C0004E03968786800F0FFFB00BFE0E07B68F4
:10CF8C0093F89C32022B02D0032B15D026E0BB7BEE
:10CF9C00002B0CD0BB7B802B09D0BB7B194678684F
:10CFAC0001F0C4F88021786801F0C0F81CE0396801
:10CFBC00786800F0E1FB17E03B685B88002B12D12E
:10CFCC00BB7B03F07F03002B04D0BB7B1946786836
:10CFDC0001F0CBF8786800F097FC04E039687868C9
:10CFEC0000F0CAFB00E000BFAAE07B6893F89C321B
:10CFFC00022B02D0032B32D097E0BB7B002B07D047
:10D00C00BB7B802B04D03968786800F0B5FB91E0CD
:10D01C0097F90E30002B0BDABB7B03F07F02134623
:10D02C009B0013449B0010337A68134404330BE0C9
:10D03C00BB7B03F07F0213469B0013449B0003F55C
:10D04C00A8737A6813440433BB60BB6800221A606F
:10D05C00BB6802221946786800F0F8FB6AE097F981
:10D06C000E30002B11DABB7B03F00F0279681346EC
:10D07C009B0013449B000B4418331B68002B17D1E7
:10D08C003968786800F078FB54E0BB7B03F00F0242
:10D09C00796813469B0013449B000B4403F5AC7357
:10D0AC001B68002B04D13968786800F065FB41E0FF
:10D0BC0097F90E30002B0BDABB7B03F07F02134683
:10D0CC009B0013449B0010337A68134404330BE029
:10D0DC00BB7B03F07F0213469B0013449B0003F5BC
:10D0EC00A8737A6813440433BB60BB7B002B02D05B
:10D0FC00BB7B802B03D1BB6800221A600EE0BB7B8C
:10D10C001946786801F050F80346002B03D0BB6831
:10D11C0001221A6002E0BB6800221A60BB6802227E
:10D12C001946786800F092FB04E03968786800F0E2
:10D13C0023FB00BF04E03968786800F01DFB00BFDA
:10D14C0004E03968786800F017FB00BFFB7B1846D9
:10D15C001037BD4680BD000080B584B000AF78604C
:10D16C00396000233B810023FB600023FB723B688A
:10D17C005B881B0A9BB2013B062B00F2288101A2A3
:10D18C0052F823F0ADD10008C5D1000805D2000833
:10D19C00DBD30008DBD300087BD30008A7D300083F
:10D1AC007B68D3F8B0321B687A68127C07F10801EF
:10D1BC0010469847F86012E17B681B7C002B0DD160
:10D1CC007B68D3F8B4329B6A07F108021046984783
:10D1DC00F860FB68013302221A7000E17B68D3F817
:10D1EC00B432DB6A07F1080210469847F860FB6816
:10D1FC00013302221A70F2E03B685B88DBB2052B2C
:10D20C0000F2AC8001A252F823F000BF31D200082A
:10D21C0065D2000899D20008CDD2000801D30008CD
:10D22C0035D300087B68D3F8B0325B68002B0BD089
:10D23C007B68D3F8B0325B687A68127C07F108011E
:10D24C0010469847F86091E03968786800F094FAD5
:10D25C00FB7A0133FB7289E07B68D3F8B0329B68B0
:10D26C00002B0BD07B68D3F8B0329B687A68127CA9
:10D27C0007F1080110469847F86077E0396878683C
:10D28C0000F07AFAFB7A0133FB726FE07B68D3F81B
:10D29C00B032DB68002B0BD07B68D3F8B032DB6884
:10D2AC007A68127C07F1080110469847F8605DE037
:10D2BC003968786800F060FAFB7A0133FB7255E04C
:10D2CC007B68D3F8B0321B69002B0BD07B68D3F88A
:10D2DC00B0321B697A68127C07F108011046984736
:10D2EC00F86043E03968786800F046FAFB7A01335D
:10D2FC00FB723BE07B68D3F8B0325B69002B0BD040
:10D30C007B68D3F8B0325B697A68127C07F108014C
:10D31C0010469847F86029E03968786800F02CFAD4
:10D32C00FB7A0133FB7221E07B68D3F8B0329B6946
:10D33C00002B0BD07B68D3F8B0329B697A68127CD7
:10D34C0007F1080110469847F8600FE039687868D3
:10D35C0000F012FAFB7A0133FB7207E03968786847
:10D36C0000F00AFAFB7A0133FB7238E037E07B6895
:10D37C001B7C002B09D17B68D3F8B4325B6B07F1B3
:10D38C00080210469847F86029E03968786800F080
:10D39C00F3F9FB7A0133FB7221E07B681B7C002BD9
:10D3AC000DD17B68D3F8B4321B6B07F10802104621
:10D3BC009847F860FB68013307221A700FE0396850
:10D3CC00786800F0D9F9FB7A0133FB7207E0396811
:10D3DC00786800F0D1F9FB7A0133FB7200BFFB7A5D
:10D3EC00002B1CD13B89002B11D03B68DB88002B18
:10D3FC000DD03B68DA883B89934228BF13469BB219
:10D40C003B813B891A46F968786800F01FFA3B6843
:10D41C00DB88002B04D1786800F076FA00E000BFBE
:10D42C001037BD4680BD00BF80B584B000AF7860BA
:10D43C0039603B689B88002B30D13B68DB88002B24
:10D44C002CD13B685B887F2B28D83B685B88DBB290
:10D45C0003F07F03FB737B6893F89C32032B04D19E
:10D46C003968786800F088F91DE07B68FA7B83F8EE
:10D47C009E22FB7B1946786800F0C1FE786800F0AC
:10D48C0043FAFB7B002B04D07B68022283F89C229E
:10D49C0009E07B68012283F89C2204E039687868F3
:10D4AC0000F06AF900BF00BF1037BD4680BD000018
:10D4BC0080B582B000AF786039603B685B88DAB2C7
:10D4CC00414B1A70404B1B78012B04D93968786892
:10D4DC0000F052F975E07B6893F89C32022B02D075
:10D4EC00032B23D062E0384B1B78002B1AD0364B21
:10D4FC001B781A467B685A607B68032283F89C224F
:10D50C00314B1B7819467868FFF7E7F90346022B75
:10D51C0004D13968786800F02FF952E0786800F08F
:10D52C00F3F94EE0786800F0EFF94AE0264B1B78EF
:10D53C00002B12D17B68022283F89C22224B1B7891
:10D54C001A467B685A60204B1B7819467868FFF79F
:10D55C00E3F9786800F0D8F933E01B4B1B781A46D6
:10D56C007B685B689A421DD07B685B68DBB21946AE
:10D57C007868FFF7D1F9144B1B781A467B685A6010
:10D58C00114B1B7819467868FFF7A7F90346022B55
:10D59C0004D13968786800F0EFF812E0786800F090
:10D5AC00B3F90EE0786800F0AFF90AE039687868F2
:10D5BC0000F0E2F8044B1B7819467868FFF7ACF9D9
:10D5CC0000BF0837BD4680BD9804002080B582B0EE
:10D5DC0000AF786039603B68DB88012B04D0396878
:10D5EC00786800F0C9F822E07B6893F89C32022B33
:10D5FC0002DC002B03DC15E0032B0BD012E07B6864
:10D60C0000229A607B68083301221946786800F082
:10D61C001DF90CE07B68043301221946786800F090
:10D62C0015F904E03968786800F0A6F800BF00BF6F
:10D63C000837BD4680BD80B582B000AF78603960D8
:10D64C007B6893F89C32013B022B1ED83B68DB882D
:10D65C00022B04D03968786800F08EF81AE07B68E9
:10D66C000122DA607B68D3F8A432002B05D07B68EA
:10D67C00DB6843F002027B68DA607B680C330222C1
:10D68C001946786800F0E2F804E03968786800F030
:10D69C0073F800BF00BF0837BD4680BD80B582B0AF
:10D6AC0000AF786039603B685B88012B06D17B68E2
:10D6BC000122C3F8A422786800F026F900BF0837CD
:10D6CC00BD4680BD80B582B000AF786039607B68A4
:10D6DC0093F89C32013B022B0BD83B685B88012BE7
:10D6EC000CD17B680022C3F8A422786800F00CF9F6
:10D6FC0004E03968786800F03FF800E000BF00BF34
:10D70C000837BD4680BD80B483B000AF7860396007
:10D71C003B681A787B681A703B685A787B685A7039
:10D72C003B6802331B781A463B6803331B781B0299
:10D73C009BB213449AB27B685A803B6804331B78C3
:10D74C001A463B6805331B781B029BB213449AB2F2
:10D75C007B689A803B6806331B781A463B68073314
:10D76C001B781B029BB213449AB27B68DA8000BF11
:10D77C000C37BD4680BC704780B582B000AF786076
:10D78C0039608021786800F0D1FC0021786800F0C5
:10D79C00CDFC00BF0837BD4680BD80B586B000AF5C
:10D7AC00F860B9607A600023FB75FB68002B32D0FF
:10D7BC00F86800F034F8034601339BB25B009AB270
:10D7CC007B681A80FB7D5A1CFA751A46BB68134499
:10D7DC007A6812781A70FB7D5A1CFA751A46BB6867
:10D7EC00134403221A7012E0FB685A1CFA60FA7D8B
:10D7FC00511CF9751146BA680A441B781370FB7DED
:10D80C005A1CFA751A46BB68134400221A70FB683E
:10D81C001B78002BE8D100BF1837BD4680BD80B403
:10D82C0085B000AF78600023FB7305E0FB7B013310
:10D83C00FB737B6801337B607B681B78002BF5D115
:10D84C00FB7B18461437BD4680BC704780B584B04E
:10D85C0000AFF860B9601346FB80FB680222C3F886
:10D86C009422FA88FB68DA61FA88FB681A62FB88F2
:10D87C00BA680021F86800F0E1FC00231846103764
:10D88C00BD4680BD80B584B000AFF860B96013466A
:10D89C00FB80FB88BA680021F86800F0CFFC0023FD
:10D8AC0018461037BD4680BD80B584B000AFF86017
:10D8BC00B9601346FB80FB680322C3F89422FA88F4
:10D8CC00FB68C3F85C21FA88FB68C3F86021FB880D
:10D8DC00BA680021F86800F0D4FC00231846103711
:10D8EC00BD4680BD80B584B000AFF860B96013460A
:10D8FC00FB80FB88BA680021F86800F0C2FC0023AA
:10D90C0018461037BD4680BD80B582B000AF786038
:10D91C007B680422C3F8942200230022002178683B
:10D92C0000F08CFC002318460837BD4680BD80B53E
:10D93C0082B000AF78607B680522C3F89422002384
:10D94C0000220021786800F09CFC00231846083760
:10D95C00BD4680BD80B500AF002212491248FEF7CB
:10D96C0062FF0346002B01D0F5F76CFE0F490E4801
:10D97C00FEF784FF0346002B01D0F5F763FE0C493C
:10D98C000948FEF7B5FE0346002B01D0F5F75AFE09
:10D99C000548FEF78CFF0346002B01D0F5F752FE2D
:10D9AC0000BF80BD3C0100209C040020280000200A
:10D9BC002C01002080B485B000AF786039601EE087
:10D9CC00144B1B889BB201339BB2DBB2FB81FA89EF
:10D9DC00114B1B889BB2DBB29A4203D17B6801339B
:10D9EC007B600CE07B685A1C7A600A4A128892B2FF
:10D9FC00D2B21978094B9954064AFB8913803B68BB
:10DA0C005A1E3A60002BDBD100BF00BF1437BD4655
:10DA1C0080BC70476010002062100020600F002056
:10DA2C0080B400AF064B1B889AB2064B1B889BB286
:10DA3C00D31A9BB2DBB21846BD4680BC704700BF00
:10DA4C00601000206210002080B483B000AF104B37
:10DA5C001B889AB20F4B1B889BB29A4202D14FF093
:10DA6C00FF3310E00A4B1B889BB2DBB20A4AD35C33
:10DA7C007B60074B1B889BB201339BB2DBB29AB223
:10DA8C00034B1A807B6818460C37BD4680BC704728
:10DA9C006210002060100020600F002080B500AFE5
:10DAAC00002205490548FEF739FE05490348FEF7F3
:10DABC004EFE0023184680BD600B00209C04002005
:10DACC006007002080B400AF00231846BD4680BC20
:10DADC007047000080B483B000AF03463960FB711F
:10DAEC001346BB80FB79232B4AD801A252F823F0B2
:10DAFC008DDB00088DDB00088DDB00088DDB00085A
:10DB0C008DDB00088DDB00088DDB00088DDB000849
:10DB1C008DDB00088DDB00088DDB00088DDB000839
:10DB2C008DDB00088DDB00088DDB00088DDB000829
:10DB3C008DDB00088DDB00088DDB00088DDB000819
:10DB4C008DDB00088DDB00088DDB00088DDB000809
:10DB5C008DDB00088DDB00088DDB00088DDB0008F9
:10DB6C008DDB00088DDB00088DDB00088DDB0008E9
:10DB7C008DDB00088DDB00088DDB00088DDB0008D9
:10DB8C0000BF002318460C37BD4680BC704700BF51
:10DB9C0080B582B000AF786039603B681B68002BA1
:10DBAC0005D03B681B6819467868FFF703FF796856
:10DBBC000548FEF7CCFD0448FEF70BFE0023184683
:10DBCC000837BD4680BD00BF9C04002080B584B0E2
:10DBDC0000AF78600B467B800023FB730D4BD3F8B2
:10DBEC00B832BB60BB68D3F81432002B01D00123D0
:10DBFC000BE07B881A4679680648FEF78FFD0548CE
:10DC0C00FEF7B8FD0346FB73FB7B18461037BD4689
:10DC1C0080BD00BF9C04002080B483B000AF0346DD
:10DC2C003960FB713B6812221A80034B18460C3783
:10DC3C00BD4680BC704700BF5801002080B483B043
:10DC4C0000AF03463960FB713B6804221A80034B1A
:10DC5C0018460C37BD4680BC704700BF6C010020D5
:10DC6C0080B582B000AF03463960FB71FB79002BA5
:10DC7C0005D13A6807490848FFF78FFD04E03A6878
:10DC8C0004490548FFF789FD024B18460837BD4685
:10DC9C0080BD00BF6410002050F3000880B582B036
:10DCAC0000AF03463960FB713A6804490448FFF73A
:10DCBC0074FD024B18460837BD4680BD6410002029
:10DCCC0068F3000880B582B000AF03463960FB7181
:10DCDC003B681A221A8000F043F8024B18460837AA
:10DCEC00BD4680BD7001002080B582B000AF0346F8
:10DCFC003960FB71FB79002B05D13A68074908485C
:10DD0C00FFF74BFD04E03A6804490548FFF745FD71
:10DD1C00024B18460837BD4680BD00BF641000207A
:10DD2C007CF3000880B582B000AF03463960FB710C
:10DD3C00FB79002B05D13A6807490848FFF72DFD00
:10DD4C0004E03A6804490548FFF727FD024B1846E2
:10DD5C000837BD4680BD00BF6410002088F3000862
:10DD6C0080B584B000AF0F4B1B68FB600E4B1B687B
:10DD7C00BB600E4B1B687B60FA687B681344FB60CE
:10DD8C00FB68002B09D008220949F86800F014F848
:10DD9C0004220849B86800F00FF800BF1037BD46E0
:10DDAC0080BD00BFE8F7FF1FECF7FF1FF0F7FF1F68
:10DDBC00720100208201002080B487B000AFF860AF
:10DDCC00B9601346FB710023FB750023FB7527E03C
:10DDDC00FB681B0F092B0BD8FB681B0FDAB2FB7D02
:10DDEC005B001946BB680B443032D2B21A700AE0A1
:10DDFC00FB681B0FDAB2FB7D5B001946BB680B445A
:10DE0C003732D2B21A70FB681B01FB60FB7D5B00E2
:10DE1C000133BA68134400221A70FB7D0133FB7581
:10DE2C00FA7DFB799A42D3D300BF00BF1C37BD46A5
:10DE3C0080BC704780B584B000AF78607B681B688D
:10DE4C000D4A934213D10D4BDB690C4A43F400038A
:10DE5C00D3610A4BDB6903F40003FB60FB6800220F
:10DE6C0000211420F7F7DBFD1420F7F7F4FD00BFB9
:10DE7C001037BD4680BD00BF005C00400010024062
:10DE8C0080B582B000AF78607B68D3F8D4227B6811
:10DE9C0003F5267319461046FEF751FD00BF0837EF
:10DEAC00BD4680BD80B582B000AF78600B46FB707C
:10DEBC007B68D3F8D402FA78796813469B00134434
:10DECC00DB000B4403F5B2731A68FB781946FEF7B6
:10DEDC0083FD00BF0837BD4680BD80B582B000AF62
:10DEEC0078600B46FB707B68D3F8D402FA787968BB
:10DEFC0013469B001344DB000B4424331A68FB7855
:10DF0C001946FEF7DAFD00BF0837BD4680BD80B567
:10DF1C0082B000AF78607B68D3F8D4321846FEF735
:10DF2C00EAFE00BF0837BD4680BD80B584B000AFA7
:10DF3C0078600123FB737B689B79022B01D0F5F78A
:10DF4C0081FB7B68D3F8D432FA7B11461846FEF776
:10DF5C009AFE7B68D3F8D4321846FEF753FE00BF06
:10DF6C001037BD4680BD000080B582B000AF786030
:10DF7C007B68D3F8D4321846FEF794FE7B689B7A04
:10DF8C00002B05D0044B1B69034A43F006031361B5
:10DF9C0000BF0837BD4680BD00ED00E080B582B003
:10DFAC0000AF78607B68D3F8D4321846FEF78EFE4B
:10DFBC0000BF0837BD4680BD80B582B000AF786029
:10DFCC00284A7B68C2F8D4327B68264AC3F8C02240
:10DFDC00244B254A1A60234B08221A71214B02222A
:10DFEC009A71204B00229A721E4B0022DA721D4B42
:10DFFC0000221A731B48F8F7F0FA0346002B01D0E5
:10E00C00F5F720FB7B68D3F8C0021823002200210F
:10E01C00FAF701F87B68D3F8C0025823002280215C
:10E02C00F9F7F9FF7B68D3F8C002C02300228121E5
:10E03C00F9F7F1FF7B68D3F8C0024FF48873002224
:10E04C000121F9F7E8FF7B68D3F8C0024FF4807325
:10E05C0000228221F9F7DFFF002318460837BD465E
:10E06C0080BD00BF64120020005C004080B584B00D
:10E07C0000AF78600023FB730023BB737B68D3F87D
:10E08C00C0321846F8F79FFB0346FB73FB7B184620
:10E09C0000F04EF90346BB73BB7B18461037BD46E8
:10E0AC0080BD80B584B000AF7860084611461A4632
:10E0BC000346FB700B46BB7013463B800023FB737F
:10E0CC000023BB737B68D3F8C002BB783A88F9781D
:10E0DC00F8F7F3FC0346FB73FB7B184600F028F9BA
:10E0EC000346BB73BB7B18461037BD4680BD80B55D
:10E0FC0084B000AF78600B46FB700023FB730023E9
:10E10C00BB737B68D3F8C032FA7811461846F8F71F
:10E11C0031FD0346FB73FB7B184600F009F90346FF
:10E12C00BB73BB7B18461037BD4680BD80B584B031
:10E13C0000AF78600B46FB700023FB730023BB73AE
:10E14C007B68D3F8C032FA7811461846F8F7D9FD37
:10E15C000346FB73FB7B184600F0EAF80346BB73DF
:10E16C00BB7B18461037BD4680BD80B584B000AF70
:10E17C0078600B46FB700023FB730023BB737B683A
:10E18C00D3F8C032FA7811461846F8F71AFE03464F
:10E19C00FB73FB7B184600F0CBF80346BB73BB7BD1
:10E1AC0018461037BD4680BD80B485B000AF78608E
:10E1BC000B46FB707B68D3F8C032FB6097F90330D9
:10E1CC00002B0BDAFB7803F07F02F96813469B00F7
:10E1DC001344DB000B4412331B780BE0FB7803F089
:10E1EC007F02F96813469B001344DB000B4403F5D4
:10E1FC00A9731B7818461437BD4680BC704780B590
:10E20C0084B000AF78600B46FB700023FB730023D7
:10E21C00BB737B68D3F8C032FA7811461846F8F70E
:10E22C0028FC0346FB73FB7B184600F081F8034681
:10E23C00BB73BB7B18461037BD4680BD80B586B01E
:10E24C0000AFF8607A601A460B46FB7213463B81AE
:10E25C000023FB750023BB75FB68D3F8C0023B8918
:10E26C00F97A7A68F8F716FD0346FB75FB7D1846BC
:10E27C0000F05EF80346BB75BB7D18461837BD46EB
:10E28C0080BD80B586B000AFF8607A601A460B4648
:10E29C00FB7213463B810023FB750023BB75FB68A7
:10E2AC00D3F8C0023B89F97A7A68F8F7ABFC0346DD
:10E2BC00FB75FB7D184600F03BF80346BB75BB7D38
:10E2CC0018461837BD4680BD80B582B000AF786067
:10E2DC000B46FB707B68D3F8C032FA7811461846AF
:10E2EC00F8F7C1FC034618460837BD4680BD000050
:10E2FC0080B483B000AF7860024B18460C37BD4633
:10E30C0080BC70473C15002080B483B000AF7860AF
:10E31C0000BF0C37BD4680BC704780B483B000AFE3
:10E32C0078600B46FB7000BF0C37BD4680BC704755
:10E33C0080B485B000AF0346FB710023FB73FB79FF
:10E34C00032B17D801A252F823F000BF69E3000891
:10E35C006FE3000875E300087BE300080023FB7300
:10E36C000BE00223FB7308E00123FB7305E002239F
:10E37C00FB7302E00223FB7300BFFB7B18461437D0
:10E38C00BD4680BC704700BF0EB46FF0004110B5A5
:10E39C0000249DB01FAB0290069007910491094890
:10E3AC00094953F8042B0591006802A901931B94A9
:10E3BC0000F092F9029B1C701DB0BDE8104003B038
:10E3CC00704700BF8C0100200802FFFF0346024487
:10E3DC00934200D1704703F8011BF9E7014B186811
:10E3EC00704700BF8C01002070B500260C4D0D4C01
:10E3FC00641BA410A64209D100F076FC00260A4D3D
:10E40C000A4C641BA410A64205D170BD55F8043B00
:10E41C0098470136EEE755F8043B98470136F2E78A
:10E42C0000F5000800F5000800F5000804F50008E8
:10E43C007047704738B50546002940D051F8043C68
:10E44C000C1F002BB8BFE41800F0DEF81C4A136850
:10E45C0033B9636014602846BDE8384000F0DAB880
:10E46C00A34208D9206821188B4201BF19685B6848
:10E47C0009182160EDE71A465B680BB1A342FAD983
:10E48C0011685018A0420BD12068014450188342E7
:10E49C001160E0D118685B68084410605360DAE7DB
:10E4AC0002D90C232B60D6E7206821188B4201BFC0
:10E4BC0019685B680918216063605460CBE738BD4C
:10E4CC00A018002070B50F4E0C463168054611B9E6
:10E4DC0000F0A8FB30602146284600F0A3FB431C4B
:10E4EC0003D14FF0FF34204670BDC41C24F003044C
:10E4FC00A042F8D0211A284600F094FB0130F2D14A
:10E50C00EFE700BF9C1800202DE9F843CD1C25F047
:10E51C00030508350C2D38BF0C25002D064601DBF4
:10E52C00A94204D90C2333600020BDE8F883DFF83E
:10E53C00D48000F069F8D8F800301C4644BB29465A
:10E54C003046FFF7BFFF431C044658D1D8F80040B3
:10E55C002746002F43D1002C4BD023683946304638
:10E56C0004EB030900F05EFB814542D12168304683
:10E57C006D1A2946FFF7A6FF01303AD023682B44C9
:10E58C002360D8F800305A6862BBC8F800700FE0FE
:10E59C002268521B20D40B2A17D96119A34225607B
:10E5AC0018BF5960636808BFC8F8001062514B600F
:10E5BC00304600F02FF804F10B00231D20F007006B
:10E5CC00C21A1CBF1B1AA350AFE76268A3420CBF50
:10E5DC00C8F800205A60EBE723466468AEE73C4677
:10E5EC007F68B6E71A465B68A342FBD100235360F1
:10E5FC00DEE70C233046336000F00CF894E705603E
:10E60C00D6E700BFA01800200148FFF711BF00BFDC
:10E61C00981800200148FFF70CBF00BF9818002085
:10E62C002DE9F0471F468E688246BE420C46904646
:10E63C000B682DD8B1F90C2012F4906F26D06569B7
:10E64C00096905EB4505A3EB010905EBD5757B1CA9
:10E65C004B446D109D4238BF1D46530527D52946A6
:10E66C00FFF752FF064660B34A46216900F0F8FAFC
:10E67C00A38923F4906343F08003A38126614E4465
:10E68C0026603E466561A5EB0905A560BE4200D932
:10E69C003E4632464146206800F0AAFA0020A368A4
:10E6AC009B1BA360236833442360BDE8F0872A4694
:10E6BC0000F0E4FA06460028E0D150462169FFF745
:10E6CC00B9FE0C23CAF80030A3894FF0FF3043F099
:10E6DC004003A381E9E700002DE9F04F98468B89B0
:10E6EC0007461B060D4614469DB010D50B6973B931
:10E6FC004021FFF709FF2860286130B90C233B60EB
:10E70C004FF0FF301DB0BDE8F08F40236B6100234C
:10E71C00099320238DF8293030234FF00109CDF8CF
:10E72C000C80DFF898818DF82A3023469A4613F82E
:10E73C00012B0AB1252AF9D1BAEB040B0BD05B469D
:10E74C00224629463846FFF76BFF013000F0A780C0
:10E75C00099A5A4409929AF80030002B00F09F80D5
:10E76C0000234FF0FF32CDE905230AF1010A04938F
:10E77C0007938DF853301A935446052214F8011B55
:10E78C004E4800F05FFA049AD8B9D00644BF202353
:10E79C008DF85330110744BF2B238DF853309AF862
:10E7AC0000302A2B15D0544600204FF00A0C079A43
:10E7BC00214611F8013B303B092B4BD9B0B10792E4
:10E7CC0014E0A0EB080309FA03F31343A2460493E5
:10E7DC00D2E7039B191D1B680391002BBBBF5B4247
:10E7EC0042F0020207930793B8BF049223782E2BB2
:10E7FC000AD163782A2B32D1039B02341A1D1B6871
:10E80C00039243EAE3730593DFF8B4A00322504666
:10E81C00217800F017FA38B14022049BA0EB0A00D3
:10E82C00824013430134049314F8011B062225483B
:10E83C008DF8281000F006FA002836D0224B1BBBAE
:10E84C00039B073323F0070308330393099B3344DB
:10E85C0009936AE70C4601200CFB0232A8E700235F
:10E86C004FF00A0C194601340593204610F8012B81
:10E87C00303A092A03D9002BC6D00591C4E70446C7
:10E88C0001230CFB0121F0E703AB00932A46384629
:10E89C000E4B04A9AFF30080421C0646D6D1AB89BF
:10E8AC005B063FF52DAF09982CE703AB00932A4686
:10E8BC003846064B04A900F07DF8EDE7C2F40008D9
:10E8CC00C8F40008CCF40008000000002DE6000895
:10E8DC002DE9F047164698468A680B69074693421D
:10E8EC00B8BF1346336091F843200C46DDF82090F6
:10E8FC000AB1013333602368990642BF336802338F
:10E90C003360256815F0060506D104F1190AE36891
:10E91C0032689B1AAB422BDC94F843302268003BE4
:10E92C0018BF0123920630D44146384604F1430205
:10E93C00C847013023D02368226903F00603042B57
:10E94C0014BF002533684FF0000608BFE56804F1DA
:10E95C001A0408BFED1A54F8123C08BF25EAE575F5
:10E96C009342C4BF9B1AED18B5421AD1002008E09F
:10E97C000123524641463846C847013003D14FF077
:10E98C00FF30BDE8F0870135C1E73020E11881F890
:10E99C0043005A1C94F845102244023382F8431069
:10E9AC00C2E70123224641463846C8470130E6D02B
:10E9BC000136D9E72DE9FF470F7E9146782F804627
:10E9CC000C469A460C9E01F1430207D8622F0AD8D6
:10E9DC00002F00F0D180582F00F0B88004F14206CF
:10E9EC0084F842703AE0A7F16303152BF6D801A125
:10E9FC0051F823F059EA00086DEA0008E9E900082B
:10EA0C00E9E90008E9E90008E9E900086DEA00080D
:10EA1C00E9E90008E9E90008E9E90008E9E9000882
:10EA2C006BEB000897EA000825EB0008E9E9000801
:10EA3C00E9E900088DEB0008E9E9000897EA00080D
:10EA4C00E9E90008E9E900082DEB000833681A1D14
:10EA5C001B68326004F1420684F8423001239CE0CA
:10EA6C0033682068191D3160060601D51D6803E066
:10EA7C004506FBD5B3F90050002D03DA2D236D426A
:10EA8C0084F843300A23584811E02168336808069B
:10EA9C0053F8045B02D4490648BFADB26F2F336004
:10EAAC0014BF0A2308235048002184F843106668D9
:10EABC00002EA66005DB21682E4321F004012160A5
:10EACC004BD01646B5FBF3F103FB1157C75D06F8A7
:10EADC00017D2F46BB420D46F4D9082B0BD1236880
:10EAEC00DF0708D5236961689942DEBF302306F839
:10EAFC00013C06F1FF36921B22614B4621464046F3
:10EB0C00CDF800A003AAFFF7E3FE01304AD14FF085
:10EB1C00FF3004B0BDE8F087236843F02003236086
:10EB2C007827324884F84570236831681F0651F8FD
:10EB3C00045B02D45F0648BFADB23160D90744BF55
:10EB4C0043F0200323601DB11023ADE72648E9E70D
:10EB5C00236823F020032360F6E71646BDE73368ED
:10EB6C002568181D616930602E061B6801D5196077
:10EB7C0002E06806FBD51980002316462361BCE72A
:10EB8C00336800211A1D32601E686268304600F03E
:10EB9C0059F808B1801B606063682361002384F816
:10EBAC004330AAE73246494640462369D0470130F4
:10EBBC00ADD023689B0713D4E068039B9842B8BF81
:10EBCC001846A6E70123324649464046D047013055
:10EBDC009DD00135E36803995B1AAB42F2DCEBE79D
:10EBEC00002504F11906F5E7D3F40008E4F4000855
:10EBFC00884210B501EB020402D98442234607D89F
:10EC0C00431EA14208D011F8012B03F8012FF8E79D
:10EC1C00014602448A4200D110BD13F8014D02F89E
:10EC2C00014DF7E738B50023054D044608462B6027
:10EC3C00F6F78EF9431C02D12B6803B1236038BD63
:10EC4C0094180020034610B5C9B2024493421846EA
:10EC5C0001D1002003E0047801338C42F6D110BDC1
:10EC6C000A44914200F1FF3300D1704710B511F8FE
:10EC7C00014B914203F8014FF9D110BD2DE9F04140
:10EC8C00074614460D4621B91146BDE8F041FFF781
:10EC9C003BBC2AB9FFF7CEFB25462846BDE8F081E0
:10ECAC0000F01AF88442064602D8B4EB500FF4D8A0
:10ECBC0021463846FFF728FC804608B94546ECE764
:10ECCC00B4422246294628BF3246FFF7C9FF2946DF
:10ECDC003846FFF7AFFBF1E751F8043C181F002B47
:10ECEC00BCBF0B58C0187047F8B500BFF8BC08BCC7
:10ECFC009E467047F8B500BFF8BC08BC9E467047EE
:10ED0C00696E666F0A0000000A70776D2025642515
:10ED1C00642564256425642564256425640000004D
:10ED2C000A3078256C78203078256C78203078255E
:10ED3C006C78203078256C78203078256C782030F1
:10ED4C0078256C78203078256C78203078256C7894
:10ED5C00000000000A503D30782578206368343D6F
:10ED6C0025303564206368353D2530356420636873
:10ED7C00363D25303564206368373D2530356420B9
:10ED8C006368383D25303564000000000A73744315
:10ED9C0069636C6F3D2530356420737450756C73EA
:10EDAC00616E74693D253035640000000A494430B9
:10EDBC0030303030300000000A62307C310000000E
:10EDCC000A3F6D6E73767676767620733D667C623E
:10EDDC00000000000A3F6D6E7376767676762030F2
:10EDEC00303030303E3D76767676763C3D3939396A
:10EDFC00393900000A3F6D6E73767676767620315F
:10EE0C003E3D6D3C3D3400000A3F6D6E7376767668
:10EE1C00767600000A6565203078253032783D30F2
:10EE2C0078253034780000000A65652072656164CD
:10EE3C00206572726F722025640000000A3F6572B3
:10EE4C006161206865782076616C756573000000DF
:10EE5C000A3F6572616100000A646F6E652030784C
:10EE6C00253032783D307825303478000A656520BD
:10EE7C007772697465206572726F72202564000068
:10EE8C000A3F6577616176767676206865782076BC
:10EE9C00616C7565730000000A3F657761612068DD
:10EEAC0065782076616C7565730000000A3F6577A4
:10EEBC0061617676767600000A3078253032783DBE
:10EECC002535642000000000726465727220256490
:10EEDC00200000000A0000000A3F656400000000EA
:10EEEC000A3F6578000000000A6D3170776D617023
:10EEFC003D2564206D3170776D63683D2564206D10
:10EF0C003270776D61703D2564206D3270776D6362
:10EF1C00683D2564206D3370776D61703D256420EC
:10EF2C006D3370776D63683D2564206D3470776D3B
:10EF3C0061703D2564206D3470776D63683D256488
:10EF4C00000000000A6D3154696D656F75744D6178
:10EF5C006E3D2564206D3254696D656F75744D611D
:10EF6C006E3D2564206D3354696D656F75744D610C
:10EF7C006E3D2564206D3454696D656F75744D61FB
:10EF8C006E3D2564200000000A7472616D703D2591
:10EF9C0064207472616D706D616E3D2564000000BB
:10EFAC000A6D3170776D4D616E3D2564206D327048
:10EFBC00776D4D616E3D2564206D3370776D4D61BD
:10EFCC006E3D2564206D3470776D4D616E3D25640A
:10EFDC00000000000A61704D3173746172743D253C
:10EFEC00642061704D3173746F703D2564206368CB
:10EFFC004D3173746172743D25642063684D3173B7
:10F00C00746F703D256400000A61704D3273746139
:10F01C0072743D25642061704D3273746F703D25A0
:10F02C00642063684D3273746172743D256420638F
:10F03C00684D3273746F703D256400000A61704D29
:10F04C003373746172743D25642061704D33737435
:10F05C006F703D25642063684D3373746172743D29
:10F06C0025642063684D3373746F703D2564000014
:10F07C000A61704D3473746172743D256420617043
:10F08C004D3473746F703D25642063684D34737414
:10F09C006172743D25642063684D3473746F703DE8
:10F0AC00256400000A3F6576000000000A3F657287
:10F0BC007C777C647C787C76000000000A3F65726B
:10F0CC006161207C20657761617676767600000040
:10F0DC000A3F00000A70756C73616E74693D2558A7
:10F0EC00000000000A737470756C73616E74693D76
:10F0FC00255800000A73744369636C6F3D256400E6
:10F10C000A646F6E652025643D2564000A656520E0
:10F11C007772697465206572726F722025640000C5
:10F12C004C6F616445450A000A6D3170776D6170F2
:10F13C003D2564206D3170776D63683D2564206DCD
:10F14C003270776D61703D2564206D3270776D6320
:10F15C00683D2564206D3370776D61703D256420AA
:10F16C006D3370776D63683D2564206D3470776DF9
:10F17C0061703D2564206D3470776D63683D256446
:10F18C00000000000A6D3154696D656F75744D6136
:10F19C006E3D2564206D3254696D656F75744D61DB
:10F1AC006E3D2564206D3354696D656F75744D61CA
:10F1BC006E3D2564206D3454696D656F75744D61B9
:10F1CC006E3D2564200000000A7472616D703D254F
:10F1DC0064207472616D706D616E3D256400000079
:10F1EC000A6D3170776D4D616E3D2564206D327006
:10F1FC00776D4D616E3D2564206D3370776D4D617B
:10F20C006E3D2564206D3470776D4D616E3D2564C7
:10F21C00000000000A61704D3173746172743D25F9
:10F22C00642061704D3173746F703D256420636888
:10F23C004D3173746172743D25642063684D317374
:10F24C00746F703D256400000A61704D32737461F7
:10F25C0072743D25642061704D3273746F703D255E
:10F26C00642063684D3273746172743D256420634D
:10F27C00684D3273746F703D256400000A61704DE7
:10F28C003373746172743D25642061704D337374F3
:10F29C006F703D25642063684D3373746172743DE7
:10F2AC0025642063684D3373746F703D25640000D2
:10F2BC000A61704D3473746172743D256420617001
:10F2CC004D3473746F703D25642063684D347374D2
:10F2DC006172743D25642063684D3473746F703DA6
:10F2EC00256400000A6D3161703D2564000000004A
:10F2FC000A6D3261703D2564000000000A6D3361B7
:10F30C00703D2564000000000A6D3461703D256479
:10F31C00000000000A6D3163683D256400000000A8
:10F32C000A6D3263683D2564000000000A6D33638A
:10F33C00683D2564000000000A6D3463683D256457
:10F34C000000000053544D333220566972747561BD
:10F35C006C20436F6D506F727400000053544D69F4
:10F36C0063726F656C656374726F6E6963730000B2
:10F37C0043444320436F6E66696700004344432057
:10F38C00496E7465726661636500000028003C007C
:10F39C004600460023002800280028001400140012
:10F3AC0014001400E600640082002C0101001B0014
:10F3BC000A001E0001000100000000000001140002
:10F3CC003C0046002800280032000A003601C20129
:10F3DC001E0036015401AE011E00AE010A004001B0
:10F3EC008C00B801140018012800B80101001B00A2
:10F3FC000A001E0001000100000000000000640073
:10F40C003C004600280028003200080001000200E1
:10F41C0003000400050006000700080009000A00AC
:10F42C000B000C000D000E000F001000110012005C
:10F43C0013001400150016001700180019001A000C
:10F44C001B001C001D001E001F00200021002200BC
:10F45C0023002400250026002700280029002A006C
:10F46C002B002C002D002E002F003000310032001C
:10F47C0033003400350036003700380039003A00CC
:10F48C003B003C003D003E003F00400000000000FF
:10F49C000000000001020304060708090000000038
:10F4AC000102030402030405060708090A0B0C0DEC
:10F4BC000E0F10100102232D302B2000686C4C0015
:10F4CC006566674546470030313233343536373858
:10F4DC0039414243444546003031323334353637B6
:0CF4EC003839616263646566000000004E
:08F4F800540CFF7F010000002D
:04F5000031010008CD
:04F504000D010008ED
:10F5080000F80008C8C864040404040404040400DF
:10F5180000127A0010000000010000000A06000234
:10F52800000000400100000089C200087DC30008F7
:10F53800EBC30008000000002DC6000831C5000814
:10F54800D7C500080000000000000000000000000F
:10F558009DC600087DC60008BDC60008DDC60008B7
:10F5680009024300020100C032090400000102023E
:10F5780001000524001001052401000104240202F1
:10F58800052406000107058203080010090401008C
:10F59800020A0000000705010200020007058102B7
:10F5A8000002000009024300020100C03209040001
:10F5B80000010202010005240010010524010001D8
:10F5C800042402020524060001070582030800102E
:10F5D80009040100020A00000007050102400000BA
:10F5E800070581024000000009074300020104C02A
:10F5F800320904000001020201000524001001057F
:10F6080024010001042402020524060001070582E2
:10F618000308001009040100020A000000070501A0
:10F62800024000000705810240000000A9DA000836
:10F63800D1DA0008E1DA00089DDB000825DC0008C3
:10F6480049DC0008A9DC00086DDC0008D1DC0008F2
:10F65800F5DC000831DD000812010002020200405A
:10F668008304405700020102030100000403090457
:10F678001A03000000000000000000000000000065
:10F6880000000000000000000000000090010020C1
:10F69800000000005C170020C41700202C18002070
:10F6A8000000000000000000000000000000000052
:10F6B8000000000000000000000000000000000042
:10F6C8000000000000000000000000000000000032
:0CF6D80000000000000000000000000026
:0400000508004FD5CB
:00000001FF
